:100000000C940C0E0C94290E0C94290E0C94290EB1
:100010000C94290E0C942E100C9453120C94290E4F
:100020000C94290E0C94290E0C94290E0C94290E74
:100030000C94290E0C94290E0C942A240C94290E4D
:100040000C9475150C9464130C943E100C94F50FDD
:100050000C94290E0C94401F0C94290E0C94290E1C
:100060000C94290E0C94290E0C94290E0C94290E34
:100070000C94290E0C94D2240C9467120C94151233
:100080000C94290E0C94455C0C94290E8B565757F2
:10009000C65594566B57F8550E56B957B957B957B8
:1000A0002C56B957B957B957B957A8563757375774
:1000B0005357EC56EC56EA56E856E656B957B95738
:1000C000B957B957B957B957B9577B56B957B957EF
:1000D000B957B957B957B957B957B957B957B957A0
:1000E000B957B957B957B957B957B957B957B95790
:1000F000B957B957B957B957B957B957B957B95780
:10010000B957B957B957B957B957AA579C578A57CA
:100110006F5745617379436F6E74726F6C00204D39
:100120004300696E636F6D70617469626C6520482D
:100130005700312E342E32005F03AF01D7006B0021
:10014000470035001A0011000102031304050611CF
:10015000070809120A000B0C100F0E0D0101010512
:100160000D1F0C04040E1F04041F0E041F1F1F008C
:100170001F1F1F001F1F1F001F111F001F111F0027
:100180001F1F1F001F111F001F111F00000609174E
:1001900017090600000609121412090603070F1EAC
:1001A0001C18100003050912141810000707070790
:1001B0000707070707050505050505071C1018179C
:1001C000150705071C101817110202021C1018123F
:1001D000140605021C101817140601061C10181529
:1001E000150701011C101816110201061C10181623
:1001F000110204071C10181216020207040A110A41
:100200000A0E00000C17141714170C001C101810FD
:10021000160505051F0A0A0A0A0A1F000E11111FFA
:100220001B1B1F0002060F1F0F060200080C1E1FDB
:100230001E0C08000E0E0E0E1F0E0400040E1F0EE4
:100240000E0E0E0000C030F00CCC3CFC03C333F3A8
:100250000FCF3FFFC303F333CF0FFF3FAAC0803060
:10026000F0B020E0A00CCC8C3CFCBC2CECAC08C862
:100270008838F8B828E8A803C38333F3B323E3A38B
:100280000FCF8F3FFFBF2FEFAF0BCB8B3BFBBB2BBA
:10029000EBAB02C28232F2B222E2A20ECE8E3EFE60
:1002A000BE2EEEAE0ACA8A3AFABA2AEA004060972F
:1002B0007048685878446454744C6C5C7C42625258
:1002C000724A6A5A7A466656764E6E5E7E41615131
:1002D000714969597945659F754D6D5D7D436353DE
:1002E000734B6B5B7B476757774F6F5F7F101814BB
:1002F0001C121A161E1119151D131B171FD0D8D446
:10030000DCD2DAD6DED1D9D5DDD3DBD7DF90989435
:100310009C929A969E9199959D939B5055040605A3
:1003200007C4C6C5C78486858734363537F4F6F5E5
:10033000F7B4B6B5B724262527E4E6E5E7A4A6A5D5
:10034000A701C18131F1B121E1A10DCD8D3DFDBDEF
:100350002DEDAD09C98939F9B929E9A92020202055
:1003600020200000204D4D4920200000204D4D014F
:100370002020000020444343202000002053544FFD
:100380005020000053484F52542100002048414C57
:100390005420000000000000000000002050524FD8
:1003A0004720000052455345542000007E0E0E0E9B
:1003B0000E1B1B1C0E1B1B7E0E0E0E0E232D004152
:1003C00044523A20256C6420202020202020202028
:1003D00020002D2D2D2D202000252D3564002533C6
:1003E0006400202001022020202020202000252D34
:1003F000356400252D31312E313173000002070B99
:100400001014191D22262B3035393F43484C5156C4
:100410005B5F64696D72767B7F0002070C10151AB2
:100420001E23282C31363A3F44484D52565B6064B7
:10043000696E73797F00020C151D263039434C56C6
:100440005F69727F2530386C75005741524E494EB6
:10045000473A20004552524F523A200062616420D0
:10046000706172616D657465722076616C7565008E
:10047000706F776572206973204F666600747572BD
:100480006E6F75742071756575652066756C6C008E
:10049000636F6D6D616E642071756575652066753D
:1004A0006C6C006E6F2064617461006E6F20736C01
:1004B0006F7420617661696C61626C65006C6F6B52
:1004C000206275737900696C6C6567616C20747566
:1004D000726E6F757420616472657373004D432092
:1004E000696E2048414C54004D4320696E2053549E
:1004F0004F50004C207B4C6F6B232C205B5370655E
:1005000065645D2C205B464C5D2C205B4469725D0C
:100510002C205B46315D2C205B46325D2C205B46F7
:10052000335D2C205B46345D7D0054207B54726E1D
:1005300074232C205B436F6C6F725D2C205B5374B3
:10054000617475735D7D0046207B4C6F6B232C209E
:100550005B46315D2C205B46325D2C205B46335D73
:100560002C205B46345D2C205B46355D2C205B46A1
:10057000365D2C205B46375D2C205B46385D7D0068
:10058000484C2048656C7020666F72206C6F6B2041
:10059000636F6D6D616E64730D0048462048656C35
:1005A0007020666F722066756E6374696F6E20636B
:1005B0006F6D6D616E64730D0048542048656C70FA
:1005C00020666F72207475726E6F757420636F6D24
:1005D0006D616E647300507772206F6666004861CB
:1005E0006C7465642100507772206F6E0044434341
:1005F0002070726F6772616D005245534554004818
:10060000616C746564210D5D004C20257520257595
:100610002025632025632025632025632025632072
:10062000256300756E75736564004D6F746F726F2E
:100630006C61204F6C64004D6F746F726F6C612041
:100640004E657700444343004620257520256320EE
:10065000256320256320256320256320256320252D
:1006600063202563004658202575202563202563D7
:100670002025632025632025632025630054202541
:1006800064202563202564004D43205265766973FC
:10069000696F6E2000312E342E32000D5365724E7C
:1006A000722E2025386C75004D5420256420256459
:1006B000005352202564004D6F64756C652023251E
:1006C000642028696E70757420312E2E3820262003
:1006D000392E2E313629203D200053452025640037
:1006E0003537363030002575000D5D002564005A21
:1006F0007A4100556E6B6E6F776E20636F6D6D6122
:100700006E64000D5D003132000032340000343878
:1007100000003936000031343400313932003338CA
:100720003400353736004142434445464748494A3C
:100730004B4C4D4E4F505152535455565758595A91
:10074000303132333435363738392E2C3A2D2B238D
:100750002F3D3C7C3E20004D4D204920203134204F
:10076000004D4D20492020323761004D4D20492059
:1007700020323762004D4D20012020313420004DC1
:100780004D20012020323761004D4D2001202032C4
:100790003762004443432020203134200044434347
:1007A000202020323820004443432020313238209A
:1007B000004C6F636D656E75000000000000000066
:1007C000004443432D70726F6772616D6D2E00009F
:1007D000004D6F64656C6261616E7369742E000018
:1007E00000496E7374656C6C696E67656E0000001D
:1007F00000536F667477617265205570646174652B
:10080000004C4344207665726C69636874696E6756
:10081000004D6173746572436F6E74726F6C00008B
:10082000004578697400000000000000000000002E
:10083000004B69657A656E20000000000000000032
:100840000044617461666F726D61740000000000A5
:10085000004E61616D20202020202000000000005B
:1008600000496E766F657220202020000000000095
:1008700000435620286279746529000000000000BA
:10088000004356202862697429000000000000001F
:100890000042617369736164726573000000000057
:1008A000004C616E67206164726573000000000097
:1008B00000526567697374657200000000000000F3
:1008C00000506167652D4D6F6465000000000000F9
:1008D00000486F6F666473706F6F720000000000F5
:1008E000007338382D696E7374656C6C696E67655A
:1008F0006E436F6E666967757261746965000000AA
:1009000000426F6F73746572000000000000000009
:1009100000496E74657266616365204261756400AA
:100920000057697373656C00000000000000000050
:10093000004C6F63666F726D617400000000000010
:10094000004D4D207369676E61616C7061757A65E9
:10095000007338382D6D6F64756C65000000000001
:10096000007338382D6D6F64756C65746573740031
:10097000004B6F7274736C2E20706F6C2E00000031
:10098000004B6F7274736C2E206765762E0000002A
:1009900000616C6C652057697373656C0000000022
:1009A0000057697373656C666F726D617400000047
:1009B000004D696E2E736368616B656C74696A645F
:1009C000004D61782E736368616B656C74696A644D
:1009D000004D656E75204C6F636F000000000000D5
:1009E0000050726F6772616D2E2044434300000017
:1009F0000045746174205265736561752E000000B6
:100A0000005265676C6167657300000000000000BC
:100A1000004D414A206C6F67696369656C00000096
:100A2000004C756D696E6F7369746500000000009D
:100A3000004D6173746572436F6E74726F6C000069
:100A4000004578697400000000000000000000000C
:100A50000053656C656374696F6E200000000000D0
:100A600000466F726D617420646F6E6E6565730011
:100A7000004E6F6D2020202020202000000000006C
:100A80000053616973696520202020000000000088
:100A90000043562028627974652900000000000098
:100AA00000435620286269742900000000000000FD
:100AB00000416472657373652064652062617365CB
:100AC0000041647265737365206C6F6E67756500B5
:100AD00000526567697374657200000000000000D1
:100AE00000506167652D4D6F6465000000000000D7
:100AF00000566F6965207072696E636970616C651C
:100B0000005265676C61676520733838000000002B
:100B100000436F6E66696775726174696F6E00007D
:100B200000426F6F737465720000000000000000E7
:100B300000496E7465726661636520426175640088
:100B400000436F6E662E2041696775696C6C612E7B
:100B500000466F726D6174206C6F636F000000005F
:100B6000005061757365207369676E616C204D4D2F
:100B7000004D6F64756C6573207338380000000099
:100B80000054657374206D6F64756C65207338381C
:100B900000506F6C2E6372742D6369726375697493
:100BA0000053656E732E206372742D6369726374D3
:100BB00000746F75732041696775696C6C657300AB
:100BC00000466F726D61742061696775696C6C2E87
:100BD00000547073206D696E2E696D70756C732E84
:100BE00000547073206D61782E696D70756C732E72
:100BF000004C6F6B204D656EFC0000000000000093
:100C0000004443432D50726F6772616D6D672E0013
:100C100000416E6C6167656E7A757374616E640015
:100C20000045696E7374656C6C756E67656E000067
:100C300000536F66747761726520557064617465E6
:100C4000004C43442042656C6575636874756E673B
:100C5000004D6173746572436F6E74726F6C000047
:100C600000457869740000000000000000000000EA
:100C70000041757377E4686C656E20000000000029
:100C800000446174656E666F726D617400000000EF
:100C9000004E616D65202020202020000000000013
:100CA0000045696E7472616720202000000000001A
:100CB0000043562028627974652900000000000076
:100CC00000435620286269742900000000000000DB
:100CD0000042617369732D4164726573736500002E
:100CE000006C616E67652041647265737365000016
:100CF00000526567697374657200000000000000AF
:100D000000506167652D4D6F6465000000000000B4
:100D1000004861757074676C6569730000000000BD
:100D2000007338382D45696E7374656C6C756E6729
:100D3000004B6F6E66696775726174696F6E000053
:100D400000426F6F737465720000000000000000C5
:100D500000496E7465726661636520426175640066
:100D6000005765696368656E0000000000000000C0
:100D7000004C6F6B666F726D6174000000000000C4
:100D8000004D4D2D5369676E616C20506175736520
:100D9000007338382D4D6F64756C650000000000DD
:100DA000007338382D4D6F64756C74657374000072
:100DB000004B75727A7363686C2E2D506F6C2E0029
:100DC000004B75727A7363686C2E2D456D70662EBC
:100DD00000616C6C65205765696368656E00000092
:100DE000005765696368656E666F726D61740000B7
:100DF000006D696E2E20536368616C747A65697446
:100E0000006D61782E20536368616C747A65697433
:100E1000004C6F636F6D6F74697665206D656E75DC
:100E2000004443432070726F6772616D6D696E6735
:100E3000004C61796F757420737461747573000070
:100E40000053657474696E67730000000000000051
:100E500000536F66747761726520557064617465C4
:100E6000004C4344206261636B6C696768740000E6
:100E7000004D6173746572436F6E74726F6C000025
:100E800000457869740000000000000000000000C8
:100E90000053656C656374200000000000000000D2
:100EA000004461746120666F726D6174000000001F
:100EB000004E616D652020202020200000000000F1
:100EC00000456E7472792020202020000000000070
:100ED0000043562028627974652900000000000054
:100EE00000435620286269742900000000000000B9
:100EF000005072696D617279206164647265737308
:100F000000457874656E642E206164647265737345
:100F1000005265676973746572000000000000008C
:100F200000506167652D4D6F646500000000000092
:100F3000004D61696E20747261636B0000000000F7
:100F4000007338382073657474696E67730000002D
:100F50000044656C6574650000000000000000003E
:100F600000426F6F737465720000000000000000A3
:100F700000496E7465726661636520426175640044
:100F800000506F696E7473000000000000000000E4
:100F9000004C6F632E20666F726D6174000000005C
:100FA000004D4D207369676E616C207061757365CB
:100FB00000733838206D6F64756C65730000000035
:100FC00000733838206D6F64756C652074657374B8
:100FD0000053686F727420632E20706F6C2E0000B7
:100FE0000053686F727420632E2073656E732E0039
:100FF00000616C6C20506F696E747300000000001B
:1010000000506F696E747320666F726D61740000BA
:10101000006D696E2E7377697463682E74696D65EF
:10102000006D61782E7377697463682E74696D65DD
:1010300000202D2D2D2D0025357500536F667477FA
:101040002E205600312E342E32005365724E722EF1
:101050002025386C75003A2000253575002533644D
:10106000002534643A20002D2D2D00253364002006
:101070004F4B202020200020202020202020004333
:10108000563A20202020204269743A203D20004317
:10109000563A253464204269743A25643D00202D77
:1010A0002D2D0025346400202D2D2D2D2D002536CD
:1010B0006400202E2E2E2E202020202020202020D4
:1010C000002533642C256473002534646D7300306F
:1010D00030204261756400446F776E6C6F616420EC
:1010E0002E2E2E002564206D730020253264004EC4
:1010F000723A2025326420200073686F72742028B1
:10110000312E356D73292000006C6F6E67202834F6
:101110002E3032356D732900004D6F746F726F6C15
:101120006100000000000000004443432020202014
:101130002000000000000000004D4D2000000000D5
:1011400000000000000000000044434300000000D5
:10115000000000000000000000706F736974697681
:101160006520284D4D290000006E65676174697621
:1011700065202844434329000053617665202020E0
:10118000202020202020202000526573746F72657B
:101190002020202020202020005361766520202060
:1011A000202020202020202000526573746F72655B
:1011B000202020202020202000206C61796F757471
:1011C000207374617475732000206C61796F75747D
:1011D0002073746174757320004B6F727220283114
:1011E0002E356D7329202000004C616E6720283455
:1011F0002E3032356D732900004D6F746F726F6C35
:101200006100000000000000004443432020202033
:101210002000000000000000004D4D2000000000F4
:1012200000000000000000000044434300000000F4
:10123000000000000000000000506F7369746965D1
:101240006620284D4D290000004E65676174696570
:101250006620284443432900004D6F64656C626139
:10126000616E7369742E2020004D6F64656C62613D
:10127000616E7369742E2020004865727374656C0A
:101280006C656E2020202020004F70736C61616EB1
:1012900020202020202020200020686572737465A3
:1012A0006C6C656E2020202000206F70736C616173
:1012B0006E2020202020202000436F75727420288B
:1012C000312E356D73292000004C6F6E6720283455
:1012D0002E3032356D732900004D6F746F726F6C54
:1012E0006100000000000000004443432020202053
:1012F0002000000000000000004D4D200000000014
:101300000000000000000000004443430000000013
:10131000000000000000000000706F7369746976BF
:101320006520284D4D290000006E6567617469765F
:10133000652028444343290000456E726567697340
:101340007472656D656E7420005265737461757298
:101350006174696F6E20202000456E726567697345
:101360007472656D656E7420005265737461757278
:101370006174696F6E2020200020457461742052D2
:1013800065736561752E20200020457461742052BC
:1013900065736561752E2020004B75727A202831A7
:1013A0002E356D7329202000004C616E6720283493
:1013B0002E3032356D732900004D6F746F726F6C73
:1013C0006100000000000000004443432020202072
:1013D0002000000000000000004D4D200000000033
:1013E0000000000000000000004443430000000033
:1013F000000000000000000000706F7369746976DF
:1014000020284D4D29000000006E656761746976E3
:10141000202844434329000000416E6C6167656EDB
:101420007A757374616E642000416E6C6167656EDD
:101430007A757374616E64200057696564657268BB
:1014400065727374656C6C6E005370656963686572
:10145000726E20202020202000207769656465724C
:1014600068657273742E202000207370656963684C
:1014700065726E202020202000696E636F6D7061A0
:10148000742E20466F726D617400496E636F6D70CB
:101490002E20466F726D6174202000466F726D6160
:1014A0007420696E636F6D7061742E00696E6B6F6E
:1014B0006D7061742E20466F726D6174002E2E2E39
:1014C0002077616974696E67202E2E2E2000233DDF
:1014D00064656C6574650000000000000000002871
:1014E0006E6F20656E7472792900000000000000A4
:1014F0002E2E2E2064656C6574696E67202E2E2E4C
:1015000000206661756C740000000000000000009F
:10151000000020444343206F6E6C792100000000DE
:101520000000002A3D43616E63656C2020200000AE
:10153000000000002070726F6772616D696E670055
:1015400000000000002D73686F727420636972637D
:101550007569742D20002A72656164200000000006
:10156000000000000000002A777269746500000026
:1015700000000000000000002E2E2E2077726974FB
:10158000696E67202E2E2E20002E2E2E2072656171
:1015900064696E67202E2E2E200021212120666195
:1015A000756C742021212120202000204F4B202009
:1015B0002020202020202020202020002E2E2E2021
:1015C000736176696E67202E2E2E2020002E2E202D
:1015D000726573746F72696E67202E2E2000233D32
:1015E00044656C2E202A3D43616E63656C200023A8
:1015F0003D596573202A3D43616E63656C20200070
:1016000020636F6E66696775726174696F6E202002
:10161000004F4646000000000000000000000000EF
:1016200000002A2A2A206E6F20547261696E202AD7
:101630002A2A002A2073686F7274206369726375A6
:10164000697420002A2A2A2074696D65206F7574D8
:10165000202A2A2A00506F696E7420202534642FB6
:10166000253464000000436F6E66696775726174AB
:10167000696F6E2020200020636F6E666967757247
:101680006174696F6E2020002E2E2E2077616368B2
:1016900074656E202E2E2E2000233D7769737365AE
:1016A0006E000000000000000000286765656E20E5
:1016B000696E766F65722900000000202E2E2E20A4
:1016C00077697373656E202E2E2E000020666F756D
:1016D0007400000000000000000000000020416CC9
:1016E0006C65656E204443432100000000002A3DE4
:1016F0002041666272656B656E000000000000208C
:1017000050726F6772616D6D6572656E00000000EA
:101710002D2D4B6F7274736C756974696E672D2D06
:10172000002A4C657A656E00000000000000000091
:1017300000002A5363687269000000000000000086
:101740000000002E2E2073636872696A76656E2031
:101750002E2E00002E2E2E206C657A656E202E2EE9
:101760002E202000002021212120466F7574202189
:10177000212120200000204F4B202020202020204D
:10178000202020202000002E2E2E204F70736C6110
:10179000616E202E2E2E00004865727374656C6C8D
:1017A000656E20202020200000233D77697373653B
:1017B0006E202A3D616662720000233D4A61202A44
:1017C0003D41666272656B656E20002077697373B8
:1017D000656E202020202020202020005549540024
:1017E000000000000000000000000000002A2A2A7B
:1017F000206765656E204C6F63202A2A2A002A2AFA
:101800006B6F7274736C756974696E672A2A002A2B
:101810002054696A646F766572736368722E2A0059
:1018200057697373656C732534642F253464000025
:1018300000436F6E66696720202020202020202032
:10184000200020436F6E6669672020202020202022
:1018500020200050617469656E74657A0000000094
:1018600000000000233D7375707072696D65720031
:1018700000000000007669646500000000000000C0
:101880000000000000005375707072657373696F1B
:101890006E00000000000020457272657572000045
:1018A00000000000000000002044434320756E69E2
:1018B0007175656D656E7400002A3D4162616E64EC
:1018C0006F6E20200000000000002050726F6772D1
:1018D000616D6D6174696F6E0000002D436F7572EC
:1018E000742D636972637569742D20002A4C6563D9
:1018F000742E00000000000000000000002A456374
:1019000072697400000000000000000000002E2E2C
:101910002E204563726974757265202E2E2E002E5E
:101920002E2E204C656374757265202E2E2E20009D
:1019300021212120457272657572202121212020EC
:1019400000204F4B2020202020202020202020205D
:10195000200020456E72656769737472656D656EEF
:1019600074200020526573746175726174696F6EC2
:1019700020202000233D5375707072202A3D416263
:10198000616E642E00233D4F7569202A3D416261DE
:101990006E646F6E2000205375707072696D657291
:1019A00020202020202000496E6163746966202079
:1019B00020202020202020002A20506173206465F0
:1019C000206C6F636F202A20002A20436F75727489
:1019D0002D6369726375697420002A2054656D70E7
:1019E0007320646570617373652000416967756970
:1019F0006C2E2534642F253464000000456E72651A
:101A00006769737472656D656E742020005265732A
:101A1000746175726174696F6E20202020002E2E13
:101A20002E2077617274656E202E2E2E20200023CA
:101A30003D4CF6736368656E000000000000000016
:101A4000286B65696E2045696E74726167290000B4
:101A500000202E2E2E206CF673636865202E2E2E0D
:101A60002000204665686C657200000000000000E0
:101A7000000000206E75722066FC722044434321F2
:101A8000000000002A203D204162627275636800F8
:101A900000000000002050726F6772616D6D696513
:101AA00072756E6700002D2D204B75727A73636816
:101AB0006C75DF202D2D002A6C6573656E000000AB
:101AC00000000000000000002A736368722E00000E
:101AD0000000000000000000002E2E2073636872DA
:101AE000656962656E202E2E00002E2E2E206C65FC
:101AF00073656E202E2E2E202000002121212046ED
:101B000065686C657220212121200000204F4B2048
:101B1000202020202020202020202000002E2E20E9
:101B200073706569636865726E202E2E0000776998
:101B3000656465726865727374656C6C656E0023AC
:101B40003D4CF6736368656E202A3D416262720007
:101B5000233D4A61202A3D4162627275636800003C
:101B600000206CF6736368656E2020202020202002
:101B7000200041555300000000000000000000005C
:101B80000000002A2A206B65696E65204C6F6B206F
:101B90002A2A20002A2A204B75727A7363686C7592
:101BA000DF202A2A002A205A656974FC6265727354
:101BB0006368722E2A00576569636865202534645E
:101BC0002F2534640000004B6F6E66696775726183
:101BD00074696F6E20202000204B6F6E66696775F8
:101BE000726174696F6E2020005B6E6F206D65738B
:101BF000736167655D005B756E6B6E6F776E2065F8
:101C000072726F725D005B756E6B6E6F776E2073B4
:101C100074617475735D000011241FBECFEFD0E1B5
:101C2000DEBFCDBF12E0A0E0B1E0E6E6FAED00E0F5
:101C30000BBF02C007900D92AA3DB107D9F71DE076
:101C4000AAEDB2E001C01D92A532B107E1F70C94F4
:101C5000950E0C94000081E08093DB020895982F8C
:101C60008091DA02891731F0863021F0853029F42D
:101C7000963019F080E090E008959093DA02892F71
:101C80008250823058F40E949D1E1092C8068091A6
:101C9000DA02823051F40E943E2907C0943019F4D0
:101CA0000E94C01E02C00E94AC1E8091DA028630E3
:101CB00011F40E9486548091DA02813019F482E096
:101CC0000E94CA664AED52E063E08FEF0E943B55E6
:101CD0000E942B0E81E090E0089508958091DA0231
:101CE0009927089580E00E94721A2FEF8F3F920784
:101CF00019F0682F80E009C081E00E94721A2FEF6E
:101D00008F3F920721F0682F81E00E945D3E0E9484
:101D100051550E9473640E94142D8091DB02882328
:101D200011F40E945219A8950895CFEFD0E1DEBFBB
:101D3000CDBF0E9447520E94730F0E9478250E94D7
:101D4000F3620E94EE1E0E94875221E04EE468E09A
:101D50000E94A00F21E04EE468E087E00E94B911E4
:101D60000E94571378940E9425150E947F52FC010F
:101D700084810E94BB1962E171E082E00E94F01947
:101D80000E94CA52813059F060E081E00E946818D8
:101D900062E271E082E00E94F019A895FECF6EE148
:101DA00071E082E00E94F01960E081E00E94681812
:101DB00066E582E00E94C01962E371E082E00E9461
:101DC000F0190E947F528C0181E00E943D17882308
:101DD00019F081E00E94825282E00E943D17882320
:101DE00019F080E00E94825283E00E943D17882310
:101DF00019F082E00E94825284E00E943D178823FD
:101E000019F083E00E94825280E00E942F0E80E051
:101E10000E943D17882319F084E10E9413510E940B
:101E2000ED5F40E050E060E28FEF0E943B5580E0C4
:101E30000E94413E81E00E94413E8091CA069091FD
:101E4000CB06A091CC06B091CD06805D9740A04016
:101E5000B04078F40E94720E8091CA069091CB0631
:101E6000A091CC06B091CD06805D9740A040B040D7
:101E700088F3F80181859285892BC9F00E94862913
:101E8000EC0144969E01215F3F4FAC01B901F8017E
:101E9000818592850E94B95EBC01892B29F0F801E9
:101EA000818592858A8B9B8B6115710519F4F801E8
:101EB000628173818FEF0E94F65381E011C00E940E
:101EC0002F2D0E94FF17FFEF8F3F9F07C1F70E9442
:101ED000720E8091DB028823A1F31092DB0280E076
:101EE0000E941A2BEECF8FE78ABB1BBA80E187BB1B
:101EF00018BA80EF84BB8FEF85BB8BEB81BB8CEC7A
:101F000082BB86E082B987EF83B98093610081EF5D
:101F1000809362008FE18093640089E18093650083
:101F20000E943C5C10926A001ABE8AB78A608ABF1F
:101F30000E949616A89588E181BD8CE081BD089528
:101F4000E82F10929C0680919C0680939B068091BE
:101F50009B068093BE068091BE068093BD0691E0ED
:101F60009093C7068C9A119A82B18E7E82B9199A83
:101F700083B18E7E83B982E08BB99498E83008F003
:101F8000E92FFF27EE0FFF1FE85CFE4FA591B491EC
:101F9000653010F465E003C0693008F068E04F7DFB
:101FA0006550660F453411F4606203C04F3409F484
:101FB0006063223008F068608B2F992787FD9A951F
:101FC0008F7080939000A9B96093950088EB8AB9CF
:101FD00080E090E008959091BD068091BE0698172C
:101FE00011F00C9B559A089508951F920F920FB609
:101FF0000F9211248F939F93EF93FF939091BD06BF
:102000008091BE06981761F088B7806188BF0C9BED
:1020100009C089B7806189BF8091C70680FF02C06F
:10202000559813C08091BE06E82FFF27E556F94F5B
:1020300084A18CB98091BE068F5F8093BE0680918B
:10204000BE06883010F01092BE06FF91EF919F916E
:102050008F910F900FBE0F901F9018951F920F92A7
:102060000FB60F9211248F9389B78F7E89BF559A2F
:102070008F910F900FBE0F901F9018951F920F9287
:102080000FB60F9211242F933F934F935F936F934B
:102090007F938F939F93AF93BF93EF93FF93809121
:1020A0009B06282F332780919C0699270197281794
:1020B000390741F080919B068F3179F480919C061D
:1020C000882359F480919C068F5F80939C068091B1
:1020D0009C06803210F010929C069BB180919B066A
:1020E000E82FFF27E556F94F8CB18283228194FDBA
:1020F0000CC080919B068F5F80939B0680919B060E
:102100008032A8F010929B0612C0222381F4209303
:102110009C0680919C0680939B069498822F0E9437
:10212000413E21E04EE468E0822F0E94A00F8091A2
:102130009B06282F332780919C06281B310937FFE7
:1021400002C0205E3F4F213131050CF0949AFF917F
:10215000EF91BF91AF919F918F917F916F915F911F
:102160004F913F912F910F900FBE0F901F90189598
:1021700050E060E070E027E0813D920708F051E018
:102180002FE0813A920708F052E023E28932920769
:1021900008F053E026E3813B920708F054E026E480
:1021A0008135920708F055E028E8893B920708F04E
:1021B00056E0895D964D08F057E078948BB19927E9
:1021C00026E0969587952A95E1F79C01217030705D
:1021D00080FFB9016F5F7F4FA89587E26031780774
:1021E00068F321E04EE468E0852F0E94A00F089577
:1021F00089B1282F3327809190009927982F88271D
:10220000282B392B60E040E050E0FA01E85CFE4FFB
:10221000859194918217930729F06F5F4E5F5F4F0E
:10222000683098F3862F99278330910509F184301F
:1022300091054CF481309105A9F082309105ACF400
:10224000892B69F024C085309105C1F08530910556
:1022500094F086309105A9F00797B1F018C080EB93
:1022600094E0089580E699E0089580EC92E1089565
:1022700080E895E2089580E498E3089580E09BE487
:10228000089580E096E9089580E091EE089580E059
:1022900090E008950895482F07C08091BE068823D6
:1022A00091F4559A7894A8958091BD06282F3327EC
:1022B0008091BE06992701972817390791F38091DD
:1022C000BD06873051F38091BD06E82FFF27E55604
:1022D000F94F44A38091BD068F5F8093BD06809126
:1022E000BD06883010F01092BD06559A80E090E04F
:1022F000089580919B06282F332780919C06281BE8
:10230000310937FF02C0205E3F4F203131050CF408
:10231000949890919B0680919C06981719F48FEFE2
:102320009FEF089580919C06E82FFF27E556F94F0F
:102330008281282F332780919C068F5F80939C0693
:1023400080919C06803210F010929C06C90108957D
:102350000895882331F08091C70681608093C70675
:1023600008958091C7068E7F8093C706559A089579
:102370000895E82F10926F0680916F0680936E0685
:1023800080916E06809391068091910680939006CD
:1023900091E090939A0681B3886281BB8A981598E0
:1023A000939A92981D9882E080939B009598E830CC
:1023B00008F0E92FFF27EE0FFF1FE85CFE4FA59105
:1023C000B491653010F465E003C0693008F068E04E
:1023D0004F7D6550660F8B2F992787FD9A958F70DB
:1023E00080939800A0939900453411F4606203C073
:1023F0004F3409F46063223008F0686060939D00F8
:1024000088EB80939A0080E090E008959091900688
:1024100080919106981739F00D9905C080919A0026
:10242000806280939A00089508951F920F920FB6CC
:102430000F9211248F939F93EF93FF9390919006A7
:1024400080919106981761F088B7806288BF0D9BD4
:102450000DC089B7806289BF80919A0680FF06C04F
:1024600080919A008F7D80939A0014C0809191068C
:10247000E82FFF27E259F94F84A180939C008091B7
:1024800091068F5F8093910680919106883010F0BD
:1024900010929106FF91EF919F918F910F900FBE37
:1024A0000F901F9018951F920F920FB60F92112444
:1024B0008F9389B78F7D89BF80919A0080628093C6
:1024C0009A008F910F900FBE0F901F9018951F923A
:1024D0000F920FB60F9211242F933F934F935F9358
:1024E0006F937F938F939F93AF93BF93EF93FF93DC
:1024F00080916E06282F332780916F0699270197C8
:102500002817390741F080916E068F3179F4809158
:102510006F06882359F480916F068F5F80936F0652
:1025200080916F06803210F010926F0690919B00A0
:1025300080916E06E82FFF27E259F94F80919C00A9
:102540008283828194FD0CC080916E068F5F8093A0
:102550006E0680916E06803278F010926E060CC086
:10256000882351F480936F0680916F0680936E06E6
:10257000959881E00E94413E80916E06282F332776
:1025800080916F06281B310937FF02C0205E3F4F44
:10259000213131050CF0959AFF91EF91BF91AF91E8
:1025A0009F918F917F916F915F914F913F912F916B
:1025B0000F900FBE0F901F901895482F0BC0809161
:1025C00091068823B1F480919A00806280939A00EA
:1025D0007894A89580919006282F332780919106B2
:1025E000992701972817390771F380919006873052
:1025F00031F380919006E82FFF27E259F94F44A369
:10260000809190068F5F809390068091900688302D
:1026100010F01092900680919A00806280939A0048
:1026200080E090E0089580916E06282F33278091F6
:102630006F06281B310937FF02C0205E3F4F203153
:1026400031050CF4959890916E0680916F0698175D
:1026500019F48FEF9FEF089580916F06E82FFF2701
:10266000E259F94F8281282F332780916F068F5FBF
:1026700080936F0680916F06803210F010926F0683
:10268000C90108950895882331F080919A068160E8
:1026900080939A06089580919A068E7F80939A0679
:1026A00080919A00806280939A000895089587B37C
:1026B000876087BBBB9888B3896088BB1DB88EB123
:1026C0008FB187E78DB908951F920F920FB60F92C1
:1026D00011242F938F939F93EF93FF932FB18091AA
:1026E000DC02E82FFF27E452FD4F22838F5F8093A7
:1026F000DC02883110F01092DC029091F702E92F91
:10270000FF27E452FD4F248D27FDC09A8091F602E9
:10271000981759F0C098892F8F5F8093F7028831FE
:1027200010F01092F7022FB902C0C09A6F98FF9173
:10273000EF919F918F912F910F900FBE0F901F904F
:1027400018958091F702282F33278091F602281BD5
:102750003109C90147968831910514F0C9010197E3
:1027600008950895282F6F9919C0C0988FB16F9A56
:102770008091F6029091F702891711F42FB91CC0CD
:10278000E92FFF27E452FD4F848D8FB9892F8F5F8A
:102790008093F702883110F01092F7028091F602D0
:1027A000E82FFF27E452FD4F248F8F5F8093F602BE
:1027B000883110F01092F60280E090E00895809148
:1027C000DC022091DD02821719F48FEF9FEF08954C
:1027D000E22FFF27E452FD4F8281482F5527822F99
:1027E0008F5F8093DD02883110F01092DD02CA0104
:1027F000907008950895882311F0DD9A0895DD986A
:10280000089508950F931F93CF93282FDE9B63C0E5
:10281000882309F060C0809112039091130353E064
:10282000969587955A95E1F7182FC0911203C770B6
:10283000022FCF9901E09BB3892F8F7A8BBB94FF36
:1028400002C081E001C0822F0E94FB13A0911203FD
:10285000B0911303412F55276C2F7727C091610A40
:10286000002399F0FA01ED51F54F20E830E002C065
:10287000359527956A95E2F78081822B8083FA014E
:10288000ED55F54F8081822B0EC0FA01ED51F54FC9
:1028900080E890E002C0959587956A95E2F7982FB9
:1028A00090958081892380839D012F5F3F4F3093D6
:1028B0001303209312038C2F992744E0880F991F4C
:1028C0004A95E1F72817390758F0DC9A109213035C
:1028D0001092120305C0222311F0DE9A01C0DE9887
:1028E000CF911F910F91089500000000000000009B
:1028F0000895882341F0809165008460809365008D
:102900000E9474140895809165008B7F8093650008
:10291000089508959B01AC018091CA069091CB0661
:10292000A091CC06B091CD0682179307A407B507F6
:10293000A0F08091CA069091CB06A091CC06B091F0
:10294000CD06821B930BA40BB50B80509041A04089
:10295000B040A0F080E090E008958091CA06909188
:10296000CB06A091CC06B091CD06281B390B4A0BA3
:102970005B0B2050304F4F4F5F4F18F081E090E0DD
:10298000089580E090E008950895EF92FF920F93EC
:102990001F93AA27BB27E090CA06F090CB060091B0
:1029A000CC061091CD06E80EF91E0A1F1B1F01C0B0
:1029B000A895C801B7010E948A148823C9F31F9102
:1029C0000F91FF90EF9008950F931F93CF93C82F0F
:1029D000162F042F809165008D7F8093650080E025
:1029E0000E9479148AB38F608ABB8BB3807F9C2F3F
:1029F00092959F70892B8BBB112321F080916500EC
:102A0000816003C0809165008E7F8093650081E0C6
:102A10000E94791480E00E947914002329F088E054
:102A200090E00E94C5140DC08BB3807FCF708C2BBB
:102A30008BBB0E94741481E00E947914802F0E9445
:102A40007914CF911F910F91089588E290E00E9430
:102A5000C51441E060E080E30E94E41441E060E0DE
:102A600080E30E94E41441E060E080E30E94E4140B
:102A700041E060E080E20E94E41488E20E945E1877
:102A800088E00E945E1881E00E945E1886E00E9445
:102A90005E188CE00E945E186CE372E080E00E9499
:102AA000971964E172E081E00E9497196CE172E08D
:102AB00082E00E94971964E072E083E00E94971917
:102AC00064EF71E084E00E9497196CEE71E085E09C
:102AD0000E94971964EE71E086E00E9497196CEDF0
:102AE00071E087E00E94971908951F920F920FB628
:102AF0000F9211241F932F933F934F935F936F93E4
:102B00007F938F939F93AF93BF93EF93FF938091A6
:102B100010038F5F80931003282F237009F0F4C0F7
:102B200086958695877099278330910509F47CC036
:102B3000843091054CF48130910551F1823091053A
:102B4000DCF5892B89F0E0C08530910509F4A2C03D
:102B5000853091050CF49CC08630910509F4CEC0F7
:102B6000079709F4CFC0D0C08091CA069091CB06D8
:102B7000A091CC06B091CD060196A11DB11D809308
:102B8000CA069093CB06A093CC06B093CD0680C026
:102B90008091CA069091CB06A091CC06B091CD064B
:102BA00081709070A070B070892B19F00E9450173E
:102BB000ABC00E941117A8C081E00E9402140E94BD
:102BC0006E0E833009F0A0C00E94F91E2091C80645
:102BD0003091C9068823E9F02E5F3F4F3093C90634
:102BE0002093C8060E947F52FC019681992309F424
:102BF0008BC08AE0989F900111248091C806909123
:102C0000C9068217930708F47FC081E00E942F0E47
:102C10007BC02115310509F477C021503040309335
:102C2000C9062093C80670C080911103882309F457
:102C30006BC08AB3807F8ABB822F0E9479148091F7
:102C40006500826080936500809165008E7F80932F
:102C500065000000000081E00E94791419B380E053
:102C60000E9479141295107F0E94741481E00E94D2
:102C7000791489B38F70182B80E00E947914812F0A
:102C8000992787FD90958827990F881F992733C02A
:102C9000822F35C0609111036623B1F59091CE0665
:102CA0008091CF06981789F01091CF06E12FFF276A
:102CB000E253F94F82811F5F103108F0162F8038E0
:102CC00091F48091CE06811719F480E090E013C052
:102CD000E12FFF27E253F94F82811F5F103108F087
:102CE000162F462F02C0462F61E00E94E414109375
:102CF000CF0681E090E08093110306C081E00E943E
:102D0000021402C00E94E517FF91EF91BF91AF91AD
:102D10009F918F917F916F915F914F913F912F91F3
:102D20001F910F900FBE0F901F90189510927D006D
:102D300017BE11BE89E683BF87B7816087BF82EF68
:102D40008FBD3AE13EBD4FEC50E057BD46BD85EB2F
:102D500090E09BBD8ABD99BD88BD22EC20938B007D
:102D600030938A00509381004093800090938700B5
:102D7000809386000E947F52FC0180858093610AC7
:102D80000895EF92FF920F931F93AA27BB27E0901D
:102D9000CA06F090CB060091CC061091CD06E80E45
:102DA000F91E0A1F1B1F02C00E94720EC801B70144
:102DB0000E948A148823C1F31F910F91FF90EF9016
:102DC0000895282F220F61112160822F8370815076
:102DD000823028F424FF02C02E6001C0217F822FA0
:102DE0009927089590911603E92FFF27EA5EFC4F7B
:102DF0008283892F8F5F80931603883010F01092A2
:102E000016039091170380911603981741F4892FA8
:102E10008F5F80931703883010F010921703089586
:102E200008950F931F9311B1812F8074682F8091A3
:102E300014030E94E116082F809314031078612F69
:102E4000809115030E94E11680931503007C807C1D
:102E5000003829F4882339F0803C61F408C000343C
:102E600049F4803C11F484E103C0882319F485E11E
:102E70000E94F2161F910F910895843118F080E09E
:102E800090E0089520E030E0E82FFF27E05EFC4F5F
:102E90008081882311F021E030E0C9010895089570
:102EA000FF920F931F93CF9380913903E82FFF2751
:102EB000EC5CFC4F008113B31083FF248091390335
:102EC000E82FFF27EE0FFF1FEE0FFF1FEF0DF11D85
:102ED000E85BFE4FC49110FD42C000FF14C0C23138
:102EE00029F481E10E943D17882331F48C2F0E9440
:102EF000F216C43108F054C0EC2FFF27E05EFC4FFF
:102F000081E080834DC0C43108F04AC0EC2FFF2718
:102F1000DF01A05EBC4F9C919F5F9C93992311F4AD
:102F20009F5F9C93E131F105DCF1E331F1056CF039
:102F30007397B1F580913303853690F18CE10E944F
:102F4000F21681E0809333032BC0809131038937DF
:102F500038F180913203893718F185E01FC0C43100
:102F600028F4EC2FFF27E05EFC4F108200FD18C014
:102F70008C2F80680E94F2160E946E0E853081F4BC
:102F8000C13121F482E10E943D1705C0C23141F4F4
:102F900081E10E943D17882319F486E00E942F0EDC
:102FA00016950695F39483E08F1508F087CF8091EE
:102FB00039038F5F80933903853010F01092390305
:102FC000CF911F910F91FF90089590913903943004
:102FD00029F485B3806F85BB97980895979A85B338
:102FE0008F7020E130E002C0220F331F9A95E2F784
:102FF000922F9095907F892B85BB0895089580919D
:10300000160320911703821719F48FEF9FEF08958D
:10301000E22FFF27EA5EFC4F8281482F5527822F3F
:103020008F5F80931703883010F010921703CA0146
:1030300008950895CF93C82F1CC08091CF06882390
:1030400039F580E00E94721A2FEF8F3F920719F036
:10305000682F80E009C081E00E94721A2FEF8F3F35
:10306000920721F0682F81E00E945D3E0E94515539
:10307000A8958091CE06282F33278091CF069927D7
:10308000019728173907E9F28091CE068F30A9F20F
:10309000F8948091CE06E82FFF27E253F94FC283C0
:1030A0008091CE068F5F8093CE068091CE068031D0
:1030B00010F01092CE067894CF9108951F93182F98
:1030C00080E80E941A18812F0E941A181F910895F3
:1030D0008295880F880F807C860F80680E945E181A
:1030E00008950E9468188EE00E945E1808958CE092
:1030F0000E945E180895FF920F931F93CF93F82EAE
:103100006091F1068091F0060E946818C0E000EE20
:1031100016E08091F206C81778F4FF2021F0F8013C
:1031200061918F0101C060E282E00E94C019CF5F0F
:103130008091F206C81788F3CF911F910F91FF90ED
:1031400008959093FB068093FA06892B89F170937A
:10315000F9066093F806CB01AA27BB272091CA067F
:103160003091CB064091CC065091CD06280F391FE7
:103170004A1F5B1F2093F4063093F5064093F60632
:103180005093F7068091F3068E7F8093F306211506
:1031900031054105510561F42F5F3F4F4F4F5F4FA0
:1031A0002093F4063093F5064093F6065093F70605
:1031B00008950895AF92BF92CF92DF92EF92FF925F
:1031C0000F931F93CF93DF93D82EC62EEA0180EE84
:1031D000E82E86E0F82E1092FB061092FA0681E0A7
:1031E0008D1568F1EFE0E61750F14115510539F101
:1031F000FA0101900020E9F731970E2F041B0131ED
:1032000008F000E16C2D8D2D0E94681857010023F5
:1032100061F0102F8881F50181935F018991682FFA
:1032200082E00E94C0191150A9F7F701D08AC18A23
:10323000028B64EF71E08BE798E10E94A118DF91A7
:10324000CF911F910F91FF90EF90DF90CF90BF90A3
:10325000AF900895CF93DF93CDB7DEB7A0970FB6A9
:10326000F894DEBF0FBECDBF282FDE01119690E08F
:10327000FA014F5F5F4F8491882321F08D939F5F08
:103280009F31B0F31C92AE014F5F5F4F822F0E94BF
:10329000DA18A0960FB6F894DEBF0FBECDBFDF914F
:1032A000CF9108958091FA069091FB06892BA9F1A0
:1032B0006091F4067091F5068091F6069091F706FC
:1032C0000E948A14882349F18091F306E091FA065E
:1032D000F091FB06817009958091F30691E08927B2
:1032E0008093F3068091F8069091F9069C0144279B
:1032F00055278091CA069091CB06A091CC06B0913B
:10330000CD06820F931FA41FB51F8093F4069093E0
:10331000F506A093F606B093F70608950895109267
:10332000FB061092FA0681E00E945E1808950F9342
:103330001F93CF93DF93EB018830C0F4992723E0EC
:10334000880F991F2A95E1F780640E945E1807E0B4
:1033500010E0FE01219684910E941A18015010403D
:1033600017FFF7CF60E0862F0E946818DF91CF919A
:103370001F910F910895813308F080E381BF089574
:1033800099278130910539F1823091051CF4892B00
:10339000F1F00895029711F567FF15C0643E31F012
:1033A000663F41F06C3F51F0643C11F461EE0BC09C
:1033B000663D11F46FEE07C06C3D11F465EF03C07C
:1033C0006F3D09F462EE862F0E941A180895862F29
:1033D0000E944B110895862F0E94DD1208950895D2
:1033E0001F93CF93DF93182FEB01FB0164916623AA
:1033F00049F0812F0E94C0192196FE018491682F07
:103400008823B9F7DF91CF911F9108951F93CF9330
:10341000DF93182FEB018881882341F08991682F71
:10342000812F0E94C01988818823C1F7DF91CF9135
:103430001F9108951F93CF93DF93CDB7DEB7C0558B
:10344000D0400FB6F894DEBF0FBECDBF67961FAD5C
:10345000679769968EAD9FAD6997AE01475A5F4FEA
:10346000BC01CE0101960E94DD6BBE016F5F7F4FF4
:10347000812F0E94061AC05BDF4F0FB6F894DEBFA3
:103480000FBECDBFDF91CF911F9108951F93CF93B2
:10349000DF93CDB7DEB7C055D0400FB6F894DEBF8E
:1034A0000FBECDBF67961FAD679769968EAD9FAD76
:1034B0006997AE01475A5F4FBC01CE0101960E9449
:1034C000066CBE016F5F7F4F812F0E94061AC05BA2
:1034D000DF4F0FB6F894DEBF0FBECDBFDF91CF91A7
:1034E0001F91089599278130910571F082309105DF
:1034F0001CF4892B31F00BC0029749F40E94FF178E
:1035000008950E94791108950E94131308958FEF72
:103510009FEF08950895FC018F3F910519F010F079
:10352000E0E0F0E0E45AFD4F84919927089590E09F
:103530008F3010F08EE001C081118F5F442311F0B5
:1035400028E001C0242F77276230710581F06330B5
:10355000710524F46130710541F00EC063307105CE
:1035600041F06430710539F007C0236005C0246064
:1035700003C0266001C02760281729F4442311F0F6
:103580002AE001C025E043E050E0990F990F80FD4B
:10359000926020FD9160869526954150504057FFDE
:1035A000F4CF892F992708959C01FB018F3791054E
:1035B00028F48F77808388E090E00895832F9927FF
:1035C000806C8183208380E190E008950895FC0160
:1035D0004081242F332781819927019728173907A4
:1035E00029F04F3031F48181882319F481E090E093
:1035F000089580E090E0089508951F938CEF96E081
:103600000E94E71A182F8EE697E00E94E71A182BFF
:10361000812F99271F910895AF92BF92CF92DF9289
:10362000EF920F931F93CF93DF93EC016B015A013D
:10363000122F80916C03882369F40B3059F00C3001
:1036400049F0CB010E940427992783709070892B41
:1036500009F48CC080916C038823B1F58981282FEF
:103660003327888199272817390771F1AC01F901AF
:10367000A3E0EE0FFF1FAA95E1F7E21BF30BEC0F9F
:10368000FD1F828193818C159D05A1F48481958114
:103690008A159B0579F48681801761F4013019F44D
:1036A0008085882339F080858E1509F45FC0E08617
:1036B00017835CC02F5F3F4F2031310514F020E0AD
:1036C00030E02417350799F6CE010E94E71A282F1B
:1036D000882319F080E090E04BC088819927FC0195
:1036E00073E0EE0FFF1F7A95E1F7E81BF90BEC0F83
:1036F000FD1FC282D38288819927FC0163E0EE0F0F
:10370000FF1F6A95E1F7E81BF90BEC0FFD1FA48280
:10371000B58288819927FC0153E0EE0FFF1F5A956F
:10372000E1F7E81BF90BEC0FFD1F17838881992740
:10373000FC0143E0EE0FFF1F4A95E1F7E81BF90B90
:10374000EC0FFD1F068388819927FC0133E0EE0F03
:10375000FF1F3A95E1F7E81BF90BEC0FFD1FE08620
:1037600088818F5F8883803108F0288381E090E032
:10377000DF91CF911F910F91EF90DF90CF90BF908D
:10378000AF9008959F92AF92BF92CF92DF92EF9247
:10379000FF920F931F93CF93DF93EC015B016A01BC
:1037A000922EF02E1E2D892B31F48EE697E00E948A
:1037B000C21BCCEFD6E080916C03882321F087E018
:1037C000CE36D807C1F00E946E0E8250833098F436
:1037D000F894E12E0F2D292DA601B501CE010E94EE
:1037E0000C1B7894882329F485E090E00E94C5148E
:1037F000EACF10926F03DF91CF911F910F91FF904D
:10380000EF90DF90CF90BF90AF909F900895EF9290
:103810000F93CF93DF93EC01E62E0E94C025FC01AD
:10382000892B89F08085992783709070039711F414
:1038300023E001C026E001E040E050E0BE018CEF53
:1038400096E00E94C21B81E090E0DF91CF910F9142
:10385000EF900895EF920F93CF93DF93EC010E94C6
:10386000C025FC01892BA9F0808599278370907071
:10387000039731F486818F67E82E01E024E003C0CE
:10388000EE2402E02BE040E050E0BE01CA010E94BD
:10389000C21B81E090E0DF91CF910F91EF900895EE
:1038A000EF920F93CF93DF93EC010E94C025FC01B0
:1038B000892B81F0808599278370907001970297FA
:1038C00048F4EE2402E02BE040E050E0BE01CA01E3
:1038D0000E94C21B81E090E0DF91CF910F91EF90A9
:1038E0000895EF920F93CF93DF93EC010E94C025D0
:1038F000FC01892B79F0808599278370907001975E
:1039000049F4EE240AE024E040E050E0BE01CA01A0
:103910000E94C21B81E090E0DF91CF910F91EF9068
:103920000895AF92BF92CF92DF92EF920F93CF9311
:10393000DF935C016B010E94C025EC01892B09F427
:1039400051C088859927837090708230910571F5F8
:10395000D7FE05C06E81888199810E94071CC0FE38
:1039600009C0EE8006E024E040E050E0B501CA0165
:103970000E94C21BC1FE09C0EE8007E024E040E0C7
:1039800050E0B501CA010E94C21BC2FE09C0EE8010
:1039900008E024E040E050E0B501CA010E94C21BEB
:1039A000C3FE20C0EE8009E024E016C00397D1F4E6
:1039B000C6018F709078892B49F0EE2403E024E053
:1039C00040E050E0B501CA010E94C21B8C2D807FEF
:1039D00049F0EE2404E0202F40E050E0B501CA0198
:1039E0000E94C21B81E090E0DF91CF910F91EF9098
:1039F000DF90CF90BF90AF900895EF920F931F93F9
:103A0000CF93DF93EC01162F0E940427837081501F
:103A1000823050F4EE2402E0212F40E050E0BE015D
:103A20008CEF96E00E94C21B81E090E0DF91CF9185
:103A30001F910F91EF900895EF920F93E62E66235A
:103A400019F0EE240CE001C00BE023E040E050E070
:103A5000BC01CA010E94C21B81E090E00F91EF906F
:103A60000895EF920F93262FEE240DE040E050E0F2
:103A7000BC01CA010E94C21B81E090E00F91EF904F
:103A80000895EF920F93EE240EE0282F40E050E0CF
:103A9000BA01CA010E94C21B81E090E00F91EF9031
:103AA0000895EF920F93FC0180916C03882319F421
:103AB00080E090E013C06770862F806F442311F080
:103AC000862F886FE82E01E121E040E050E0BF0141
:103AD0008CEF96E00E94C21B81E090E00F91EF9086
:103AE0000895EF920F93FC0180916C03882319F4E1
:103AF00080E090E013C06770862F806E442311F041
:103B0000862F886EE82E01E121E040E050E0BF0101
:103B10008CEF96E00E94C21B81E090E00F91EF9045
:103B20000895EF920F93FC01E62E80916C03882399
:103B300019F480E090E00BC002E121E040E050E0A9
:103B4000BF018CEF96E00E94C21B81E090E00F91D4
:103B5000EF900895EF920F93FC01E62E80916C0395
:103B6000882319F480E090E00BC003E121E040E0FD
:103B700050E0BF018CEF96E00E94C21B81E090E014
:103B80000F91EF900895EF920F93FC01E62E809134
:103B90006C03882319F480E090E00BC00FE021E073
:103BA00040E050E0BF018CEF96E00E94C21B81E034
:103BB00090E00F91EF900895EF920F93FC01E62EA5
:103BC00080916C03882319F480E090E00BC000E141
:103BD00021E040E050E0BF018CEF96E00E94C21B64
:103BE00081E090E00F91EF900895EF920F93FC0128
:103BF000E42E04E124E0AB01BF0180E090E00E94EC
:103C0000C21B81E090E00F91EF900895982F8823D8
:103C100091F01092FD068091FD068093FC0681E0F4
:103C200080936E0380916E0380936C03BD9A87B777
:103C3000846087BF089587B78B7F87BF90936C039D
:103C4000BD98C59808950895EF920F93E0906C0386
:103C5000EE2069F5882359F1E092FD068091FD067A
:103C60008093FC0688E1ECE3F3E011928A95E9F792
:103C70000EE022E040E050E0BA018CEF96E00E94B6
:103C8000C21B81E080936E038BE390E099BD88BDF9
:103C900088B599B59BBD8ABD87E790E097BD86BD85
:103CA0001DBC1CBC87B7846087BFBE9A05C0BE9888
:103CB000C69887B78B7F87BF0F91EF900895EF92DB
:103CC0000F93E0906C03EE2071F5882361F1E09290
:103CD0006F0780916F0780936E0788E1E4E5F3E05A
:103CE00011928A95E9F70EE022E040E050E0BA0137
:103CF0008EE697E00E94C21B8BE390E090938700D2
:103D00008093860087E790E0909381008093800005
:103D1000109289001092880080917D0084608093C9
:103D20007D00139A07C013981B9880917D008B7FAC
:103D300080937D000F91EF90089580E00E94061E11
:103D400081E00E94241E81E00E945F1E809162003B
:103D5000846080936200089580E00E94061E809136
:103D600062008B7F8093620080E00E94241E80E0CE
:103D70000E945F1E10926E0381E00E94CA66089541
:103D800080E00E94241E80E00E945F1E81E00E946D
:103D9000CA66809162008B7F8093620088E1ECE3C9
:103DA000F3E011928A95E9F783E080934E038FEF59
:103DB00080933C038BE390E099BD88BD88B599B5AD
:103DC0009BBD8ABD87E790E097BD86BD81E00E94DC
:103DD000061E82E090E00E94C11608950E947F5264
:103DE000FC01808182FF02C0C79A0895C798089598
:103DF00008950E947F52FC01808182FF07C080E00D
:103E000090E0B79907C081E090E0089586B39927C4
:103E100080789070089508950E946E0E833021F08E
:103E20000E946E0E843021F480916F0399270895CB
:103E300081E090E00895089580916D039927089599
:103E400010926D03089590938403809383030895E3
:103E50008091810390918203089580E1E0E7F3E08F
:103E600011928A95E9F710928003109282031092C2
:103E700081038FEF9FE790938403809383030895DA
:103E800078941F920F920FB60F9211242F933F93A5
:103E90004F938F939F93EF93FF938091800388308C
:103EA00010F01092800380918003E82FFF27EE0F1F
:103EB000FF1FE059FC4F24B135B1208331838F5F60
:103EC00080938003109282031092810320E030E0FF
:103ED00047E0E0E7F3E081919191280F391F4150CD
:103EE00047FFF9CF309382032093810380918303AE
:103EF00090918403821793071CF481E080936D03F3
:103F0000FF91EF919F918F914F913F912F910F9042
:103F10000FBE0F901F9018955F926F927F928F92B5
:103F20009F92AF92BF92CF92DF92EF92FF920F9348
:103F30001F93CF93DF93EC015B0155246E567740BE
:103F400011F441E0542EF50190818181981709F018
:103F50008AC0552019F481E080936F0380916C032F
:103F6000882339F0EE240DE021E040E050E0BA0172
:103F700077C0552019F00E94EA2602C00E948F26C1
:103F80006C01009731F4EE2401E022E0AC01BC01A9
:103F900067C0FC01808599278370907082309105FD
:103FA00081F0833091051CF4019721F05CC00397E8
:103FB000D1F159C0F601E68001E022E040E050E096
:103FC0004DC0F6011681E12E01E022E040E050E014
:103FD00060817181C5010E940C1B0E948B26837039
:103FE000482F55274130510591F04230510524F4B6
:103FF0004115510541F037C04230510559F0433069
:10400000510571F030C0E12E06E022E026C0E12E1D
:1040100007E002C0E12E08E022E040E050E01DC0D1
:10402000E12E09E0F9CFF601E68001E0202F40E023
:1040300050E060817181C5010E940C1B0E948B269B
:104040009927AC014170507080FF04C0EE2403E05A
:1040500021E0E3CFEE2404E021E0F60160817181EC
:10406000C5010E940C1BF50181819927FC0133E0F9
:10407000EE0FFF1F3A95E1F7E81BF90BEA0DFB1D68
:10408000E280F380F50181819927FC0123E0EE0FA6
:10409000FF1F2A95E1F7E81BF90BEA0DFB1D648071
:1040A0007580F50181819927FC0103E0EE0FFF1F68
:1040B0000A95E1F7E81BF90BEA0DFB1D9680F50167
:1040C00081819927FC0113E0EE0FFF1F1A95E1F79C
:1040D000E81BF90BEA0DFB1D8084F501818199270E
:1040E000FC01B3E0EE0FFF1FBA95E1F7E81BF90BF7
:1040F000EA0DFB1D2781215027832223B1F4F5010E
:1041000081819927FC01A3E0EE0FFF1FAA95E1F73B
:10411000E81BF90BEA0DFB1D2683F50181818F5FFA
:1041200081838181803108F02183892D8B508230F9
:1041300038F4C7010E943C65082FCC24DD2407C059
:1041400010916C03112329F0CC24DD2403E010E04E
:1041500012C0C7010E94C0256C01009729F0182DDC
:10416000FC010085037005C001E0FEE09F1609F424
:1041700003E051101078802F9927813091050CF4BD
:1041800049C28330910524F0039709F406C142C265
:10419000C7010E948B1A982F829586958695837009
:1041A0008A83292F220F220F298371E0B72EBA8A22
:1041B00082E1888B82E0898BC114D10449F1F60138
:1041C0008481958197FF02C023602983812F9927DD
:1041D0008F779070892BE1F0F60180850E947D2910
:1041E0000F97B4F01F5FF60180850E948625892B0A
:1041F00029F410FF03C089818B258983212F207822
:10420000812F99278F71907095958795122F182B74
:10421000892D99278730910509F48FC08830910541
:104220009CF48230910509F47DC08330910524F41B
:10423000019709F440C0EEC18330910509F43BC0F9
:10424000069709F474C0E6C18A30910509F48BC061
:104250008B30910544F48830910509F478C00997B2
:1042600009F47BC0D7C10D970CF0D4C1C70153E04E
:10427000969587955A95E1F7907001960E948B1A52
:10428000982F82958695869583708A83990F990FCA
:104290009983FBE09F1611F418820AC087E0E82298
:1042A000FF24E4E5F2E0EE0EFF1EF701849188831F
:1042B00082E08A8B39C081E090E017FD892F212FA1
:1042C0002F702F3010F02EE001C021112F5F013030
:1042D00061F443E050E0990F990F20FD936026951B
:1042E0004150504057FFF7CF1BC0882331F0283092
:1042F00010F085E007C08DE005C0283010F48AE09A
:1043000001C082E043E050E0990F990F20FD9260D8
:1043100080FD9160269586954150504057FFF4CF1F
:10432000988378C180EC888384E0898B73C1F6011F
:1043300084818170482F61E005C0F601848182701C
:10434000482F62E0812F8F770E94971A24C0F601D0
:1043500084818470482F63E0F5CFF60184818870F2
:10436000482F64E0EFCFC7010E948B1A982F8295E7
:104370008695869583708A83990F990F93609983A8
:1043800082E08A8BF601848195818F7090708C5BBE
:104390009D4FFC01849188833DC183E08A8B01E0BD
:1043A000098B88E1888B892D99278D30910509F437
:1043B000D9C08E309105BCF48430910509F4BAC09F
:1043C0008530910544F48130910509F441C003978B
:1043D00009F49AC011C18530910509F4B8C00B9752
:1043E0000CF40AC10FC08231910524F40F970CF030
:1043F000C9C0C3C0843191050CF4DFC0449709F4EF
:10440000ECC0FAC088E090E0E80EF91EC70143E076
:10441000969587954A95E1F78F7380688A83C701DF
:104420008095909535E0969587953A95E1F7282FF8
:10443000207720688E2D8770282B29839CE0991681
:1044400011F428602983898191E089278983D4C068
:10445000F601808599278C7090700897B9F48FE3E6
:104460008A83812F99278F779070009731F08F374B
:10447000910511F4117801C01F5F1983CE010396D5
:10448000BC01C7010E94D41A885EB5C017FF02C0E4
:1044900080E601C080E48983F60180850E947D2941
:1044A000212F3327BE016E5F7F4F0F97B4F0C901F4
:1044B0008F779070009731F08F37910511F412E0EB
:1044C00001C01D5F812F86958F709981982B9983EC
:1044D00010FF2BC09061998328C0C9018F7790701D
:1044E000009731F08F37910511F411E001C01F5F83
:1044F0001F702981212B2983F6018481958197FFE3
:1045000014C02061298311C080E88983F6012481C9
:104510002F70822F806889838481958197FF02C0E4
:1045200020692983CE010296BC01C7010E94D41ADA
:10453000805F61C080EA8983F6018481958124E0EF
:10454000969587952A95E1F78F70806B09C080EA70
:104550008983F60184819581892F99278F70806ADC
:104560008983E0CF1982CE010296BC01C7010E9467
:10457000D41A805F888B098B3FC08FEF8A831982A2
:1045800081E029C0F1E19F1611F488E709C080E1BC
:10459000981611F484E704C09FE0991611F48CE793
:1045A0008B838F2D9927982F93708B81892B8B83E9
:1045B000EA82898280E2888B0DC080E78A83E2E10B
:1045C0009E1611F488E78A838E2D87709A81982B26
:1045D0009A8389828AE0898B0FC0872D99278370FF
:1045E0008C6E8B836A828982CE010496BC01C701DE
:1045F0000E94D41A805E888B20E0988996959695C3
:104600009695915031F0FE01E90FF11D8081282728
:10461000F8CF28838A89833011F010926E03DF91DE
:10462000CF911F910F91FF90EF90DF90CF90BF90AF
:10463000AF909F908F907F906F905F900895CF93F1
:10464000DF93DC01FC018489882319F42589222366
:1046500061F021E0882321F08150FD01848B21C08D
:10466000FD0185898150858B1CC0FD0182898330C5
:1046700019F487898823A9F4FD019389892F8695E8
:1046800086958695E80FF11D8081282F3327892F85
:1046900099278770907002C0359527958A95E2F723
:1046A0002170FD013289832F99278230910531F0E5
:1046B00083309105CCF0039721F016C0CBE6D0E013
:1046C00015C0222319F0C7E7D0E002C0CEECD0E03D
:1046D000FD018389882351F48689882339F482E097
:1046E000858B81E0868B2BC0C7EDD0E0FD018389EF
:1046F000882329F58589882311F58189882399F4F0
:1047000080916E038823D9F480916C038823B9F4D7
:1047100081E00E94A052882319F0C35BDF4E0FC0D6
:10472000CD5ED94F0CC0832F99278130910529F098
:10473000029729F4C857DD4F02C0C05FDA4FCE019F
:10474000DF91CF910895DC01FC018489882319F45D
:104750008589882311F021E02BC0FD013389932F37
:104760009150938B8289833069F42789222351F4F5
:10477000892F992787709070079721F481E0878BA4
:10478000338B16C0FD01178A9389892F86958695EC
:104790008695E80FF11D8081282F3327892F9927CF
:1047A0008770907002C0359527958A95E2F7217041
:1047B000FD01828999278230910549F08330910566
:1047C0001CF4019761F01BC0039789F018C02223E5
:1047D00019F08CE590E0089580E190E0089522239F
:1047E00019F08EEB90E008958CE190E0089522237B
:1047F00019F08BE390E0089587E690E008958BE34D
:1048000090E008950895FC018089838B818982302E
:1048100010F482E0818B8289992781309105B4F070
:10482000833091051CF0039761F010C081E00E9475
:10483000A052882319F08DE490E1089583E196E079
:10484000089580E1848B82E390E0089582E390E014
:10485000089508951F920F920FB60F9211241F937F
:104860002F933F934F935F936F937F938F939F9378
:10487000AF93BF93CF93DF93EF93FF9380916C033C
:10488000882331F00E941C1F882311F010924D03E1
:1048900080913A038823A1F080916E03882329F048
:1048A0008BE390E099BD88BD02C019BC18BC8BE3B6
:1048B00090E09BBD8ABD87E790E097BD86BD5EC056
:1048C000CCE3D3E0CE010E941F23AC019C01255014
:1048D00030408CB59DB58217930718F457BD46BD7F
:1048E0000EC08CB59DB5C29697BD86BDCE010E9407
:1048F00003242CB53DB5280F391F37BD26BD809147
:104900004F03882381F510915103112361F58091A4
:104910004D03882381F481E080933A0386B7846055
:1049200086BF78946CEF76E08CE393E00E948C1F56
:10493000F89410923A0380914D038150898B8091B5
:104940004C038B8B80914E03833049F480916C0330
:10495000882311F084E101C080E18C8B01C01C8BA5
:104960001D8A1F8A1E8A8CE393E00E94A323992745
:104970009BBD8ABD8AB59BB599BD88BDFF91EF915E
:10498000DF91CF91BF91AF919F918F917F916F9167
:104990005F914F913F912F911F910F900FBE0F90FC
:1049A0001F9018951F920F920FB60F9211241F930C
:1049B0002F933F934F935F936F937F938F939F9327
:1049C000AF93BF93CF93DF93EF93FF9380913B031C
:1049D0008823B1F080916E03882339F08BE390E057
:1049E000909387008093860004C0109287001092F5
:1049F000860087E790E0909381008093800064C0F8
:104A0000C4E5D3E0CE010E941F23AC019C012550D8
:104A1000304080918800909189008217930728F494
:104A2000509381004093800016C08091880090913F
:104A30008900C2969093810080938000CE010E94ED
:104A400003242091880030918900280F391F30936A
:104A500081002093800080916703882361F5109185
:104A60006903112341F580916503882391F481E066
:104A700080933B0380917C00846080937C007894D9
:104A80006EE677E084E593E00E948C1FF894109224
:104A90003B03809165038150898B809164038B8BEC
:104AA00080916603833019F480E18C8B01C01C8BEC
:104AB0001D8A1F8A1E8A84E593E00E94A3239927FA
:104AC0009093870080938600FF91EF91DF91CF91C3
:104AD000BF91AF919F918F917F916F915F914F9116
:104AE0003F912F911F910F900FBE0F901F9018951F
:104AF00080E892E0E0EEF7E011920197E9F710927A
:104B00008603109285031092600A08958F7020E04A
:104B100030E08550823010F421E030E0C901089582
:104B20000F931F93CF93DF93CDB7DEB724970FB6C4
:104B3000F894DEBF0FBECDBF8FEF9FEFAFEFBFEF9B
:104B400089839A83AB83BC8300E210E044E050E0A9
:104B5000B801CE0101960E9451670E94720E0C5F4F
:104B60001F4F8FE00C3D180788F324960FB6F8947A
:104B7000DEBF0FBECDBFDF91CF911F910F91089582
:104B80009C01009741F408958AE0A89FC001112478
:104B90008052984F0895A0E0B091600AAB17A0F43E
:104BA00040E050E0BA01FA01E60FF71FE052F84F7B
:104BB000808191818217930739F3AF5F6F5F7F4FD9
:104BC000475F5F4FAB1778F380E090E0089508955A
:104BD000CF92DF92EF92FF920F931F93CF93DF93C9
:104BE000CDB7DEB723970FB6F894DEBF0FBECDBFAB
:104BF0007C016C010894C108D1088FEFC81687E2C8
:104C0000D806A0F5C7010E94C0258C01892B09F0A8
:104C100072C02091600A203450F48AE0289F8001FD
:104C200011240052184F2F5F2093600A22C000EE1B
:104C300017E0B80120E030E0A901AFE3F901E40F8B
:104C4000F51FE052F84F9185F8018185891708F426
:104C50008B01A1504F5F5F4F275F3F4F665F7F4FD4
:104C6000A7FFECCFF8018185882319F480E090E05C
:104C700043C0F801E082F182FFEFCF16F7E2DF06D2
:104C8000E0F480E2E82EF12CA89543E050E0B70173
:104C9000CE0101960E94356729813A81F801808111
:104CA000918128173907C9F084E090E0E80EF91ED9
:104CB0009CEDE9169FE0F90638F3F80180819181B7
:104CC0008F3F910519F010F083E00BC088E00E943F
:104CD000A052882321F083E003C08B8101C082E0D1
:104CE000F801808780E8F801868314821582128299
:104CF000138211861782C80123960FB6F894DEBF7F
:104D00000FBECDBFDF91CF911F910F91FF90EF901C
:104D1000DF90CF9008958091870399270895EF92AF
:104D2000FF921F93CF93DF939091600A992319F418
:104D300080E090E049C0809185038F5F8093850378
:104D4000891738F0809187038F5F809387031092D3
:104D50008503909185038AE0989FE0011124C05259
:104D6000D84F80918703992787709070892BA9F479
:104D70001E81E12EFF24C7018F779070892B69F087
:104D800088850E948625892B41F0E0FC06C01F5FC4
:104D9000612F888199810E94071C80918703992740
:104DA00087709070049751F488859927837090706C
:104DB000019721F4888199810E94711C89858F3F18
:104DC00011F08F5F8987CE01DF91CF911F91FF9006
:104DD000EF9008959091600A992319F480E090E093
:104DE0000895809186038F5F80938603891710F062
:104DF00010928603909186038AE0989FC001112447
:104E00008052984F089508950E94C025FC01009794
:104E100009F4089580859927089508950E94C02572
:104E2000FC01009709F40895868199270895089553
:104E30000E94C025FC01009709F4089584819581A2
:104E400008950895BF92CF92DF92EF92FF920F9351
:104E50001F93CF93DF93CDB7DEB723970FB6F894A8
:104E6000DEBF0FBECDBF7C01B62E0E94E825FC013F
:104E7000892BB1F180858B1599F1B08611869FEF52
:104E8000C92ED92E00E210E0A89543E050E0B80109
:104E9000CE0101960E94356789819A818E159F0502
:104EA00011F468010DC0D7FE05C028E280309207DA
:104EB00008F068010C5F1F4F2FE00C3D120720F334
:104EC0008E159F0511F0D7FC0BC0BB82E982FA82D8
:104ED000A89544E050E0B601CE0101960E945167CA
:104EE00023960FB6F894DEBF0FBECDBFDF91CF91F2
:104EF0001F910F91FF90EF90DF90CF90BF9008959A
:104F0000CF92DF92FF920F931F93CF93DF93EC0129
:104F1000F62E142F892B09F480C088850E947D29E4
:104F2000482F5885752F73708F2D99278F77907024
:104F3000242F3327281739071CF420E8F222F42AFB
:104F40006E816F1509F469C01986112319F08F81DC
:104F500081608F838F2D992780789070C62EDD24F5
:104F60009601207830708217930799F1C6018F77E8
:104F70009070009711F020E8F2227330B1F4892B81
:104F8000D1F4852F99278C709070089711F58F2D8B
:104F900099278F779070892BE1F48F2D8160682F8E
:104FA000888199810E94071C14C0892B49F088814F
:104FB00099810E94071C888199810E942A1C09C03E
:104FC00060E0888199810E94071C888199810E94F4
:104FD000501CFE820F2D1127C8018F779070892BEE
:104FE000B9F088850E948625892B91F000FD03C0C9
:104FF0008F2D8F5F08C00894C108D1080C151D05BE
:1050000039F48F2D8150682F888199810E94071C67
:105010006F2D888199810E94071CDF91CF911F918C
:105020000F91FF90DF90CF900895FF920F931F9301
:10503000CF93DF93EC01162FF42E0E946E0E833077
:1050400009F01078CE010E94E825EC010E814F2D69
:10505000612F0E9480278A819B810097B1F00E9476
:10506000E825EC018E81282F332720783070802F9F
:105070009927807890702817390711F080E8182751
:105080004F2D612FCE010E948027DF91CF911F917C
:105090000F91FF900895EF92FF920F931F93CF937C
:1050A000DF93EC017B01892BE1F10C811D81061757
:1050B0001707B9F11986442319F08F8181608F8316
:1050C000EC82FD82888599278370907081309105EC
:1050D00031F0813091052CF104971CF51BC098012B
:1050E00020703078C701807090782817390729F030
:1050F0006E81888199810E94071C0F7010708FE06B
:10510000E822FF240E151F0561F0888199810E9415
:10511000711C07C00E251F25B801888199810E9446
:10512000911CDF91CF911F910F91FF90EF90089507
:10513000FF920F931F93CF93DF938B01F42E0E9466
:10514000E825EC01892B49F18A819B81892B01F1AA
:10515000C8018F709F7B4F2DBC01CE010E944B2850
:105160008A819B810E94E825EC01892BB1F0C8015E
:1051700080709074880F991F007F107024E016953E
:1051800007952A95E1F7802B912B4F2DBC0102C08A
:105190004F2DB801CE010E944B28DF91CF911F9176
:1051A0000F91FF900895EF92FF920F931F93CF936B
:1051B000DF937C018B010E94E825EC01892B61F0D3
:1051C000C8010E94E825FC01892B31F00A831B836A
:1051D0001986E282F3821186DF91CF911F910F91A0
:1051E000FF90EF900895009759F00E94E825FC0188
:1051F000892B31F082819381128213821186F3CF41
:1052000008950895EF92FF920F931F93CF93DF932A
:10521000CDB7DEB726970FB6F894DEBF0FBECDBF71
:105220007C010E94C0258C01892BD9F0B701CE01E9
:1052300001960E94B854F801448155816681CE01DF
:1052400001960E949B54AE014F5F5F4F6AE08FEF63
:105250000E943B55F801448155816681C7010E9437
:10526000EE2926960FB6F894DEBF0FBECDBFDF91B4
:10527000CF911F910F91FF90EF9008951F93CF93BF
:10528000DF9310E0C0EED7E09091600A1917F0F4B8
:105290008985899FC00111248035910534F08E8164
:1052A00099278F779070892B59F08E8180788E8323
:1052B000888199810E942A1C888199810E940229F3
:1052C0001F5F2A969091600A191710F3DF91CF9112
:1052D0001F9108950F931F938C01C8010E94F51D23
:1052E00084E00E94411D61E0C8010E94311D8AE0F6
:1052F0000E94411D1F910F910895E82FFF27EF7025
:10530000F070E455FC4F84919927089588E893E064
:1053100008958091960382FF05C080918A03909141
:105320008B030895809188039091890308950895CF
:105330008091960382608093960308950F931F9344
:10534000CF93DF93C8E8D3E08091960399278C012F
:105350000170107080FF03C080E090E021C0609178
:105360008E0370918F03809190039091910361154A
:1053700071058105910531F00E948A14882311F48A
:10538000C8010EC01A821B821A8A1B8A10928903D6
:10539000109288031E861C8A0E942B0E81E090E0EA
:1053A000DF91CF911F910F9108959C0180918A0305
:1053B00090918B03892B11F4C90108952F703F7BC5
:1053C00077FD3064CB018F70907044E0880F991F97
:1053D0004A95E1F7822B932B08950895FC01809163
:1053E00088039091890320918A0330918B03E817F9
:1053F000F907F9F460939803232BB1F080918C03A3
:1054000090918D03F4E096958795FA95E1F7BC01AC
:105410006F707070892F99278695869580FD7068CA
:10542000CA010E94D5290FC050938D0340938C036D
:105430000EC0E217F30769F4BA0180918C039091D2
:105440008D030E94D52990938D0380938C030E9435
:105450002B0E089508959C01892B69F410929603F0
:1054600010928E0310928F0310929003109291036A
:105470000E949E2908956093980350938D03409352
:105480008C038091CA069091CB06A091CC06B09176
:10549000CD0688519C4FAF4FBF4F816080938E03E4
:1054A00090938F03A0939003B09391038091960300
:1054B00082FF10C081608B7F8093960330938B03B3
:1054C00020938A03B90180918803909189030E94F7
:1054D000D32807C08E7F809396033093890320934F
:1054E00088030E942B0E08950895209196032B7F28
:1054F00021602093960390938B0380938A0380917D
:105500008C0390918D030E94D52990938D038093F5
:105510008C030E942B0E0895CF93DF93EB018093B1
:1055200097030E947D2980939903209759F04CE9B5
:1055300053E060E070E0CE010E94B95ED0939B031F
:10554000C0939A030E942B0EDF91CF910895CF93C1
:10555000C82F882319F064ED71E002C064EF71E098
:1055600084E00E949719CC2319F06CEC71E002C022
:105570006CEE71E085E00E949719CC2319F064EC81
:1055800071E002C064EE71E086E00E949719CC23BE
:1055900019F06CEB71E002C06CED71E087E00E94E5
:1055A0009719CF910895CF93DF93C82FDD27C4FFBC
:1055B00002C083E001C085EA0E941A18C0FF02C041
:1055C00084E001C085EA0E941A18C1FF02C085E08C
:1055D00001C085EA0E941A18C2FF02C086E001C01D
:1055E00085EA0E941A18C3FF02C087E001C085EA5D
:1055F0000E941A18DF91CF9108958093A8030E940A
:105600002B0E0895882319F06CE971E002C064EA5A
:1056100071E082E00E94971908950895882319F097
:105620006CEA71E002C064EB71E081E00E949719BE
:10563000089508950F931F93CF9308E813E0C09146
:10564000A803CC2399F060E081E00E9468188C2FB9
:1056500081500E94A251BC0182E00E94F019109278
:10566000A80388EE93E00E94C11602C0882319F0B7
:105670000E948F1903C0682F0E94681880918803C8
:1056800090918903892BF9F00E947F52FC0182815D
:10569000938140918803509189038417950749F4B9
:1056A0002185328580919A0390919B0328173907B1
:1056B00051F04283538380919A0390919B03818799
:1056C00092870E9406522091880330918903211508
:1056D000310529F4F80124833583108A17868091D7
:1056E000960382FD0DC08091920390919303A09147
:1056F0009403B09195030097A105B10519F105C078
:105700006CEB73E082E00E94F0198091920390911B
:105710009303A0919403B0919503BF93AF939F938C
:105720008F938FEB93E09F938F9382E08F930E94F0
:10573000461A8DB79EB707960FB6F8949EBF0FBE58
:105740008DBF43C02115310531F462ED73E082E075
:105750000E94F01918C03F932F9389ED93E09F9317
:105760008F93C2E0CF930E94461A809196030F90C8
:105770000F900F900F900F9080FF02C08C2F01C0F0
:1057800080E20E941A18C09197030E946E0E853025
:1057900010F085E00EC0833061F48C2F9927837060
:1057A000907023E0880F991F2A95E1F7845A9C4F47
:1057B00008C0992703E0880F991F0A95E1F78458DC
:1057C0009C4FBC0182E00E94F0196CE080E00E94D6
:1057D00068188091980399278F7790709F938F9383
:1057E0008EED93E09F938F9382E08F930E94461AF1
:1057F000809197039927837090700F900F900F906E
:105800000F900F90019779F483E10E943D17882350
:1058100031F080E00E941A1864E671E010C080E266
:105820000E941A180FC080E00E941A1880919803F5
:1058300087FF03C06CE372E002C064E372E080E0C3
:105840000E9497190E946E0EC82F813049F488E09B
:105850000E946D51AC0160E08C2F0E942A19E0C0BB
:1058600040E050E060E0862F0E94DA18C0E08AE055
:105870000E943D17882371F080918A0390918B03D9
:10588000892B39F48091970399278370907003973F
:1058900009F4C1E060E081E00E9468188091920301
:1058A00090919303A0919403B09195030097A10563
:1058B000B10509F442C08DE00E943D17882329F408
:1058C0008EE00E943D17882381F182EE93E09F9342
:1058D0008F93C2E0CF930E94461A8DE00E943D173D
:1058E0000F900F900F90882379F06CEA71E081E0BF
:1058F0000E94971964EA71E08C2F0E9497196CE25C
:1059000071E08EE09BE20EC064EB71E081E00E94EA
:1059100097196CE971E08C2F0E9497196CE271E085
:1059200082E09BE20E94A1187BC086E00E946D513C
:10593000BC0182E00E94F01944C080918A039091DA
:105940008B03009769F19F938F938EEE93E09F9363
:105950008F9382E08F930E94461A80918C039091DE
:105960008D0314E0969587951A95E1F7282F2F70EF
:10597000892F9927869586950F900F900F900F90FD
:105980000F9080FD2061822F0E94D32ACC2321F02A
:105990008CE30E941A1815C080E20E941A182CC0CD
:1059A0008CE993E09F938F9383EF93E09F938F9382
:1059B00082E08F930E94461A0F900F900F900F90E5
:1059C0000F90CC23C9F080918A0390918B03892B8F
:1059D00099F480918C0390918D03A4E0969587951E
:1059E000AA95E1F78F7080610E94D32A81E00E941E
:1059F000A72A6CEF71E011C020918C032F70809169
:105A00008C0390918D0397FD2061822F0E94D32AF1
:105A100080E00E94A72A64E072E083E00E94971968
:105A2000CF911F910F91089560918E0370918F0314
:105A30008091900390919103611571058105910505
:105A400061F00E948A14882341F010928E03109214
:105A50008F03109290031092910308950895EF928E
:105A6000FF920F931F93CF93DF93EC01E8E8EE2EA4
:105A7000E3E0FE2E81319105CCF48F3091050CF0DE
:105A8000D0C08A30910509F4F4C18B30910534F40B
:105A9000009709F40BC197FDFBC11BC18C30910528
:105AA00009F462C00D970CF07EC044C185319105A8
:105AB000D9F18631910574F48231910509F4D1C090
:105AC000823191050CF4E4C083319105D1F1449702
:105AD000B1F0DEC18F3891056CF48D3891050CF072
:105AE00062C08C31910509F4B4C08A38910509F47B
:105AF000CDC1CEC18339910509F4C8C1C9C1809116
:105B0000980399278F7790702091990333278217F4
:105B100093070CF0BDC10E946E0E833009F0B8C12E
:105B2000809198038F5F1DC020919803822F992741
:105B30008F779070892B09F4ABC121502093980383
:105B4000A5C180919703992783709070019729F4DC
:105B500064E671E080E00E94971980919803809537
:105B600080788093980392C18AE00E943D17882331
:105B700099F080918A0390918B03892B69F0809131
:105B80008C0390918D0320E030E48227932790933B
:105B90008D0380938C037AC180918C0390918D0347
:105BA00020E030E850C08091920390919303A0913F
:105BB0009403B09195030097A105B10581F120915F
:105BC00092033091930321503040220F331FCE01B6
:105BD0008F7790700E9709F42160C7FF1AC041E0DB
:105BE00060E0C9010E940F6460E070E0CB010E9498
:105BF000A11864E172E081E00E9497196CE172E003
:105C000082E00E949719F701128613861486158682
:105C10003DC141E0642FC9010E940F6437C1C7FD37
:105C200035C11C2F1D508AE00E943D1781111C5F59
:105C300021E030E002C0220F331F1A95E2F7809175
:105C40008C0390918D0382279327F701848395839A
:105C50001DC16CE380918803909189030E94FD1C13
:105C600015C1F89483E00E942F0E882319F084E078
:105C70000E94CA6683E10E943D17882339F06BE4D5
:105C800080918803909189030E94FD1C7894FEC046
:105C90008AE00E943D17811182E00E942F0E882326
:105CA00009F4F4C084E00E94CA66F0C080919203B7
:105CB00090919303A0919403B09195030097A1054F
:105CC000B10539F48FEF0E94135181E00E941A2B25
:105CD000DFC08091920390919303A0919403B091BF
:105CE00095039C01AD0163E0220F331F441F551F34
:105CF0006A95D1F7280F391F4A1F5B1F280F391FDC
:105D00004A1F5B1FCE01AA2797FDA095BA2F280F27
:105D1000391F4A1F5B1F2030F8E23F07F0E04F07B2
:105D2000F0E05F070CF0B4C0F701228733874487A7
:105D30005587ACC0C8E8D3E020919203309193031B
:105D4000409194035091950360918A0370918B0365
:105D5000211531054105510509F47FC06115710513
:105D600019F10091880310918903C801AA27BB2764
:105D700082179307A407B50741F0CB01AA27BB27D9
:105D800082179307A407B50779F4809196038E7F55
:105D9000F7018687C8010E94F328F7011282138257
:105DA000109289031092880380918803909189034F
:105DB0009C01442755278091920390919303A091D1
:105DC0009403B091950360919603281739074A0709
:105DD0005B0729F481E068276B7F6E8745C06C7F85
:105DE0006E871A8A1B8A1C8A60919C0381E00E943C
:105DF000681880E00E946D51BC0182E00E94F01999
:105E000080919603992796958795969587959C01FD
:105E10002170307080FD11C02A833B832C833D8329
:105E200030938903209388031F86609192037091B9
:105E300093038FEF0E94F6530BC040919203509151
:105E4000930360918803709189038FEF0E9412542D
:105E5000809196038B7F8E8707C0672B29F48091F2
:105E600096038460F70186871A861B861C861D862A
:105E70000DC010929203109293031092940310920B
:105E80009503809196038B7F809396030E942B0E3F
:105E9000DF91CF911F910F91FF90EF900895FC013A
:105EA000EC5BFF4F8081E454F040882319F480E0DC
:105EB00090E00895E95BFF4F8081E754F04088232C
:105EC00029F48481883511F0883719F481E090E055
:105ED000089580E090E008950895CF93DF93EC015A
:105EE0000E944F2F882319F480E090E01FC0FE012C
:105EF000E95BFF4F8081882351F4CC5BDF4F8881C1
:105F0000C454D040823018F481E090E00FC080810A
:105F1000882311F08C8101C08D81992787FD909590
:105F2000809590958827990F881F9927DF91CF91A9
:105F30000895CF93C82FCF7719F480E090E029C05F
:105F4000862F0E947D29282F33272B31310589F098
:105F50002C31310524F42E30310529F017C02C31B5
:105F6000310569F013C0EC2FFF27EB5CFB4F8491E8
:105F70000BC0EC2FFF27E75EFB4F849105C0EC2F91
:105F8000FF27E450FC4F8491992703C0CF5F8C2FEB
:105F90009927CF910895CF93C82FCF7719F480E038
:105FA00090E02EC0C150862F0E947D29282F3327D4
:105FB0002B31310579F02C31310524F42E303105A7
:105FC00029F01CC02C31310569F018C08C2F99279D
:105FD00008960DC083E0C89FC00111240B966EE0A7
:105FE00070E007C08C2F9927880F991F079669E0EA
:105FF00070E00E94986CCB01992702C08C2F9927E2
:10600000CF910895019791F40E947F52FC01818104
:10601000882311F484E608C0843011F485E604C0B6
:106020008150843008F08150992708958FEF9FEFB9
:10603000089508951F93CF93C82FFB01142F8181DA
:10604000282F332782819927982F8827282B392BAF
:10605000C90101978F5F974210F062E010C01123D1
:1060600021F0C9010E94E82503C0C9010E94C02592
:10607000009751F4112311F06BE001C06AE08C2FFE
:106080000E94C01980E090E0CF911F910895EF9297
:10609000FF920F931F93CF93DF93EB01E42E41E028
:1060A0000E941A308C01892B19F48FEF90E064C0A4
:1060B0000E94FD1A882319F088E090E05DC0FB8003
:1060C000EE2051F021E0F21639F4F82EF80180812B
:1060D00091810E942A1C08C0EE2031F0F8016085F1
:1060E0008B810E94CB2FF82E6C81862F992785FFFC
:1060F00002C0F0E8FF2AF801C481D581DF7784FD72
:10610000D06867FF05C0C07F8F709070C82BD92BF7
:106110002F2D332720783070F8016681862F99273C
:10612000807890702817390731F0607840E08081DE
:1061300091810E94152840E06F2DF80180819181A6
:106140000E94152840E0BE01F801808191810E94E3
:106150009828F801808191810E9402290E946E0E88
:10616000833019F480E090E007C0823019F481E4B4
:1061700090E002C082E490E0DF91CF911F910F91F7
:10618000FF90EF90089541E00E94473099270895CD
:1061900040E00E944730992708951F93CF93DF93E3
:1061A000182F40E0812F0E941A30EC01892BF1F06A
:1061B00060E0812F0E94C01968858E810E94992F0E
:1061C000682F812F0E94C0196C816F708C819D8116
:1061D00097FD60618E8187FD6062812F0E94C019EA
:1061E0008E818F77682F812F0E94C0198FEF90E0EA
:1061F000DF91CF911F9108951F93CF93DF93182FB5
:1062000040E0812F0E941A30EC01892BC9F060E038
:10621000812F0E94C01988858370682F812F0E946A
:10622000C01988850E947D29682F812F0E94C0197E
:106230006FEF812F0E94C0196FEF812F0E94C0194C
:106240008FEF90E0DF91CF911F9108950F931F93EF
:10625000CF93DF938B0141E00E941A30EC01892B30
:1062600019F48FEF90E014C08C819D818070F8014B
:1062700023813327822B932B40E0BC0188819981B5
:106280000E949828888199810E94022980E090E0EC
:10629000DF91CF911F910F9108950F931F93CF938B
:1062A000DF938B0141E00E941A30EC01892B19F435
:1062B0008FEF90E018C02C813D81307CF801838104
:1062C00099278F739070982F8827282B392B40E0BF
:1062D000B901888199810E949828888199810E94BA
:1062E000022980E090E0DF91CF911F910F910895F6
:1062F0001F93CF93DF93182F40E0812F0E941A3015
:10630000EC01892B41F060E0812F0E94C0196C8163
:10631000812F0E94C0198FEF90E0DF91CF911F91E4
:1063200008951F93CF93DF93182F40E0812F0E9491
:106330001A30EC01892B69F060E0812F0E94C019AE
:106340008C819D81892F99278F73682F812F0E94BF
:10635000C0198FEF90E0DF91CF911F910895DF92E8
:10636000EF92FF920F931F93CF93DF93982F8B01A0
:10637000823008F059C088E4989F7001112489EA9E
:1063800093E0E80EF91EFB018181C82FDD27828191
:10639000992787709070982F8827C82BD92B219721
:1063A000F7E0C83FDF0718F082E090E03FC00E94AE
:1063B0006E0E833039F00E946E0E823019F086E046
:1063C00090E034C0CC0FDD1FF801628167FFC1602F
:1063D000862F9927E6E096958795EA95E1F771E093
:1063E000D72ED82287010B5B1F4FF8018081918146
:1063F000FFEF8F3F9F0749F040E0642F0E940F643A
:106400008FEF9FEFF8018083918340E06D2DCE01E7
:106410000E940F64882319F489E090E007C0DD2012
:1064200019F0F801C083D18380E090E0DF91CF9133
:106430001F910F91FF90EF90DF900895FF920F93BF
:106440001F93CF93F82EFB018181082F11278281A2
:10645000992787709070982F8827082B192B87E031
:10646000083F180718F082E090E01CC0C8010E94A5
:10647000FF62873611F0873411F4C4E001C0C0E038
:10648000C801880F991F0E943C65039709F4C160F9
:1064900060E08F2D0E94C0196C2F8F2D0E94C019B3
:1064A0008FEF90E0CF911F910F91FF9008951F9370
:1064B000CF93182FFB01C181CC2319F482E090E027
:1064C0000FC060E00E94C019EC2FFF27EE5DF44F73
:1064D00080818095682F812F0E94C0198FEF90E0F6
:1064E000CF911F9108951F93CF93182FFB01C18166
:1064F000C150C03218F082E090E015C060E00E9408
:10650000C01960E08C2F0E941A5C682F812F0E94B6
:10651000C01961E08C2F0E941A5C682F812F0E94A5
:10652000C0198FEF90E0CF911F9108950E94355CC4
:1065300080E090E008951F93CF93182FFB01818195
:106540009927009719F0039729F008C0C091610AB4
:10655000CC0F07C0C091620AC17003C082E090E016
:106560000AC060E0812F0E94C0196C2F812F0E9409
:10657000C0198FEF90E0CF911F910895FB018181A9
:106580009281282F33272115310521F02330310541
:1065900059F014C0913490F4892F9927019695955C
:1065A00087958093610A0DC08091620A992311F04A
:1065B000816001C08E7F8093620A03C082E090E018
:1065C000089580E090E008950895EF92FF920F9370
:1065D0001F93CF93DF93CDB7DEB760970FB6F894D4
:1065E000DEBF0FBECDBFF82E63E00E94C01961E090
:1065F0008F2D0E94C01964E08F2D0E94C01962E0A7
:106600008F2D0E94C01964E08F2D0E94C0190E9436
:10661000BC52DC01CB01BF93AF939F938F9384E473
:1066200094E09F938F938E010F5F1F4F1F930F93E3
:106630000E946D678DB79EB708960FB6F8949EBFFF
:106640000FBE8DBF33E0E32EF80191919295907FBC
:1066500081918F018053982B692F8F2D0E94C01933
:10666000EA94E7FEF1CF80E090E060960FB6F894F0
:10667000DEBF0FBECDBFDF91CF911F910F91FF9075
:10668000EF9008951F93CF93182FC0E00E946E0ED5
:10669000982F8250823008F4C8E0923009F4C0612B
:1066A0006C2F812F0E94C0198FEF90E0CF911F9126
:1066B00008951F93CF93DF93182FFB018181282F1B
:1066C000332782819927982F8827822B932B0E942A
:1066D0000230EC0197FF03C082E090E00AC060E066
:1066E000812F0E94C0196C2F812F0E94C0198FEF3B
:1066F00090E0DF91CF911F91089560E00E94C01952
:1067000082E00E942F0E8FEF90E0089580E00E94BB
:106710002F0E80E090E0089583E00E942F0E80E02D
:1067200090E0089580E090E008951F93CF93DF9369
:10673000182F0E946566EC0160E084E0989F812D2F
:106740009927112480FD61E0CE01892F9927829538
:106750008695877080FD6460C0FD6860D7FD6062CB
:10676000CE7FDF71209709F06068812F0E94C019E9
:10677000209791F060E0C1FD61E0C2FD6064C97FD7
:10678000209709F06068812F0E94C019CD2B21F05D
:1067900060E0812F0E94C0198FEF90E0DF91CF91D0
:1067A0001F9108950F931F93CF93DF93182FC0EE7F
:1067B000D7E000E08091600A081778F58F8180FFAC
:1067C00029C068858E810E94992F682F812F0E9491
:1067D000C0196C81812F0E94C0196881812F0E948D
:1067E000C01988819981892F9927682F6F738C81AF
:1067F0009D8197FD60648E8187FD6068812F0E9476
:10680000C0198E818F77682F812F0E94C0198F81C8
:106810008E7F8F830F5F2A96CDCF80E890E0DF9147
:10682000CF911F910F9108956F927F928F929F92B7
:10683000AF92BF92CF92DF92EF92FF920F931F938E
:10684000CF93DF93CDB7DEB7C254D0400FB6F894E4
:10685000DEBF0FBECDBF882E01E010E0AA249A2C27
:10686000B1E0BB2E7E01E00EF11E3701C92CDD2404
:10687000F601ED5DF34FE081EE2319F4095F1F4F40
:106880002CC0EB2141F1F70101937F01812F992762
:1068900087708083C80101970E94FF62982F873418
:1068A00011F0873621F4F701808180688083973466
:1068B00011F0923521F4F70180818064808308947F
:1068C000E11CF11CA394F601ED5DF34F9B2D909517
:1068D000808189238083BB0C19F49394F1E0BF2E4F
:1068E0000F5F1F4FF7E0093F1F0720F48FE18A1564
:1068F00008F0BCCF6A2D882D0E94C019DD247301D9
:106900000A2D11270115110581F0F70181917F01F1
:10691000682F882D0E94C019D3942D2D3327C801CC
:10692000800F911F2817390784F38FEF90E0CE5B1B
:10693000DF4F0FB6F894DEBF0FBECDBFDF91CF9112
:106940001F910F91FF90EF90DF90CF90BF90AF908D
:106950009F908F907F906F900895CF92DF92EF92EB
:10696000FF920F931F93CF93DF93D82ECC24809167
:10697000610A882309F454C0F8948C2D992787FD67
:106980009095880F991F9C012D51354F8C010D5505
:10699000154FEC01CD59D54F4881942F9095D801D2
:1069A0008C918923F901E080E82A5981952F9095EF
:1069B000F80181818923F901F180F82A2E2D3327EE
:1069C00027FD3095842F99272817390749F42F2D53
:1069D000332727FD3095852F99272817390799F0F8
:1069E0008C2D8F5F682F8D2D0E94C0196E2D8D2DDF
:1069F0000E94C0196F2D8D2D0E94C019E882F98266
:106A0000F801118210827894C3942C2D332727FD2E
:106A100030958091610A9927281739070CF4ACCF7B
:106A200060E08D2D0E94C0198FEF90E0DF91CF9133
:106A30001F910F91FF90EF90DF90CF9008951F93DB
:106A4000CF93C82F162F603418F06AE474E002C0A8
:106A500064E574E08C2F0E94F019812F99278A3009
:106A6000910589F18B3091057CF48630910511F107
:106A7000873091051CF40297D1F039C08830910518
:106A8000F9F00997D1F033C08E30910529F18F309C
:106A9000910534F48B309105C9F00D97D1F027C0E2
:106AA00081349105E1F082349105E1F020C06CE57C
:106AB00074E01AC060E774E017C06DE774E014C0BA
:106AC00060E974E011C063EA74E00EC06BEA74E040
:106AD0000BC06DEB74E008C066EC74E005C06DEDB2
:106AE00074E002C068EE74E08C2F0E94F01910343C
:106AF00020F06DE08C2F0E94C01981E090E0CF91D2
:106B00001F9108950F931F93D8018A30C0F4861700
:106B1000B0F49927FC0114E0EE0FFF1F1A95E1F77E
:106B2000E81BF90BE75CFB4F8685882341F0008169
:106B300011810417150718F02017310708F48D018B
:106B4000C8011F910F91089563EF74E00E94F0193E
:106B500081E090E008956AE275E00E94F01981E01A
:106B600090E0089567E475E00E94F01981E090E0FC
:106B700008951F93182F60E875E00E94F0196AE9E4
:106B800075E0812F0E94F01969EB75E0812F0E945A
:106B9000F01981E090E01F910895CF93C82F0E94D3
:106BA0006E0E992783309105A1F0843091052CF465
:106BB000009749F0029751F017C08430910561F0B9
:106BC000079794F40CC066ED75E00BC06EED75E0B0
:106BD00008C066EE75E005C06DEE75E002C069EFB5
:106BE00075E08C2F0E94F01981E090E0CF9108951C
:106BF000EF92FF920F931F93182F7B01042F80E0D9
:106C00000E942F0E402FB701812F0E94CD3599276A
:106C10001F910F91FF90EF900895EF92FF920F93C5
:106C20001F93182F7B01042F83E00E942F0E402F0B
:106C3000B701812F0E94CD3599271F910F91FF90A9
:106C4000EF9008956FEF75E00E94F01982E00E94C6
:106C50002F0E80E090E008950F931F93CF93C82FDD
:106C6000762F642F00E010E0A801872F0E94823564
:106C70008C01892B21F462E08C2F0E941F35C80102
:106C8000CF911F910F9108957F928F929F92AF9213
:106C9000BF92CF92DF92EF92FF920F931F93CF9309
:106CA000DF93882E942E2FEF37E260E00E942C367F
:106CB0005C01009719F481E090E062C10E94C02558
:106CC0006C01892B69F421E0291510F06AE012C0EB
:106CD000C5010E94E8256C01892B11F46BE00AC004
:106CE00031E0391508F0D6C00E94FD1A782E8823AD
:106CF00031F068E0882D0E941F35992741C1F601C7
:106D0000C481D58150EFE52E5FE7F52EEC22FD2200
:106D10008D2F992787FD90958827990F881F992790
:106D20008C0121E030E040E050E0692D82E00E94DB
:106D30008235892B21F020E030E8E22AF32ACE01C7
:106D4000817090708C0121E030E040E050E0692DCE
:106D500084E00E948235892B21F081E090E0E82ACE
:106D6000F92ACE0196958795817090708C0121E06B
:106D700030E040E050E0692D85E00E948235892BAB
:106D800021F0E2E0F0E0EE2AFF2ACE019695879509
:106D900096958795817090708C0121E030E040E0FD
:106DA00050E0692D86E00E948235892B21F024E095
:106DB00030E0E22AF32A83E0D695C7958A95E1F779
:106DC000C170D0708E0121E030E040E050E0692DCC
:106DD00087E00E948235892B21F088E090E0E82A44
:106DE000F92A472DB701C5010E949828F601608550
:106DF00086810E94992F99278C012FE730E040E08F
:106E000050E0692D81E00E948235C82F809168048E
:106E1000863411F411E015C0823511F4172D11C01C
:106E200000E010E0F601868187FF02C001E010E07B
:106E300021E030E040E050E0692D83E00E9482359F
:106E4000182FC13029F4C0E0C5010E942A1C06C0D9
:106E5000F60160858C2F0E94CB2FC82F1111C068BE
:106E60002C2F332720783070F6016681862F9927E2
:106E7000807890702817390729F0607840E0C501C4
:106E80000E94152840E06C2FC5010E941528C501FD
:106E90000E9402290E946E0E823011F461E405C046
:106EA0000E946E0E833021F062E4882D0E941F350F
:106EB000F6018481958183FF03C081E390E002C0E5
:106EC00080E390E09F938F93F6018481958182FF08
:106ED00003C081E390E002C080E390E09F938F9332
:106EE000F6018481958181FF03C081E390E002C0B7
:106EF00080E390E09F938F93F6018481958180FFDA
:106F000003C081E390E002C080E390E09F938F9301
:106F1000F601868187FF03C086E690E002C082E723
:106F200090E09F938F93F6018581282F332727FDCB
:106F30003095209530952227330F221F332781E388
:106F400090E0821B930B9F938F93608586810E94B4
:106F5000992F99279F938F93BF92AF9289E096E0E4
:106F60009F938F938F920E94461A81E090E02DB7F5
:106F70003EB72D5E3F4F0FB6F8943EBF0FBE2DBFFC
:106F8000DF91CF911F910F91FF90EF90DF90CF9005
:106F9000BF90AF909F908F907F900895CF93C82F10
:106FA0002FEF37E260E08C2F0E942C36009719F10A
:106FB0000E94C025FC01892B19F463E276E018C019
:106FC00080859927837090708230910561F08330BD
:106FD00091051CF4019721F00EC0039739F00BC006
:106FE0006AE276E005C067E376E002C064E476E03A
:106FF0008C2F0E94F01981E090E0CF9108957F924C
:107000008F929F92AF92BF92CF92DF92EF92FF92B8
:107010000F931F93CF93DF93A82EB42E2FEF37E259
:1070200060E00E942C364C01009719F481E090E05A
:1070300021C10E94C0256C01892B69F421E02B1528
:1070400010F06AE012C0C4010E94E8256C01892B8F
:1070500011F46BE00AC031E03B1508F08FC00E94CC
:10706000FD1A782E882331F068E08A2D0E941F35A2
:10707000992700C1F601E480F580E701C070C701DF
:10708000817090708C0121E030E040E050E06B2D89
:1070900081E00E948235892B09F0C160C701969575
:1070A0008795817090708C0121E030E040E050E0E5
:1070B0006B2D82E00E948235892B09F0C260C701E6
:1070C0009695879596958795817090708C0121E0B3
:1070D00030E040E050E06B2D83E00E948235892B48
:1070E00009F0C46063E0F694E7946A95E1F7F1E093
:1070F000EF22FF24870121E030E040E050E06B2DDB
:1071000084E00E948235892B09F0C860870121E064
:1071100030E040E050E06B2D85E00E948235892B05
:1071200009F0C061870121E030E040E050E06B2DC4
:1071300086E00E948235892B09F0C062870121E038
:1071400030E040E050E06B2D87E00E948235892BD3
:1071500009F0C064870121E030E040E050E06B2D91
:1071600088E00E948235892B09F0C068472DBE0156
:10717000C4010E949828C4010E9402290E946E0E38
:10718000882321F462E48A2D0E941F35F601848150
:10719000958187FF03C081E390E002C080E390E027
:1071A0009F938F93F6018481958186FF03C081E3CD
:1071B00090E002C080E390E09F938F93F60184817A
:1071C000958185FF03C081E390E002C080E390E0F9
:1071D0009F938F93F6018481958184FF03C081E39F
:1071E00090E002C080E390E09F938F93F60184814A
:1071F000958183FF03C081E390E002C080E390E0CB
:107200009F938F93F6018481958182FF03C081E370
:1072100090E002C080E390E09F938F93F601848119
:10722000958181FF03C081E390E002C080E390E09C
:107230009F938F93F6018481958180FF03C081E342
:1072400090E002C080E390E09F938F939F928F9293
:1072500088E496E09F938F93AF920E94461A81E054
:1072600090E02DB73EB72B5E3F4F0FB6F8943EBF70
:107270000FBE2DBFDF91CF911F910F91FF90EF9027
:10728000DF90CF90BF90AF909F908F907F900895A8
:107290007F928F929F92AF92BF92CF92DF92EF92A6
:1072A000FF920F931F93CF93DF93A82EB42E2FEF4F
:1072B00037E260E00E942C364C01009719F481E01F
:1072C00090E02EC10E94C0256C01892B69F421E059
:1072D0002B1510F06AE012C0C4010E94E8256C0171
:1072E000892B11F46BE00AC031E03B1508F09DC01A
:1072F0000E94FD1A782E882331F068E08A2D0E94C2
:107300001F3599270DC1F601C481D5817FEFE72E86
:1073100070ECF72EEC22FD228D2F99278170907052
:107320008C0121E030E040E050E06B2D81E00E94D4
:107330008235892B21F020E031E0E22AF32ACE01C8
:10734000892F99278695817090708C0121E030E01B
:1073500040E050E06B2D82E00E948235892B21F0C5
:1073600080E092E0E82AF92ACE01892F99278695B4
:107370008695817090708C0121E030E040E050E013
:107380006B2D83E00E948235892B21F0E0E0F4E050
:10739000EE2AFF2ACE01892F992786958695869514
:1073A000817090708C0121E030E040E050E06B2D66
:1073B00084E00E948235892B21F020E038E0E22A27
:1073C000F32ACE01892F992782958F708170907052
:1073D0008C0121E030E040E050E06B2D85E00E9420
:1073E0008235892B21F080E090E1E82AF92ACD2F1F
:1073F000DD27C295C695C770C170D0708E0121E09F
:1074000030E040E050E06B2D86E00E948235892B11
:1074100021F0E0E0F0E2EE2AFF2A472DB701C40197
:107420000E949828C4010E9402290E946E0E88239F
:1074300021F462E48A2D0E941F35F6018481958132
:10744000892F992782958695877080FF03C081E3F5
:1074500090E002C080E390E09F938F93F6018481D7
:107460009581892F992782958F7080FF03C081E3D2
:1074700090E002C080E390E09F938F93F6018481B7
:107480009581892F992786958695869580FF03C0DB
:1074900081E390E002C080E390E09F938F93F60138
:1074A00084819581892F99278695869580FF03C0D1
:1074B00081E390E002C080E390E09F938F93F60118
:1074C00084819581892F9927869580FF03C081E368
:1074D00090E002C080E390E09F938F93F601848157
:1074E0009581892F992780FF03C081E390E002C036
:1074F00080E390E09F938F939F928F9285E696E032
:107500009F938F93AF920E94461A81E090E02DB72F
:107510003EB72F5E3F4F0FB6F8943EBF0FBE2DBF54
:10752000DF91CF911F910F91FF90EF90DF90CF905F
:10753000BF90AF909F908F907F900895AF92BF9231
:10754000CF92DF92EF92FF920F931F93CF93DF932F
:10755000A82EC42F0E946E0E882311F466E05DC031
:1075600028EF37E04C2F60E08A2D0E942C366C010A
:10757000892B19F021E02A1518F481E090E083C0EE
:1075800088E4A89EC001112487559C4FC23008F49E
:107590004EC0A5E4EA2EF12CE80EF91EF701808119
:1075A0009181FFEF8F3F9F0749F040E0642F0E94D9
:1075B0000F648FEF9FEFF7018083918380914A04DE
:1075C000873411F4BB2410C0823519F4F1E0BF2ECA
:1075D0000BC002E010E021E030E040E050E06C2F12
:1075E00081E00E948235B82E00E010E021E030E01A
:1075F000A8016C2F82E00E948235EC0186010150C7
:107600001040000F111F0B0D111D40E0682FC80125
:107610000E940F64882331F469E08A2D0E941F358F
:10762000992731C0CC2319F0F70100831183C601DB
:1076300001970E94FF62C0E0D0E0082F112707FDEC
:107640001095C8010E94BF6C892B11F0C1E0D0E0F9
:10765000DF93CF93C8010E94D26C9F938F93DF92E8
:10766000CF928DE796E09F938F93AF920E94461A38
:1076700081E090E02DB73EB7275F3F4F0FB6F894FB
:107680003EBF0FBE2DBFDF91CF911F910F91FF9095
:10769000EF90DF90CF90BF90AF9008951F93182F79
:1076A00068E876E00E94F01965E976E0812F0E9493
:1076B000F0190E94BC52DC01CB01BF93AF939F93A2
:1076C0008F938BE996E09F938F931F930E94461AA6
:1076D0008DB79EB707960FB6F8949EBF0FBE8DBFAD
:1076E00081E090E01F910895EF92FF920F931F9316
:1076F000CF93DF93E82EF42E0E947F52EC01FF20FF
:10770000E1F08B8599278C0124E130E040E050E0E6
:107710006F2D80E00E9482358B878C859927880F9A
:10772000991F8C012EEF31E042E050E06F2D81E097
:107730000E948235969587958C878C859927880F2E
:10774000991F9F938F938B8599279F938F9388EA97
:1077500096E09F938F93EF920E94461A8DB79EB743
:1077600007960FB6F8949EBF0FBE8DBF81E090E0E4
:10777000DF91CF911F910F91FF90EF9008950F939C
:107780001F93CF93C82F642F442379F08091620A0E
:107790009927817090708C0121E030E040E050E04A
:1077A00080E00E9482350E942A5C8091620A9927BB
:1077B000817090709F938F9381EB96E09F938F934E
:1077C000CF930E94461A0F900F900F900F900F903A
:1077D00081E090E0CF911F910F910895DF92EF9299
:1077E000FF920F931F93CF93E82E842F00E010E0B9
:1077F00020E230E041E050E0682F80E00E948235D6
:10780000C82F882309F447C099279F938F9387EB4C
:1078100096E09F938F93EF920E94461ADC2EDA94A3
:1078200060E08D2D0E941A5C082F112781E0F82E50
:107830000F900F900F900F900F90C7E08F2D99270A
:1078400080239123892B11F061E301C060E38E2D29
:107850000E94C019C150FF0CC7FFF0CF60E28E2D0F
:107860000E94C01961E08D2D0E941A5C082F11271B
:10787000C1E0FC2EC7E08F2D992780239123892B0F
:1078800011F061E301C060E38E2D0E94C019C15068
:10789000FF0CC7FFF0CF81E090E0CF911F910F91D7
:1078A000FF90EF90DF900895FF920F931F93F82EB3
:1078B000642F8091610A9927880F991F8C0120E419
:1078C00030E040E050E080E00E9482358F5F869596
:1078D0008093610A9927880F991F9F938F938AED50
:1078E00096E09F938F93FF920E94461A0F900F90FD
:1078F0000F900F900F9081E090E01F910F91FF90FB
:107900000895CF93C82F4423C9F4C13031F460EEF9
:1079100076E08C2F0E94F01913C00E94F8109F93FC
:107920008F9386EE96E09F938F93CF930E94461A93
:107930000F900F900F900F900F9002C0C13019F46C
:1079400081E090E00DC069EE76E08C2F0E94F01986
:107950008091390490913A040E94B81080E090E040
:10796000CF9108950F931F93CF93C82F842F0FEFBC
:107970001FEF27EE33E040E050E0682F80E00E94E8
:1079800082350E94023097FF06C062E08C2F0E9471
:107990001F35992711C090709F938F938CEE96E0BE
:1079A0009F938F93CF930E94461A81E090E00F90AF
:1079B0000F900F900F900F90CF911F910F910895FE
:1079C000EF92FF920F931F93982F642F4423C9F0D7
:1079D00088E4989F7001112489EA93E0E80EF91E6B
:1079E00000E010E021E030E0A80180E00E94823554
:1079F000F701E95BFF4F892B19F081E0808301C01B
:107A0000108281E090E01F910F91FF90EF90089518
:107A1000DF92EF92FF920F931F93CF93DF93082F84
:107A2000EB01D42E823008F00EC188E4089F90014B
:107A3000112427553C4F4881142F1F71642F77273D
:107A4000CB01807E90708034910509F4A3C081340D
:107A5000910534F40097A9F0809709F463C0F3C04E
:107A60008038910509F4BFC0813891052CF4803627
:107A7000910509F4B0C0E7C0803C910509F4CCC081
:107A8000E2C021E02D1508F0E0C08981C82FDD2774
:107A9000CE010E94E825FC01892B09F4D4C0E480C2
:107AA000F58014FF05C080E090E8E82AF92A04C0B8
:107AB0008FEF9FE7E822F9221F70068100781F30C0
:107AC00019F460E8602729C080851F7011F01F300D
:107AD00019F460E070E020C00E947D29282F332730
:107AE0002C31310571F02D31310524F42B31310564
:107AF00029F010C02E37310531F00CC0110F115094
:107B000009C0110F07C089E0189F802D1124682F2C
:107B1000772702C0612F7727602B40E0CE010E94BB
:107B2000152850C0437F488375E4E72EF12CE20E00
:107B3000F31EF70180819181FFEF8F3F9F0749F08E
:107B400040E0642F0E940F648FEF9FEFF701808366
:107B500091832881203209F476C0233209F473C05E
:107B6000F1E0FD15D0F46981213231F4C62FDD2713
:107B70002197CC0FDD1F05C0C62FDD27CC0FDD1FE1
:107B8000219740E061E0CE010E940F64F701C083BD
:107B9000D18359C0F1E0FD1518F080E090E055C0A8
:107BA0008981C82FDD27CE010E94182740EFE42EDF
:107BB0004FEFF42EE822F922812F99278F709070D1
:107BC000E82AF92A40E0B701CE010E949828CE01A8
:107BD0000E94022938C060FF02C080E001C083E03B
:107BE0000E942F0E30C0112311F4812F18C0C0E065
:107BF000C11748F560E08C2F0E94095C682F802F28
:107C00000E94C01961E08C2F0E94095C682F802FB0
:107C10000E94C019CF5FECCF112321F481E00E94B4
:107C20002A5C11C0115060E0812F0E94095C682F0E
:107C3000802F0E94C01961E0812F0E94095C682F8B
:107C4000802F0E94C01981E090E0DF91CF911F91B9
:107C50000F91FF90EF90DF9008959B012F5F3F4FB2
:107C600042E0B9010E94083D8FEF90E008959B012A
:107C70002F5F3F4F41E0B9010E94083D8FEF90E038
:107C800008958230C0F4282F332788E490E0289F9D
:107C9000F001299FF00D389FF00D1124E755FC4F9E
:107CA000EC5BFF4F1082339610828FEF9FEF929321
:107CB00082930E94F966089508952F923F924F9201
:107CC0005F926F927F928F929F92AF92BF92CF926C
:107CD000DF92EF92FF920F931F93CF93DF93CDB775
:107CE000DEB725970FB6F894DEBF0FBECDBF8B83EE
:107CF000B62E823008F0DFC188E49B81989F800116
:107D0000112407551C4FB4E4CB2ED12CC00ED11E2C
:107D1000D6018C918823B1F0F80180819181A281F4
:107D2000B38188539F4FAF4FBF4FBC01CD010E941D
:107D30008A14882339F0C8010E944F2F882311F438
:107D4000D6018C938091CA069091CB06A091CC0667
:107D5000B091CD06F80180839183A283B383D601CD
:107D60008C91803408F01C92C8010E946D2F8823EA
:107D700091F0B8E0BB1641F4F6018081882309F444
:107D80009AC18150808397C1BB2009F494C1FDE062
:107D9000BF1609F4BB24D601FC90F801EF0DF11DCC
:107DA000B482F394FC92C8010E944F2FA82E88231E
:107DB00009F476C1C8010E946D2F882309F43CC1E3
:107DC000BB2009F078C1F601B08286E491E08C8393
:107DD0009D83A4E04A2E512C400E511E095B1F4F7B
:107DE000D8018C9107541040882329F4F5E04F2ED8
:107DF000512C400E511EF2018081882309F416C1D6
:107E000043E050E06FEE76E0C2010E94BD67892B2F
:107E100019F4C201039601C0C2010E941B69498284
:107E20005A82EE2486E9E9E3F4E011928A95E9F7B3
:107E300005C00894211C311C29823A8229803A808D
:107E4000D1019C91992391F09C3281F0943271F090
:107E5000953261F0892F80538A3040F0892F99271D
:107E600087FD90950E94C96C892B19F3F1018081DF
:107E7000882309F4A8C004C00F5F1F4F09831A8329
:107E800009811A81D801FC908F2D992787FD909543
:107E90000E94C96C892B81F7FF2009F496C0BCE2CF
:107EA000FB1609F482C08FE0E89E60011124E9E32B
:107EB000F4E0CE0EDF1E4801E2E0AE2EB12CAC0C99
:107EC000BD1C6624772409C00894811C911CD5012F
:107ED000FD925D010894611C711CBBE06B1671047E
:107EE0007CF4F401F080FF2059F0FCE2FF1641F031
:107EF0008F2D992787FD90950E94C96C892B21F3BE
:107F0000D5011C92F8018081843239F4C8010196B0
:107F100089839A8340E150E008C0853251F4C8015A
:107F2000019689839A8342E050E0BE016F5F7F4FE4
:107F300006C04AE050E0BE016F5F7F4FC8010E945B
:107F4000CB67DC01CB01F6018083918381E0F601F0
:107F5000868704C00F5F1F4F09831A8309811A8126
:107F6000D801FC90FF2081F08F2D992787FD9095F7
:107F70000E94C96C892B41F4BCE2FB1659F704C07E
:107F80000F5F1F4F09831A8309811A81F801F0805E
:107F9000FF2041F08F2D992787FD90950E94C96C95
:107FA000892B71F7FCE2FF1621F40F5F1F4F098345
:107FB0001A83E394E981FA818081882321F089E0A2
:107FC0008E1508F05DCFD1011C924E2D5527142F30
:107FD0008091460190914701892BD1F0EC81FD8180
:107FE00060817181C2010E949E67892B41F4EC81FE
:107FF000FD81228133812115310581F417C08C81E7
:108000009D8104968C839D83DC018D919C91E4CFAE
:1080100063EF76E08B810E94F01908C0412FB20116
:108020008B81F9010995882309F445C063E077E065
:108030008B810E94F0193FC0EEEAF1E0A8014C5F8D
:108040005F4F2F2D095B1F4FD8018C9107541040B3
:10805000882321F4A8014B5F5F4F21508091AE012E
:10806000882349F19081DA018C919817A1F48181DC
:10807000281708F10280F381E02D309749F0BA010A
:108080008B810995682F8F3F19F08B810E94C01951
:10809000F601108210C034968081882319F70BC036
:1080A0000C5F1F4F4F2DB8018B810E94083D882324
:1080B00011F0D601AC9225960FB6F894DEBF0FBE34
:1080C000CDBFDF91CF911F910F91FF90EF90DF9087
:1080D000CF90BF90AF909F908F907F906F905F9068
:1080E0004F903F902F900895FB0121E057FF04C06F
:1080F00020E0509541955F4F8330910549F18430E0
:10810000910534F48130910591F0029729F12AC04C
:108110008430910519F0059761F024C081818F5F4B
:108120008183992784179507ECF0222359F0118257
:1081300019C081818150818399278417950794F014
:10814000222321F0842F815081830CC021830AC017
:1081500012821382168A06C090E08281882309F475
:1081600091E0928380E090E008950F931F93CF9366
:10817000DF938C010E948929EC01009731F461E3BF
:1081800070E182E00E94F0190FC09F938F9387E304
:1081900090E19F938F9382E08F930E94461A0F90F5
:1081A0000F900F900F900F900115110521F0B8015D
:1081B00082E00E94F019CE01DF91CF911F910F91C3
:1081C00008950F931F93CF93DF93EC018B010097DA
:1081D00031F097FD35C00297029790F52BC060E013
:1081E00081E00E946818F8018281882359F46BE3CA
:1081F00070E182E00E94F01964E470E182E00E9484
:10820000F01918C00E94BC52DC01CB01BF93AF93A0
:108210009F938F938AE490E19F938F9382E08F9353
:108220000E94461A8DB79EB707960FB6F8949EBF68
:108230000FBE8DBF40E050E0B801CE010E947440F7
:1082400080E090E0DF91CF911F910F9108958230EF
:10825000910541F08330910541F440E050E00E94E7
:10826000744003C08FEF9FEF089580E090E0089581
:108270000895AF92BF92CF92DF92EF92FF920F9349
:108280001F93CF93DF93EC017B010E9486298C0121
:10829000C230D10509F453C0C330D1052CF4209766
:1082A000D1F0219731F092C0C630D1050CF08EC0CC
:1082B0002AC0FC016785262F2695269523706370BA
:1082C00009F461E083E0689FC0011124280F235066
:1082D000F70121837BC060E081E00E94681886E599
:1082E00090E10E94B540892B09F470C0F70191819B
:1082F0008AE0989FC0011124895A984FBC0182E0FE
:108300000E94F01963C049E050E0B701CE010E941D
:108310007440F801808191818F3F910509F008F444
:1083200055C0F7018181882311F486E08183F7012C
:108330008181863008F04AC088E0818347C0FC0113
:10834000A280B380A114B10409F040C0F70182817A
:108350008823A1F1F801C081D1812097B9F1F701FB
:108360003181832F63E00E948C6C282F2F5F832F35
:108370000E948C6C892F9927880F991F880F991F4D
:10838000282BF801C288D388622FCE010E942227B1
:10839000CE010E940427B5010E948C2AC114D10489
:1083A00069F0C80144969C01F8014785608171819C
:1083B000C6010E94F95DF801828B938B90E0F70172
:1083C0008281882309F491E0F701928380E090E0B4
:1083D000DF91CF911F910F91FF90EF90DF90CF90A1
:1083E000BF90AF900895482F30E0832F992787FDE5
:1083F0009095FC01EA5DF84F2491241729F03F5F26
:10840000222399F78FEF9FEF08950895EF92FF923F
:108410000F931F93CF93DF93EB018230910509F403
:1084200086C08330910534F4009709F43EC001976B
:1084300069F0BAC08430910509F443C084309105D5
:108440000CF470C0059709F456C0AEC00E9486298E
:108450008C01FC0180819181892B09F4A5C044E144
:10846000E42EF12CE00EF11E8E01065F1F4F659683
:108470000C171D07B8F4F7018081882339F00E949A
:10848000F34187FD03C0F701808101C080E2F8015C
:1084900081938F01F7018081882351F30894E11CB7
:1084A000F11CE6CFF80110827FC00E94B54060E069
:1084B00081E00E9468182A96BE0182E00E94061A96
:1084C00073C08981FB01E80FF11DEF012A968285B7
:1084D0000E94F3418F5FE82FFF27E7FDF095EA5DEB
:1084E000F84F8491882319F4E6E2F7E08491992704
:1084F00087FD909515C08981FB01E80FF11DEF0103
:108500002A9682850E94F341181614F08FE201C06A
:108510008150E82FFF27E7FDF095EA5DF84F849141
:10852000888342C049E050E00E9474403DC00E94F0
:1085300086298C01FC0182819381892BA9F59A817E
:10854000992349F489E08B8381E0888F99839F8BFD
:108550008A838E8B29C089818F5F89838F8B8B3033
:1085600018F11B821A821E8A8CE098012C5E3F4F04
:10857000D901FE013A9601900D928A95E1F7F80132
:1085800082899389009731F04785608171810E94CB
:10859000F95D07C0A901F8016785808191810E947A
:1085A000B15EF801828B938B80E090E0DF91CF91F8
:1085B0001F910F91FF90EF900895AF92BF92CF92CD
:1085C000DF92EF92FF920F931F93CF93DF93CDB77C
:1085D000DEB721970FB6F894DEBF0FBECDBF9C016A
:1085E0008B018230910509F455C0833091052CF43C
:1085F0000097C1F0019759F0A5C084309105D9F1D9
:10860000843091050CF441C00597C9F19BC04BE043
:1086100050E060E270E0C8010A960E946667F801C7
:10862000158A90C0FB018281882309F48BC0818167
:10863000882309F487C0065F1F4FA801B901992755
:108640000E94B95E9F938F9389E590E19F938F93EA
:1086500062E0F62EFF920E94461A60E081E00E94DE
:108660006818B8018F2D0E94061A0F900F900F9076
:108670000F900F9067C0FB018181992721C0FB01FA
:10868000818199270E94715F1DC049E050E00E94DE
:10869000744058C090E0FB018281882309F491E086
:1086A000F80192830E9486297C01F8018281882347
:1086B00061F0F70182899389009711F0828902C0E5
:1086C0000E943C5FF80181833DC05AE0A52EB12C89
:1086D000A00EB11EF8018181A501BE016F5F7F4F21
:1086E00099270E94B95E6C01F701128213821082F1
:1086F0001182BC018FEF0E94F653F70180819181B6
:10870000892B69F06981C6010E942227C6010E9457
:10871000042760E070E00E948C2A0E949829F701EB
:1087200080819181892B59F0B501C70144960E943F
:10873000A867F80181819927F701828B938B8FEFCE
:108740009FEF02C080E090E021960FB6F894DEBF64
:108750000FBECDBFDF91CF911F910F91FF90EF9092
:10876000DF90CF90BF90AF9008950F931F93CF935A
:10877000DF93EC010E9486298C01209719F0229743
:10878000C9F03DC0CE010E94B540892BC1F160E027
:1087900081E00E946818F80182899389892B11F081
:1087A00081E001C082E00E946D51BC0182E00E9424
:1087B000F01925C0FC01C281D381209701F5808189
:1087C0009181892BE1F082899389892BC1F060E046
:1087D00081E00E94681883E00E946D51BC0182E034
:1087E0000E94F01984EF91E00E94C116F80182897D
:1087F00093890E94F65DF801C28BD38B148A80E0C6
:1088000090E0DF91CF911F910F9108951F93CF9327
:10881000DF93EB018230910509F440C0833091056C
:108820002CF4009789F0019731F04CC08630910507
:108830000CF048C02EC00E947F52FC01848163E08E
:108840000E948C6C89833EC060E081E00E946818C1
:10885000898113E0819F802D11240E94BB1982E041
:1088600090E00E94C11681B7612F0E948C6C8983B1
:1088700099279F938F938DE590E19F938F9382E04B
:108880008F930E94461A0F900F900F900F900F90A9
:1088900019C04FEE5FEF0E94744014C08A81882394
:1088A00059F00E947F52398123E0329F90011124B8
:1088B000FC0124830E94065290E08A81882309F4F7
:1088C00091E09A8380E090E0DF91CF911F9108952D
:1088D0001F93CF93DF93EC018A81882309F45CC056
:1088E00060E081E00E9468188C819D819F938F9346
:1088F00081E690E19F938F9312E01F930E94461AA6
:108900008B810F900F900F900F900F90843059F43F
:1089100087E690E19F938F931F930E94461A0F90D2
:108920000F900F9010C0888599279F938F938BE6A7
:1089300090E19F938F931F930E94461A0F900F9080
:108940000F900F900F90898D9A8D97FD03C06FE661
:1089500070E10AC08E5F9F4F19F467E770E104C0B1
:1089600084E00E946D51BC0182E00E94F01981E018
:10897000888F8E8B8B8199278130910564F08330AD
:10898000910524F00497029730F402C083E001C0FF
:1089900088E08F8B01C01E8ADF91CF911F910895CF
:1089A0000F931F93CF93DF938C01FC018281882367
:1089B00011F581E08383643019F488E090E003C00E
:1089C00080E094E0F80186839783F8012481358163
:1089D000868197818217930724F481E090E0848355
:1089E000958381E0F8018283683009F410C180E04A
:1089F0000E942F0E0CC1F801848195819093D904B7
:108A00008093D804C62FDD27C430D10561F1C5306D
:108A1000D10594F4C130D10509F4C2C0C230D105EA
:108A20001CF4209701F1F3C0C230D10509F4BAC09B
:108A3000239709F4E9C0EBC0C730D10509F4B0C0F1
:108A4000C830D10544F4C530D10509F4A9C0C630F9
:108A5000D10549F0DCC0C830D10509F47EC02997A2
:108A600009F49EC0D4C0F801838181508230E0F5C2
:108A70008EEF9FEF818F928FC8010E9468446AE059
:108A800081E00E94681889E00E946D51BC0182E07B
:108A90000E94F019C430D10581F0C530D1051CF415
:108AA000CD2B21F019C0269771F016C0F8018481F2
:108AB000958101970E94CA5B0CC0F80184818150A6
:108AC0000E94EA5B06C0F8018481958101970E94AB
:108AD000FF5BF801818F928FF801818D928D97FD58
:108AE0005DC0818D80875AC06AE081E00E9468186D
:108AF0008AE00E946D51BC0182E00E94F019C430EE
:108B0000D10589F0C530D1051CF4CD2B21F046C02C
:108B10002697C1F043C0F801848195816085019753
:108B20000E94C05B16C0F8018481958109971CF0F2
:108B30008FEF9FEF0FC0F8018481608581500E9404
:108B4000DF5B07C0F80184819581608501970E94F1
:108B5000F55BF801818F928F21C00E948629FC016C
:108B60002081318121153105C9F0878599278370CE
:108B70009070039799F4F80164817581611571050E
:108B800069F083818150823048F0615070404085A7
:108B9000C9010E946A29F801138239C081E035C0F9
:108BA00084E033C0F80183818150823010F481E089
:108BB0002DC06AE081E00E946818F8018381863048
:108BC00079F489E00E946D51BC0182E00E94F019A5
:108BD000F80184819581618501970E94B65B0FC081
:108BE0008AE00E946D51BC0182E00E94F019F801F8
:108BF00084819581418D618501970E94AC5BF8016C
:108C0000818F928F86E001C087E0F8018383DF9136
:108C1000CF911F910F9108959C01FB018130910527
:108C200061F0823091051CF4892BD1F024C083308F
:108C30009105E9F00597C1F01EC08EEF9FEF818F7F
:108C4000928F4091D8045091D904CA010197805065
:108C5000944018F4448355830EC0248335830BC09D
:108C6000CB010E94684407C081E0838304C040E0D8
:108C700050E00E94744080E090E008950F931F93AD
:108C8000CF93DF938C01EB010E948629FC01808148
:108C90009181892B31F08785992783709070039794
:108CA00061F060E081E00E94681885E00E946D51EB
:108CB000BC0182E00E94F0191BC00230110541F096
:108CC0000430110589F469E0CE010E94D04410C03F
:108CD00068E0CE010E94D0448B81882349F40E9431
:108CE00077188FEF9FEF06C0BE01C8010E940C46A7
:108CF00080E090E0DF91CF911F910F910895CF9385
:108D0000DF93EB018230910509F481C08330910536
:108D100034F40097A1F08130910569F07CC0843073
:108D2000910509F462C0843091050CF46BC005977D
:108D300009F460C070C00E940C4619866CC08A811C
:108D4000882309F468C060E081E00E9468188B8184
:108D5000882331F46FE770E182E00E94F01918C0B7
:108D6000898599279F938F938C819D819F938F9362
:108D70008FE890E19F938F9382E08F930E94461A31
:108D80008DB79EB707960FB6F8949EBF0FBE8DBFE6
:108D9000898D9A8D97FD0BC0823091051CF002974A
:108DA00021F005C0898D805D03C08FE301C085E49B
:108DB0000E941A1881E0888F8E8B8B8199278630CC
:108DC000910561F08730910524F40197029758F4DA
:108DD00003C0079729F007C086E003C08CE001C0FC
:108DE0008EE08F8B18C01E8A16C08B81863039F4B6
:108DF00063E00EC08B81863011F481E001C086E013
:108E00008B8309C040E050E00E94744004C062E0DF
:108E1000CE010E94D04480E090E0DF91CF91089590
:108E20009B018230910529F08430910539F461E08D
:108E300001C060E0C9010E94D04402C00E940C46FB
:108E400080E090E008959B018230910529F0843004
:108E5000910539F465E001C064E0C9010E94D04485
:108E600002C00E940C4680E090E008959B01823091
:108E7000910529F08430910539F467E001C066E07E
:108E8000C9010E94D04402C00E940C4680E090E0DC
:108E900008951F93182F60E081E00E946818812FC9
:108EA00099278130910571F0823091051CF4892B4E
:108EB00039F013C08230910539F0039739F00DC0B5
:108EC0008BE005C08CE003C08DE001C08EE00E9405
:108ED0006D51BC0182E00E94F0191F910895CF935B
:108EE000C82F1816B4F480E00E9449476C2F80E028
:108EF00090E00E94C05B892B39F440E065E08CE192
:108F000090E00E94AC5B07C08C2F0E94D45B892B41
:108F100011F082E001C083E00E94494784EF91E0B4
:108F20000E94C116CF910895CF93DF93EB01823059
:108F30009105E1F1833091051CF4892B29F04EC095
:108F40008330910571F14AC08A81882309F446C0B3
:108F500060E081E00E9468188C819D8197FF0CC0C1
:108F60008EE990E19F938F9382E08F930E94461A3F
:108F70000F900F900F900FC09F938F9383EA90E113
:108F80009F938F9382E08F930E94461A0F900F90C9
:108F90000F900F900F9083E08F8B81E0888F8E8BE6
:108FA0001DC040E050E00E94744018C08A818823B0
:108FB00021F08C810E946F4705C081E00E944947E3
:108FC00081E08A8380E090E00E94CA5B8C839D836D
:108FD00081E08B838FE790E08E839F8380E090E039
:108FE000DF91CF9108950F931F93CF93DF938B0160
:108FF0008130910571F0823091051CF4892B79F054
:10900000B4C08230910509F43FC083309105B9F1B5
:10901000ACC08FEF9FEFFB0184839583A6C0FB015B
:109020008281882309F4A1C060E081E00E94681871
:10903000F8018481958197FF0CC087EA90E19F93A6
:109040008F9382E08F930E94461A0F900F900F909B
:109050000FC09F938F938EEA90E19F938F9382E04E
:109060008F930E94461A0F900F900F900F900F90C1
:1090700085E0F801878B81E0808F868B76C040E0A9
:1090800050E00E94744071C0FB018281882389F105
:10909000C481D581C038D10520F48C2F0E946F4740
:1090A0002EC0F8E2C030DF07A0F480E00E944947FC
:1090B0008D2F9927806C682F80E190E00E94C05B23
:1090C000009729F46C2F81E190E00E94C05B892B0E
:1090D00011F082E007C041E065E08CE190E00E9481
:1090E000AC5B83E00E94494784EF91E00E94C11687
:1090F00006C081E00E94494781E0F8018283F801BF
:109100008481958101978F37910540F480E090E04C
:109110000E94CA5BF8018483958315C080E190E0CA
:109120000E94CA5B982F8827F8018483958381E188
:1091300090E00E94CA5BF80124813581282B392BED
:109140003F7324833583F801848195818050984250
:109150002CF08FEF9FEFF8018483958381E0F80175
:1091600083838FEF97E28683978380E090E0DF919F
:10917000CF911F910F9108951F93CF93DF93EB0130
:10918000122F8230910519F1833091052CF400974C
:1091900061F0019729F02EC0863091055CF512C070
:1091A000842F0E94A052898325C060E081E00E9444
:1091B00068188981810F0E94C551BC0182E00E941C
:1091C000F01918C042E050E00E94744013C08A8138
:1091D000882351F08981882321F0842F0E94AA528C
:1091E00003C0842F0E94B25290E08A81882309F440
:1091F00091E09A8380E090E0DF91CF911F910895F4
:1092000022E048E00E94BC48089520E041E00E942E
:10921000BC4808950F931F93CF93DF938C01EB010C
:1092200026E044E00E94BC480230110529F48A81FE
:10923000882311F40E94EE1E80E090E0DF91CF9130
:109240001F910F9108951F93CF93DF93EB0182300D
:10925000910541F1833091052CF4009789F0019735
:1092600029F03CC086309105CCF517C010E080E0B5
:1092700090E00E943C65039709F411E019832EC029
:1092800060E081E00E94681889818E5F0E94C5516C
:10929000BC0182E00E94F01921C042E050E00E942F
:1092A00074401CC08A81882399F060E081E00E94AC
:1092B000681862EB70E182E00E94F01989818823CE
:1092C00019F083E090E002C081E090E00E946C65BC
:1092D00090E08A81882309F491E09A8380E090E00D
:1092E000DF91CF911F9108950F931F93CF93DF9339
:1092F0009C01EB018230910509F46BC0833091052C
:109300002CF4009739F1019731F097C08630910520
:109310000CF093C059C08C819D8101978C5F934064
:1093200010F02C833D838CEF93E08E839F8311E0BC
:109330001B831E8B83E08F8B188F00E08C819D81B7
:10934000880F991F02970E943C65039709F4012F2B
:10935000098373C060E081E00E9468188B812C81D2
:109360003D81813009F52D5F3F4F3F932F938C81D5
:109370009D819F938F938CEC92E09F938F9312E04B
:109380001F930E941A1A89818C5F0E94C551BC01EB
:10939000812F0E94F0198DB79EB707960FB6F894EB
:1093A0009EBF0FBE8DBF49C03F932F9386ED92E0C5
:1093B0009F938F9382E08F930E941A1A0F900F90C1
:1093C0000F900F900F9039C042E050E00E9474401F
:1093D00034C02A812223A1F089812C813D818823F8
:1093E00029F0220F331F63E070E004C0220F331F07
:1093F00061E070E0C90102970E9484651A821DC075
:109400008B81813019F48A832E8B17C08C819D81CA
:1094100001978C7F01968C839D83122F880F991F53
:1094200002970E943C65039709F411E0198391E0CB
:109430009B839E8B83E08F8B988F80E090E0DF9101
:10944000CF911F910F910895FF920F931F93CF9388
:10945000DF93EC018B01F42E0E947F52FC01C2309D
:10946000D10509F471C0C330D1052CF42097C9F09F
:10947000219771F07DC0C430D10509F44DC0C430CE
:10948000D1050CF44DC0C530D10509F449C070C0F8
:10949000FF2019F08485E80155C08385F801818398
:1094A00067C060E081E00E946818E8019981FF20B0
:1094B000F9F0892F6AE00E948C6C892F99279F937D
:1094C0008F9389810E948C6C99279F938F9381EC55
:1094D00090E19F938F9382E08F930E94461AEDB79D
:1094E000FEB737960FB6F894FEBF0FBEEDBF40C073
:1094F00082E3989FC00111249F938F9389EC90E1A0
:109500009F938F9382E08F930E94461A0F900F9043
:109510000F900F900F902CC0F80181818F3F41F187
:10952000FF2019F040E05FEF02C04BEE5FEFB801A3
:10953000CE010E947440FF20D9F0E8018981882380
:10954000B9F481E0898314C0E8018A81882341F05D
:109550009981FF2011F0948701C093870E940652E1
:1095600090E0F8018281882309F491E0E8019A8370
:1095700080E090E0DF91CF911F910F91FF900895CF
:1095800040E00E94244A089541E00E94244A089540
:10959000CF93DF93EB018230910559F18330910530
:1095A0002CF4009759F0019729F02FC086309105CF
:1095B00064F51AC00E948752898327C060E081E069
:1095C0000E94681889819927880F991F880F991F11
:1095D0008A5F984FBC0182E00E94F0196FEC70E145
:1095E00082E00E94F01911C048E050E00E947440EF
:1095F0000CC08A81882319F089810E948B5290E0E7
:109600008A81882309F491E09A8380E090E0DF91D9
:10961000CF910895CF93DF93EB0182309105C1F193
:109620008330910534F4009749F08130910551F170
:1096300057C0863091050CF053C024C08A8188231E
:1096400009F44EC061E080E00E9468188981885F5B
:109650000E94C551BC0182E00E94F01960E081E0E7
:109660000E9468186981623020F082E10E946D5189
:1096700004C0862F845F0E94C551BC0182E00E9415
:10968000F0192EC042E050E0BE010E94744028C094
:109690008A81882319F18981823018F48E5F898349
:1096A0001FC060E081E00E9468188981833051F416
:1096B0008FE00E946D51BC0182E00E94F0190E946F
:1096C000B46009C080E10E946D51BC0182E00E943B
:1096D000F0190E947C618FEF9FEF04C081E08A83C4
:1096E00080E090E0DF91CF910895CF938091CF04F7
:1096F000803178F01092CF041092D00461E0862F70
:109700000E946818CEE085EA0E941A18C150C7FF6F
:10971000FACF6091CF0481E00E9468188091D00454
:1097200099278130910559F0823091051CF4892BDD
:1097300021F014C0029739F011C085E001C084E027
:109740000E941A180BC080E20E941A1885E00E943D
:109750001A188091CF048F5F8093CF048091D0043A
:109760008F5F8093D004833010F01092D004CF919B
:109770000895CF93DF93EB018230910559F1833047
:1097800091051CF4892B31F053C0863091050CF003
:109790004FC01BC08A81882309F44AC061E080E081
:1097A0000E94681889E10E946D51BC0182E00E940C
:1097B000F01960E081E00E94681881E10E946D511B
:1097C000BC0182E00E94F01933C040E050E00E94EA
:1097D00074402EC08A81882329F10E94AC1E64E95E
:1097E00071E084E00E9497196CE871E085E00E94C6
:1097F000971968EC70E085E79BE40E94A11860E08F
:10980000862F0E94681883E00E946D51BC0182E09F
:109810000E94F0190E9490250E949A5F0E9428528F
:109820000E94865490E08A81882309F491E09A830B
:1098300080E090E0DF91CF910895CF92DF92EF9298
:10984000FF920F931F93CF93DF93029709F0CEC03F
:1098500060E0862F0E94681880E20E941A1860E07B
:1098600081E00E94681880E00E942F0E67ED70E191
:1098700082E00E94F01921E04EE468E086E00E9458
:10988000A00F6D9880E00E94A91180E00E94431310
:10989000CC24DD248EEF0E94B21380E00E94721A65
:1098A0008F5F9F4FD1F781E00E94721A8F5F9F4FA9
:1098B000D1F7A8950E94FF178331910509F488C05C
:1098C0008B30910509F484C00A9701F581C0CF3F20
:1098D000D10551F0209741F06C2F80E00E94C01913
:1098E0006C2F81E00E94C019CF33D10519F0CB3223
:1098F000D10519F4B4E8CB2ED12CC332D10511F027
:10990000AA9721F4A6E0CA2EA1E0DA2E0E94DF1366
:10991000EC018F5F9F4FD9F6C114D10409F4BACF7F
:10992000E090CA06F090CB060091CC061091CD06CF
:1099300088EC90E0A0E0B0E0E80EF91E0A1F1B1FC3
:109940003BC0A8950E94721AEC019FEFCF3FD90748
:1099500021F481E00E94721AEC01AFEFCF3FDA07E9
:1099600021F18C2F0E94B2130894C108D108E09015
:10997000CA06F090CB060091CC061091CD0688EC7B
:1099800090E0A0E0B0E0E80EF91E0A1F1B1F0DC01A
:10999000CF3FD10551F0209741F06C2F80E00E941D
:1099A000C0196C2F81E00E94C0190E94DF13EC01E6
:1099B0009FEFCF3FD90761F7C114D10409F468CFF5
:1099C000C801B7010E948A14882309F4BACF60CF76
:1099D00081E00E94A91181E00E9443136D9A0E94C8
:1099E000875221E04EE468E00E94A00F80E090E002
:1099F000DF91CF911F910F91FF90EF90DF90CF906B
:109A00000895CF93DF93EB018230910509F440C0B4
:109A1000833091052CF4009771F0019731F048C024
:109A2000863091050CF044C02EC00E947F52FC018C
:109A3000868189833DC060E081E00E946818698169
:109A4000662369F484E10E946D519F938F9382E0B5
:109A50008F930E94461A0F900F900F9029C085E0B7
:109A6000689FC00111249F938F9384EE90E19F9390
:109A70008F9382E08F930E94461A0F900F900F9061
:109A80000F900F9015C049EC50E00E94744010C038
:109A90008A81882339F00E947F522981FC01268324
:109AA0000E94065290E08A81882309F491E09A830B
:109AB00080E090E0DF91CF910895CF93DF93EB01A9
:109AC0008130910569F0823091051CF4892B81F079
:109AD00049C08230910539F183309105F9F042C0D7
:109AE0000E947F52FC01808599278C839D833AC018
:109AF00060E081E00E9468188C819D819F938F9324
:109B00008AEE90E19F938F9382E08F930E94461A92
:109B10000F900F900F900F900F9024C040E050E0F6
:109B20000E9474401FC08A81882361F483E08B8384
:109B300080E290E08E839F8391E0988F82E08F8B0C
:109B40009E8B0AC01E8A0E947F522C81FC012087B6
:109B50002093610A0E94065290E08A81882309F4CA
:109B600091E09A8380E090E0DF91CF910895EF92A9
:109B7000FF920F931F93CF93DF938C01EB010E9411
:109B80007F527C010230110509F463C003301105D6
:109B900044F40115110571F00130110509F446C0B6
:109BA00072C00330110509F43DC0063011050CF0F8
:109BB0006AC03CC08A81882309F465C0F7018085AA
:109BC000882309F460C060E081E00E9468188C81FD
:109BD0009D819F938F938FEE90E19F938F9382E06F
:109BE0008F930E94461A60E089810E94095C082FC9
:109BF00061E089810E94095C182FC0E80F900F90E6
:109C00000F900F900F9094E0802F8C2309F096E036
:109C1000812F8C2309F09F5F892F0E941A18C69507
:109C200091F731C01E8A81E00E942A5CF70180858D
:109C30009927AC01BE01C8010E947440898199270F
:109C400001968C839D838B818230E9F488E08B833D
:109C50001AC02A81222391F481E090E08C839D83B5
:109C6000F701808599278E839F8311E01A83822FC5
:109C70000E942A5C188F85E08F8B1E8B88E08B8377
:109C80008C818150898380E090E0DF91CF911F919A
:109C90000F91FF90EF900895CF92DF92EF92FF9295
:109CA0000F931F93CF93DF937C01C62F0E948F19D0
:109CB0000E947F526C01C33208F06FC085E0C89FDC
:109CC000800111240E5D1D4FF7018281882311F060
:109CD00080E001C082E00E941A18F6018581992770
:109CE00081309105B1F0823091051CF4892B39F057
:109CF00031C082309105B9F00397F9F02BC08C2F59
:109D0000992744E0880F991F4A95E1F78F5E914F9C
:109D10001DC08C2F992734E0880F991F3A95E1F7E1
:109D20008F50944F13C08C2F992724E0880F991FD0
:109D30002A95E1F78F52964F09C08C2F9927C4E0DE
:109D4000880F991FCA95E1F78F54984FBC0182E0A4
:109D50000E94F019E8018C8187FD0BC060E081E072
:109D60000E9468188C810E946D51BC0182E00E94A3
:109D7000F019E801EA81FB81309721F0B70180E01A
:109D800090E00995F7018689882329F06789808DFD
:109D90000E94711802C00E947718DF91CF911F9125
:109DA0000F91FF90EF90DF90CF90089560E0E2E296
:109DB000F2E0482F552747FD509520E030E08081A4
:109DC00099278417950711F4C90108956F5F2F5FD4
:109DD0003F4F3596623298F38FEF9FEF08950895C5
:109DE000BF92CF92DF92EF92FF920F931F93CF9388
:109DF000DF93CDB7DEB76B970FB6F894DEBF0FBE1B
:109E0000CDBFB82E21E2281718F480E090E0FBC106
:109E10006E010894C11CD11C8BE1F60111928A9548
:109E2000E9F7A89585E0B89EF0011124EE5DFD4F9D
:109E30000280F381E02D309721F0B60181E090E0BF
:109E400009956B2DC6010E944C4E0E94720E85E052
:109E5000B89E7001112482E292E0E80EF91E0E9481
:109E6000FF17AC018A30910509F4E9C08B309105E8
:109E700064F4009709F40AC1181619060CF41EC1FF
:109E80004F5F5F4F09F4AEC1E0CF8331910509F414
:109E90008EC08431910544F48B30910509F487C05C
:109EA000419709F49BC1D1CF8431910519F04597B1
:109EB00051F1CBCFF6018281882381F0F701228115
:109EC00033812115310531F0BE016F5F7F4F84E092
:109ED00090E081C1F60181818F5F28C0F601868BF9
:109EE000F7019081F0E2FB1534F0F70185818917C5
:109EF00011F4B39431C0892F0E94D64E682F772772
:109F000067FD709540C0F6018281882389F0F701D2
:109F1000228133812115310531F0BE016F5F7F4F02
:109F200085E090E058C1F60181818150818367C14D
:109F3000F601868B6B2DF7019081BB2091F02BEF02
:109F40003FEFE20EF31EF701808125E030E0E20EE4
:109F5000F31E891731F4BA946B2D772767FD70953E
:109F600012C030E23B1564F0D7011596F7018581E8
:109F7000891731F46F5F61321CF415968C91F8CF1C
:109F8000772767FD7095B62E85E0689FF001112454
:109F9000EE5DFD4F0280F381E02D309709F42FC173
:109FA000BE016F5F7F4F81E090E0099528C1F70106
:109FB0009181992361F1092F11270F521B4FF8014D
:109FC000808118162CF0892F0E94D64EF8018083CC
:109FD000F7018181E82FFF27EF52FB4F80810E941C
:109FE000F04E282F332727FD3095F7018181E82F88
:109FF000FF27EF52FB4FC90137FF04C0882799277D
:10A00000821B930B808337FFFAC0B1943AC0F701EB
:10A01000228133812115310551F0BE016F5F7F4FE1
:10A0200082E090E0F901099599237CF319C0F601CB
:10A030008281882309F491E0F6019283E0C0F60161
:10A0400082818823F1F0F7012281338121153105C6
:10A05000A9F0BE016F5F7F4F83E090E0F9010995A1
:10A06000F6018281882309F0CAC0F7012281338179
:10A07000BE016F5F7F4F81E090E0ADC0F6011282BC
:10A08000BEC08B2D992787FD9095BDC0F6018381B9
:10A09000813009F4DACE883089F481E00E942A5CAC
:10A0A00060E0F60181810E94095C61E0F601818136
:10A0B0000E94095C80E00E942A5CA1C0F6018381B5
:10A0C00099278530910509F454C08630910584F4B0
:10A0D0008230910581F1833091051CF40197B9F02C
:10A0E0008EC08330910599F0049709F43EC087C073
:10A0F0008730910509F456C0873091050CF44CC0A7
:10A100008830910521F0099709F453C078C0F60111
:10A1100086819781892B21F48FEF9FE78683978330
:10A12000F60186819781841795070CF468C0148224
:10A13000158282E08383F601848195819C0163E02E
:10A14000220F331F6A95E1F7280F391F280F391F97
:10A15000240F351F37FD53C08681978182179307DF
:10A160000CF44DC0248335834AC0F601108685E087
:10A170008383F60190858AE0989F90011124240F33
:10A18000351F2F3F310509F008F420878EEF9FEF30
:10A19000F601818F928F33C04830510584F5F60166
:10A1A00041872DC04230510554F5F601418F528F41
:10A1B00026C0F6018181E80FF11D842F805D828722
:10A1C000F7012281338121153105C9F0BE016F5F8E
:10A1D0007F4F82E090E0F901099511C080E00E9474
:10A1E0002F0E0DC0F6018381883009F02ECEBE01FE
:10A1F0006F5F7F4F80E090E00E94B74D26CE6B2DC1
:10A20000CE01019620CE6B960FB6F894DEBF0FBE3E
:10A21000CDBFDF91CF911F910F91FF90EF90DF9015
:10A22000CF90BF900895CF93C82F6CE571E080E088
:10A230000E94971964E671E082E00E94971964E831
:10A2400071E084E00E9497196CE771E085E00E945C
:10A25000971964E771E086E00E9497196CE671E057
:10A2600087E00E9497198091D104823210F01092F9
:10A27000D104C7FD04C08C2F0E94F04E0EC0809107
:10A28000D1040E94F04E992787FD909597FF03C057
:10A29000909581959F4F8093D1046CE372E080E0AC
:10A2A0000E9497196CE172E082E00E94971964EFB6
:10A2B00071E084E00E9497196CEE71E085E00E94E5
:10A2C000971964EE71E086E00E9497196CED71E0D9
:10A2D00087E00E949719CF910895CF93C82F8B31B3
:10A2E00018F089EE9BE12CC00E947F52FC01858111
:10A2F00099278230910581F0833091051CF40197F4
:10A3000021F018C0039779F015C081E1C89FC00102
:10A310001124825E954E14C081E1C89FC0011124B2
:10A320008D5A974E0DC081E1C89FC00111248857F6
:10A33000994E06C081E1C89FC001112483549B4EF1
:10A34000CF910895882319F086EF9BE108950E942C
:10A350007F52FC01858199278230910561F083301D
:10A3600091051CF4019721F00CC0039739F009C046
:10A370008CEA94E108958BE994E108958AE894E1E8
:10A38000089589E794E108950895CF93C82F8E30FA
:10A3900018F086E09CE138C00E947F52FC01858164
:10A3A00099278230910599F0833091051CF401972B
:10A3B00021F021C00397A9F01EC08C2F992754E0EB
:10A3C000880F991F5A95E1F787569C4E1DC08C2F18
:10A3D000992744E0880F991F4A95E1F787549D4ECD
:10A3E00013C08C2F992734E0880F991F3A95E1F715
:10A3F00087529E4E09C08C2F992724E0880F991F01
:10A400002A95E1F787509F4ECF910895EF92FF92E2
:10A410001F93CF93DF938AEDE82E84E0F82EC0E0FF
:10A42000D0E01FE1CE010E942D67F70161917F010D
:10A43000861719F0CE010E944667A8951150219603
:10A4400017FFF0CFDF91CF911F91FF90EF9008950C
:10A450009091DF04943008F091E08FE0EAEDF4E0B1
:10A4600011928A95E9F788E18093DE049093DF04E6
:10A4700081E08093DB0484E18093E00482E08093B8
:10A48000E50482E38093E6040E940652089540E2C8
:10A4900050E060E070E08AED94E00E9435678091C2
:10A4A000DC049091DD048F5F9F4F11F40E942852CD
:10A4B0008091DB04883018F081E08093DB04809188
:10A4C000E7049091E804885F974020F01092E80438
:10A4D0001092E7048091DF04843010F01092DF04C2
:10A4E0008AEF9FEFA1E0B0E0ABBFFC0187918F3F07
:10A4F00021F0882311F080936F00089508958AED6C
:10A5000094E008958093DF040E940652089580919C
:10A51000DB0499270895CF93C82F883008F0C7E04F
:10A520008091DB04C81751F0C093DB040E940652EF
:10A5300021E04EE468E08C2F0E94A00FCF91089597
:10A5400020E030E09091DA04982311F021E030E02F
:10A55000C90108959091DA04982B9093DA040E942F
:10A5600006520895982F90958091DA04892380935C
:10A57000DA040E94065208958CEF9FEFA1E0B0E04C
:10A58000ABBFFC0187919791A791B691B070BC01C8
:10A59000CD0108958FEF9FEFA1E0B0E0ABBFFC01CC
:10A5A0008791992708950E94C025FC01892BB9F055
:10A5B000AAEFB4E043E02D913C9111978081918105
:10A5C0002817390729F0828193812817390719F450
:10A5D0001D921C9211974150139647FFECCF08959E
:10A5E00008959F92AF92BF92CF92DF92EF92FF9227
:10A5F0000F931F93CF93DF93CDB7DEB726970FB698
:10A60000F894DEBF0FBECDBFC82E7B01942ECE01C5
:10A6100001960E94B854DD249AEFA92E94E0B92E39
:10A62000F501808191818E159F0509F096C0828188
:10A630008F5F8283843008F4C5C0C7010E94E8257B
:10A640008C01009709F4C0C0FFEFCF1639F59920AF
:10A6500029F0FC0164817581C7011BC0FC014481A4
:10A6600055816681C7010E942B2AC7010E94F95EAD
:10A67000BC01F80180850E948C2AF80182819381B7
:10A68000009749F00E94E825FC0164817581808172
:10A6900091810E94752A0E94982959C0992049F0F9
:10A6A000FC014481558160E0CE0101960E949B54DB
:10A6B00041C0FC01448155816681CE0101960E9412
:10A6C0009B54AE014F5F5F4F67E08C2D0E943B555E
:10A6D000F80180858F778B83C7010E94F95EBC01EA
:10A6E000CE0104960E94B8540E9451558823E1F38C
:10A6F000AE014F5F5F4F69E08C2D0E943B55F80122
:10A70000828193810E94C0258C010097D1F0FC01C9
:10A7100060817181CE0101960E94B854F801448194
:10A72000558160E0CE0101960E949B540E945155D4
:10A730008823E1F3AE014F5F5F4F68E08C2D0E94EC
:10A740003B5540E050E06DE08C2D0E943B55F501FB
:10A750001082118281E090E037C0D39483E090E0D2
:10A76000A80EB91E93E09D1508F05ACFDD240AEF1C
:10A7700014E0F80180819181892BA1F40E9489293C
:10A780008E159F0519F40E949E2907C0AE014F5FE8
:10A790005F4F65E08FEF0E943B55F801E082F18248
:10A7A000128206C0D3940D5F1F4FF3E0FD1508F72A
:10A7B00083E08D1538F4AE014F5F5F4F66E08FEF99
:10A7C0000E943B5580E090E026960FB6F894DEBFDD
:10A7D0000FBECDBFDF91CF911F910F91FF90EF90F2
:10A7E000DF90CF90BF90AF909F9008950F931F93ED
:10A7F000CF93DF93082FEB01672B79F010E040E057
:10A80000BE01802F0E94F152882339F40E945155D5
:10A810008823E1F31F5F143190F3DF91CF911F91F3
:10A820000F9108958F929F92BF92CF92DF92EF92F5
:10A83000FF920F931F93CF93DF93CDB7DEB7269789
:10A840000FB6F894DEBF0FBECDBFB82E4B016A0124
:10A85000CB010E94E8258C01892B09F445C0C60173
:10A860000E94E8257C01892B09F43EC0F80180850F
:10A870000E947D298C01F70180850E947D29081B9B
:10A88000190BC80117FF03C0909581959F4F029740
:10A89000E4F0FFEFBF1621F481E00E94FD2A24C0FE
:10A8A00086E0FE01319611928A95E9F781E089836D
:10A8B000AE014F5F5F4F61E28B2D0E943B5514C08C
:10A8C000B601C4010E94D3280FC010E041E0B601D8
:10A8D0008B2D0E94F152882399F70E9451558823AD
:10A8E000E1F31F5F143190F326960FB6F894DEBFA4
:10A8F0000FBECDBFDF91CF911F910F91FF90EF90D1
:10A90000DF90CF90BF909F908F9008950E94AC1ED3
:10A91000F894FFCF682790E027E0862F86959F5F09
:10A9200060FF03C0682F622701C0682F9830A8F32A
:10A93000862F99270895FC01262F862F8F778283F3
:10A9400026952074CA01892F9927869586958F733D
:10A95000822B8383CA0123E0969587952A95E1F798
:10A960008F778483842F8295807F8F778583089566
:10A97000FC01CB01262F2F772083880F892F881F7A
:10A98000990B91958F7781830895803480F4E82F17
:10A99000FF27662329F0E35CFA4F8AE0808308955D
:10A9A000E35CFA4F8081882311F081508083089501
:10A9B0000895EF92FF920F931F93CF93DF93782F19
:10A9C000C62F7A01A89580912A05282F33278091D8
:10A9D0002B05992701972817390741F080912A05FF
:10A9E000833039F480912B05882319F480E090E0BE
:10A9F0003BC090912A0589E0989F800111240A5F4D
:10AA00001A4F872F8068F8018083682F80E00E94AA
:10AA10008A54F801C1836C2F0E948A54982FE80150
:10AA2000229605E0E114F10431F0F70181917F01F4
:10AA30008F77888301C018826991892F0E948A5478
:10AA4000982F015007FFEECF87FD90959883809156
:10AA50002A058F5F80932A0580912A05843010F0A3
:10AA600010922A0581E090E0DF91CF911F910F9124
:10AA7000FF90EF9008950F931F93CF93DF93082FCC
:10AA8000162FEA0102C00E94720EAE01612F802FC4
:10AA90000E94D9548823B9F3DF91CF911F910F9170
:10AAA00008959F92AF92BF92CF92DF92EF92FF9262
:10AAB0000F931F93CF93DF93CDB7DEB76C970FB68D
:10AAC000F894DEBF0FBECDBF992458C227FF05C042
:10AAD000109233058FEF80933505809133058930CF
:10AAE00040F4E82FFF27EC5CFA4F20838F5F8093C0
:10AAF000330580913305893009F040C280913405D7
:10AB000087FF3CC244E3E42E45E0F42E90E017E0DA
:10AB1000F70181917F01682F892F0E948A54982F15
:10AB2000115017FFF5CF87FD909580913C05981740
:10AB300009F01FC2FF248091340588230CF019C24C
:10AB40003FE7B32EB82230913605C32EDD24409165
:10AB50003705842F99279695982F8827979587955D
:10AB6000C82AD92A20913505822F9927AA27BB27E1
:10AB7000FC013197E334F10508F0FBC1EA5BFF4FBC
:10AB8000EE0FFF1F0590F491E02D09941091380508
:10AB900080913905282F332726FD1068322F222770
:10ABA000330F330F80913A0599278F77907003E028
:10ABB000880F991F0A95E1F7282B392B80913B05C7
:10ABC000992780779070B4E095958795BA95E1F7CD
:10ABD000282B392B41E0B901C6010E94982841E099
:10ABE000612FC6010E941528C6010E94D352BDC123
:10ABF00080913805992790E4899F902D882711240A
:10AC0000C82AD92A60913905662319F041E0642FDA
:10AC100001C041E0C6010E940F64A7C180913805C0
:10AC2000682F772780913905282F3327C90187702E
:10AC300090709695982F882797958795682B792BF4
:10AC400020743070220F331F80913A05822B482FD9
:10AC5000C6010E946A2989C180913805E82EFF2427
:10AC6000002711278091390599279695982F8827D5
:10AC700097958795AA2797FDA095BA2FE82AF92AD4
:10AC80000A2B1B2B80913A05992790E4899F902DE0
:10AC900088271124AA2797FDA095BA2FE82AF92A18
:10ACA0000A2B1B2B20913B05822F9927AA27BB2714
:10ACB00087709070A070B07035E1880F991FAA1F3F
:10ACC000BB1F3A95D1F7E82AF92A0A2B1B2B2695A8
:10ACD00026952695D801C7010197A109B1098F5F73
:10ACE0009F4FAF4FB04008F040C1A601C801B70167
:10ACF0000E945E603AC10E946E0E843009F435C134
:10AD0000809136050E942F0E882309F42EC184E01D
:10AD10000E94CA662AC1C114D10409F426C1B60131
:10AD20008B2D0E94F65321C160913805C6010E9407
:10AD30002227809136058A87809137058B87C60147
:10AD40000E9404278C87AE01465F5F4F69E0A7C071
:10AD50001AE0E12EF12CEC0EFD1EAE01405F5F4FBC
:10AD6000BE01645F7F4FC6010E94B95E6C018F77A0
:10AD70008A87CC0CCD2CCC1CDD08D1948C2D8F7700
:10AD80008B8788898D8789898E871F86A70161E1D6
:10AD90008B2D0E943B558E010F5F1F4FF80194E0F1
:10ADA000818981879150319697FFFACFA70162E19F
:10ADB0008B2D0E943B55F80193E086898187915045
:10ADC000319697FFFACFA70163E169C0A3E0FA2E9D
:10ADD00033E0F30E83E0F80E8601243199F480917C
:10ADE0003805C82EDD248091390599279695982F2E
:10ADF000882797958795C82AD92A80913A058C8FFC
:10AE0000188A23C0AE01405F5F4FBE01645E7F4F72
:10AE1000C6010E94B95E6C0194E0EAE0EF1588F08B
:10AE2000DE01AF0DB11D5096E92FFF27EC5CFA4F04
:10AE300080818D939F5FF394973018F4FAE0FF15AB
:10AE400098F7FE01EF0DF11D108A9E01205F3F4F24
:10AE50004C8DB601C8010E94F95D8C018F778A87FD
:10AE6000000F012F001F110B1195802F12C02131EF
:10AE700021F4C6010E943C5F03C0C6010E94715FBD
:10AE80006C018F778A87CC0CCD2CCC1CDD08D1943B
:10AE90008C2D8F778B87AE01465F5F4F60E18B2DE6
:10AEA0000E943B5562C0C6010E94F65D5EC0809163
:10AEB0003805282F33278091390599279695982FA3
:10AEC000882797958795282B392BA901B6018B2DBB
:10AED0000E9412544AC0C6010E94F32846C0BB24F7
:10AEE000EDE3F5E08191882369F446E355E064E001
:10AEF0008B2D0E943B5580912D058B1538F4B09217
:10AF00002D0504C0B3943FE33B1560F782E08093C6
:10AF10002E052BC080912E05833038F583E0809379
:10AF20002E0530932F05409330058091380580938E
:10AF300031051092320519C080912E058230A8F497
:10AF400082E080932E0530932F05409330051092B8
:10AF500031050BC090912E05992339F481E080933F
:10AF60002E0530932F059093300561E08B2D0E94C4
:10AF7000C554109233058FEF809335050E94DF137F
:10AF80009C018FEF2F3F380709F0A0CD0E94A1133D
:10AF90000A970CF421C190912A0580912B059817EE
:10AFA00011F190912B0589E0989F70011124E6E042
:10AFB000F5E0EE0EFF1E08E010E0F70181917F0141
:10AFC0000E94B2130150104017FFF7CF80912B055C
:10AFD0008F5F80932B0580912B05843008F4FCC093
:10AFE00010922B05F9C07E010894E11CF11C570159
:10AFF00080912C05803429F060912E05662309F498
:10B0000075C08FEF89830894E11CF11C80912E0597
:10B01000992781309105C9F0823091051CF4892B64
:10B0200039F059C08230910519F10397C1F153C02D
:10B0300080E4F701819380912F05982F97708F5F9F
:10B0400080932F0591937F0148C081E4F70181939C
:10B0500080912F058770819380913005982F9F777D
:10B060008F5F8093300591937F018091300531C0CF
:10B0700082E4F701819380912F05877081938091FD
:10B0800030058F77819380913105982F9F778F5F5F
:10B090008093310591937F01809131051AC083E43B
:10B0A000F701819380912F058770819380913005FE
:10B0B0008F778193809131058F77819380913205CD
:10B0C000982F9F778F5F8093320591937F018091B6
:10B0D000320587FF02C010922E0580912E0588232D
:10B0E00009F059C080912C058F5F53C08134A1F5C0
:10B0F0008FEF89830894E11CF11C83E0F7018193B1
:10B100007F018F010894E11CF11C0E946E0E8F7765
:10B11000F801808380912C058F5F80932C050E941D
:10B1200086298C01FC01868581FF13C08081918175
:10B130000E94D35241E0F8016089808191810E9490
:10B14000152841E0F80164817581808191810E9418
:10B15000982851E0952E1FC0803410F060932C0584
:10B1600080912C05806889830894E11CF11C82E0A1
:10B17000F70181937F0180912C050E94C554809135
:10B180002C058F5F80932C0590912D05981718F44E
:10B1900080E480932C05CE010996E816F90620F488
:10B1A000F70111927F01F9CFDD24750107E010E06E
:10B1B000F70160818D2D0E948A54D82EF70181916C
:10B1C0007F010E94B2130150104017FFF1CFD7FC4E
:10B1D000D0948D2D0E94B213A895892D99276C9635
:10B1E0000FB6F894DEBF0FBECDBFDF91CF911F9198
:10B1F0000F91FF90EF90DF90CF90BF90AF909F9016
:10B200000895CF93DF93CDB7DEB726970FB6F894A6
:10B21000DEBF0FBECDBF36E0FE01319611923A95EA
:10B22000E9F74983AE014F5F5F4F0E943B55269679
:10B230000FB6F894DEBF0FBECDBFDF91CF9108955A
:10B240001F93CF93DF93EC0110E001C0A8950E94FB
:10B250000C1F8823D9F310C0A89504C081E090E0AA
:10B260000E94C1160E940C1F8823C1F361E080E098
:10B2700090E00E94311D21970E941C1F882311F429
:10B28000209751F70E941C1F811111E0C5E00EC0EC
:10B2900063E080E090E00E94311D0E94201F01C009
:10B2A000A8950E940C1F8823D9F3C1500E941C1F2F
:10B2B000882311F0CC2361F7CC2309F41C2F812FB4
:10B2C0009927DF91CF911F910895EF92FF921F93DD
:10B2D000CF93DF937C01CFEFDFEF10E0612FC70149
:10B2E0000E94AA1D80E090E00E942059882311F05E
:10B2F000C12FDD271F3F49F483E090E00E942059D1
:10B30000882331F0CFEFD0E005C01F5FD7FDE6CF37
:10B31000D7FD14C01C2FCFEFDFEF612FC7010E94B4
:10B32000AA1D83E090E00E942059882311F0C12FCC
:10B33000DD27112319F01150D7FDEFCFCE01DF919A
:10B34000CF911F91FF90EF9008954F925F926F926F
:10B350007F928F929F92AF92BF92CF92DF92EF92A5
:10B36000FF920F931F93CF93DF93CDB7DEB726974E
:10B370000FB6F894DEBF0FBECDBF782E5B01C42E92
:10B38000522E402E8091620082608093620080E0A5
:10B390000E94BB1986E0FE01319611928A95E9F769
:10B3A000AE014F5F5F4F62E28FEF0E943B550E94FC
:10B3B0002D1F83EC87B98FEE86B96FEF862E962E00
:10B3C000662480E00E942F0E82E390E00E94C11666
:10B3D00084E00E942F0E84E690E00E94C116E09067
:10B3E000CA06F090CB060091CC061091CD0680EDF8
:10B3F00097E0A0E0B0E0E80EF91E0A1F1B1FDD2455
:10B4000010927E0510927D052BC00E94281FAC0172
:10B4100020917D0530917E05C901885A9D4F841782
:10B42000950734F0C901885592404817590744F4EC
:10B4300050937E0540937D05DD2059F0DA9409C0D4
:10B44000240F351F3595279530937E0520937D0574
:10B45000D39494E09D1550F08AE090E00E94C116CC
:10B46000C801B7010E948A14882379F280917D0572
:10B4700090917E0544975CF584E393E00E94231F3E
:10B4800083E090E00E94205910E0412F612F80E07E
:10B4900090E00E94711D83E090E00E94205981118C
:10B4A00011E041E060E080E090E00E94711D83E0E7
:10B4B00090E00E94205981111F5F113041F484E116
:10B4C00090E090937E0580937D0545E0D42E809199
:10B4D0007D0590917E054497855A9B4028F4B4E001
:10B4E000BD1510F1442001F560E081E00E9468186C
:10B4F00080917D0590917E058431910514F485E15C
:10B5000006C0895B9B4014F086E101C087E10E9480
:10B510006D51BC0182E00E94F01980E00E942F0E64
:10B5200088EE93E00E94C11680917D0590917E0582
:10B53000805E9C4F0E94231F86E990E00E94C11606
:10B540000E946E0E843009F0D8C0072D11270330F9
:10B55000110509F447C0043011054CF40130110500
:10B5600039F102301105FCF4012B71F0ACC005304B
:10B5700011050CF4A8C0073011050CF453C00930B4
:10B5800011050CF0A0C06FC0452D6C2DC5010E94A7
:10B59000511D8FE090E00E942059882309F497C044
:10B5A000852C992494C06C2DC5010E94C31D4CC0EC
:10B5B00040E06C2DC5010E94711D83E090E00E9467
:10B5C0002059882309F046C041E06C2DC5010E9436
:10B5D000711D83E090E00E942059882309F477C010
:10B5E000480177C010E0012F169540E0602FC5019B
:10B5F0000E94711D83E090E00E942059882309F485
:10B6000010680F5F083080F3612FC5010E94DC1DB8
:10B6100083E090E00E942059882309F458C0812ECD
:10B62000992455C061E085E090E00E94911D8FE073
:10B6300090E00E942059C50187709070F5E07F1658
:10B6400061F46C2D0E94911D8FE090E00E942059C2
:10B650008823E9F1882499243CC00E9465594C0153
:10B6600033E0632E34C0C5019695879596958795EE
:10B67000682F6F5F85E090E00E94911D8FE090E061
:10B680000E942059C5018370907027E0721661F402
:10B690006C2D0E94911D8FE090E00E94205988231C
:10B6A00041F08824992405C00E9465594C0193E01B
:10B6B000692E61E085E090E00E94911D8FE090E0AE
:10B6C0000E94205904C08FEF882E982E08C097FC46
:10B6D00006C0442021F08CE291E00E94C11680E077
:10B6E0000E942F0E97FE09C08CE291E00E94C116C5
:10B6F000639482E0861508F064CE16B886B187B9E7
:10B700000E947F52FC0184810E94BB1981E08983E1
:10B71000AE014F5F5F4F62E28FEF0E943B55809119
:10B7200062008D7F80936200C40126960FB6F89464
:10B73000DEBF0FBECDBFDF91CF911F910F91FF9064
:10B74000EF90DF90CF90BF90AF909F908F907F90C1
:10B750006F905F904F9008950F93242F01E0462F34
:10B76000BC0180E00E94A5590F9108950F9300E05D
:10B77000202F462FBC0181E00E94A5590F9108950A
:10B780000F9301E020E0462FBC0182E00E94A55902
:10B790000F9108950F9300E0202F402FBC0183E00C
:10B7A0000E94A5590F9108950F9301E020E0482FC2
:10B7B00060E070E085E00E94A5590F9108950F9315
:10B7C000992701E020E0462FBC0185E00E94A559A1
:10B7D0000F9108950F93992700E0202F402FBC016F
:10B7E00086E00E94A5590F9108950F9301E020E093
:10B7F000462FBC0187E00E94A5590F9108950F9331
:10B8000000E0202F402FBC0188E00E94A5590F9135
:10B810000895880F61118F5FF894E82FFF27ED5589
:10B82000F54F90818091620A80FD10827894892F73
:10B8300099270895880F61118F5FF894E82FFF27EB
:10B84000DF01AD51B54F8C91ED59F54F8083789460
:10B85000992708959091620A882311F0916001C0A0
:10B860009E7F9093620A0895089580E4E3E6FAE0EB
:10B8700011928A95E9F7089584E0809374001092FC
:10B88000710082E28093700008951F920F920FB6AC
:10B890000F9211248F939F93EF93FF9380917100E8
:10B8A0009927887F90708032910509F487C0813292
:10B8B00091056CF480319105D9F0813191051CF42A
:10B8C0000897D1F07DC0489709F43FC079C0803413
:10B8D0009105A9F18134910524F4889709F441C0B8
:10B8E0006FC080359105D9F08835910561F068C049
:10B8F00080917F0587FF02C080EA01C081EA8093C2
:10B90000730085E861C0E0918505F091860580911E
:10B9100073008193F0938605E093850548C0E0911C
:10B920008505F0918605809173008193F0938605DB
:10B93000E0938505809180058150809380058091FA
:10B9400080058230F4F285EC3FC0809183059091B0
:10B950008405892F9927809373008FEF80937F054B
:10B96000D0CF80917F0587FF09C08091830590919A
:10B9700084058093730010927F05C3CF8091810569
:10B980008823E1F080918005882389F0E091850586
:10B99000F09186058191F0938605E093850580936B
:10B9A000730080918005815080938005AACF84E93F
:10B9B0008093740081E08093820508C085EA04C00A
:10B9C0008FEF8093820584E980937400FF91EF915B
:10B9D0009F918F910F900FBE0F901F90189580919F
:10B9E0007400992787709070009711F081E090E0C3
:10B9F000089508956093800590938405809383054E
:10BA00002093810550938605409385058EEF8093A2
:10BA10007F051092820585EA8093740008958091D5
:10BA20008205992787FD909508950E94FA5C01C0D0
:10BA3000A8950E940F5D892BD9F3809182059927E3
:10BA400087FD90950895AB0120E060E134E0880F18
:10BA5000991F3A95E1F70E94155D0895AB0121E029
:10BA600060E174E0880F991F7A95E1F70E94155DF7
:10BA7000089520E0AC0164E080E090E00E94155D54
:10BA8000089521E0AC0164E080E090E00E94155D43
:10BA90000895EF92FF920F931F93CF93DF93CDB74B
:10BAA000DEB722970FB6F894DEBF0FBECDBF7C0184
:10BAB00019821A8209811A8120E0AE014F5F5F4F1F
:10BAC00062E0C801E4E0880F991FEA95E1F70E945F
:10BAD000155DA89589819A81009719F08E159F05AB
:10BAE00049F7C80122960FB6F894DEBF0FBECDBF4E
:10BAF000DF91CF911F910F91FF90EF9008950F93D9
:10BB00001F93CF93DF93CDB7DEB722970FB6F8948C
:10BB1000DEBF0FBECDBF8C0101978F5F934000F554
:10BB200020E0AE014F5F5F4F62E0C801A4E0880FE4
:10BB3000991FAA95E1F70E94155DC8010E94495D11
:10BB400024E08030920760F421E0AE014F5F5F4F48
:10BB500062E0F4E0880F991FFA95E1F70E94155D05
:10BB600022960FB6F894DEBF0FBECDBFDF91CF9106
:10BB70001F910F9108950F931F93CF93DF93CDB72C
:10BB8000DEB764970FB6F894DEBF0FBECDBF8C0151
:10BB900001978F5F9340F8F4C8010E947F5DCE014A
:10BBA00041960E94395D40E150E06FEF70E0CE01B8
:10BBB00001960E9466678B899C8989839A83BE015E
:10BBC0006F5F7F4FC8010E942E5D0B8B1C8BCE01D7
:10BBD00041960E94415D64960FB6F894DEBF0FBE99
:10BBE000CDBFDF91CF911F910F9108950E94BB5D52
:10BBF00008957F928F929F92AF92BF92CF92DF92E1
:10BC0000EF92FF920F931F93CF93DF93CDB7DEB7E1
:10BC1000AA970FB6F894DEBF0FBECDBF7C014B01D3
:10BC2000742E5901232B79F1672B69F180E0E81616
:10BC300084E0F80640F5E114F10421F0C7010E9408
:10BC40007F5D1EC0CE0181960E94395D0BA11CA1B3
:10BC50000115110511F4C70112C020E0AE014D5DC0
:10BC60005F4F62E0C80134E0880F991F3A95E1F711
:10BC70000E94155DCE0181960E94415DC8017C0144
:10BC8000E114F10411F4C70158C06E010894C11CFD
:10BC9000D11CF5018B829C827D82DE01169620816B
:10BCA000222351F0CE014196A817B90728F4319606
:10BCB0002D9320812223C1F7C6014096A817B9070A
:10BCC00008F41C92E9A6FAA6CE0185960E94395D79
:10BCD000EE24FF240DA11EA101151105B1F0A895B8
:10BCE000BE016F5E7F4FC8010E94235DC6010596AD
:10BCF0004BE050E0BC01CE0146960E94AF6799230D
:10BD000024F4780109891A89E7CFF60100831183A9
:10BD1000A895B60189A59AA50E942E5D21E0AE01E5
:10BD2000475D5F4F62E0C701B4E0880F991FBA9585
:10BD3000E1F70E94155D89A59AA5AA960FB6F89419
:10BD4000DEBF0FBECDBFDF91CF911F910F91FF904E
:10BD5000EF90DF90CF90BF90AF909F908F907F90AB
:10BD600008959A01462FBC0180E090E00E94F95DA1
:10BD70000895EF92FF920F931F93CF93DF93CDB768
:10BD8000DEB760970FB6F894DEBF0FBECDBF9C0143
:10BD90007B018A0101978F5F934018F080E090E06B
:10BDA0001BC0BE016F5F7F4FC9010E94235DE1147C
:10BDB000F10419F08D81F70180830115110551F00F
:10BDC0008BE0F801DE0116960D9001928A95E1F75D
:10BDD000F80113868B819C8160960FB6F894DEBFC4
:10BDE0000FBECDBFDF91CF911F910F91FF90EF90CC
:10BDF0000895EF92FF920F931F93CF93DF93CDB7E8
:10BE0000DEB764970FB6F894DEBF0FBECDBF7C01DE
:10BE1000CE0141960E94395D09891A891BC08FEFB6
:10BE20000F3F1807D1F020E0AE014F5F5F4F64E095
:10BE3000C801062E02C0880F991F0A94E2F70E94DB
:10BE4000155D8B819C818E159F0511F4C80107C07B
:10BE500009811A810115110511F780E090E06496BF
:10BE60000FB6F894DEBF0FBECDBFDF91CF911F910B
:10BE70000F91FF90EF9008950F931F93CF93DF934F
:10BE8000CDB7DEB764970FB6F894DEBF0FBECDBF57
:10BE90008C018150944018F080E090E017C0CE01F2
:10BEA00041960E94395D0115110571F0BE016F5F69
:10BEB0007F4FC8010E94235D89819A81009721F0FC
:10BEC0002FEF8F3F920711F489899A8964960FB6F4
:10BED000F894DEBF0FBECDBFDF91CF911F910F91C0
:10BEE0000895CF93DF93CDB7DEB724970FB6F894BC
:10BEF000DEBF0FBECDBF24E08130920718F080E096
:10BF000090E00FC0009739F4CE0101960E94395D90
:10BF100089819A8106C00E94495D009711F40E94B0
:10BF2000495D24960FB6F894DEBF0FBECDBFDF91FA
:10BF3000CF910895EF92FF920F931F93CF93DF93CA
:10BF4000CDB7DEB764970FB6F894DEBF0FBECDBF96
:10BF5000198A1A8A01E010E00B8B1C8BA895CE0180
:10BF600041960E94415D40E150E06FEF70E0CE01EC
:10BF7000800F911F0E94666740E1E42EF12C83E060
:10BF80000F3F18073CF40F5F1F4F09831A830150BE
:10BF9000104002C019821A820E94720E21E0AE0186
:10BFA0004F5F5F4F60E1C7010E94155D0F5F1F4F3C
:10BFB00080E190E0E80EF91E94E000301907FCF2F1
:10BFC00064960FB6F894DEBF0FBECDBFDF91CF9160
:10BFD0001F910F91FF90EF900895EF92FF920F93B2
:10BFE0001F93CF93DF93CDB7DEB764970FB6F89466
:10BFF000DEBF0FBECDBFCE0141960E94395D89E004
:10C000000E943D17882329F08EE00E943D17882367
:10C0100051F48B899C898F5F9F4F21F589899A897B
:10C020008F5F9F4FF9F464E971E084E00E949719F3
:10C030006CE871E085E00E94971968EC70E085E794
:10C040009BE40E94A11860E0862F0E94681883E09C
:10C050000E946D51BC0182E00E94F0190E949A5F1B
:10C060000E94865409891A89C80101978F5F9340FD
:10C07000C0F4BE016F5F7F4FC8010E94235DE9805D
:10C08000FA808B819C8101978F5F974218F0C801DD
:10C090000E94BB5D8701A895C70101978F5F934000
:10C0A00040F364960FB6F894DEBF0FBECDBFDF91AC
:10C0B000CF911F910F91FF90EF900895EF92FF9213
:10C0C0000F931F93CF93DF93CDB7DEB728970FB6AB
:10C0D000F894DEBF0FBECDBF7B018C01FA018091C9
:10C0E000870590918805892B91F1E982FA820B836B
:10C0F0001C831F821886022F112700FF09C04F835F
:10C10000588740E050E0BA01CF010E94B95EFC01BF
:10C1100001FF05C08F81988590688F839887ED8394
:10C12000FE83EF2BA1F021E0AE014F5F5F4F68E08F
:10C1300080918705909188050E94155D8091870503
:10C140009091880508969093880580938705289696
:10C150000FB6F894DEBF0FBECDBFDF91CF911F9118
:10C160000F91FF90EF900895CF92DF92EF92FF92A0
:10C170001F93CF93DF93CDB7DEB728970FB6F89410
:10C18000DEBF0FBECDBF10E0C12C30E4D32E8091B6
:10C19000600A181798F5812F9927FC0123E0EE0F0C
:10C1A000FF1F2A95E1F7E80FF91FE80FF91FE0528A
:10C1B000F84F8081918189839A83828193818B83D7
:10C1C0009C83848195818D839E838085282F33274E
:10C1D0002F833887868187FD03C031602F8338879E
:10C1E00021E0AE014F5F5F4F68E0C6010E94155D20
:10C1F0001F5F88E090E0C80ED91EC9CF0E947F5211
:10C200002FEF3FEF29833A83FC01858596858B8349
:10C210009C8321E0AE014F5F5F4F68E0C6010E9442
:10C22000155D88E090E0C80ED91E0E948629FC01A9
:10C23000D0928805C0928705828993892685892BAB
:10C2400041F020FF02C023E001C021E04289538970
:10C2500007C020FF02C022E001C020E040815181E0
:10C2600060E070E080E090E00E945E6010E040E0FE
:10C2700050E06BE0812F0E943B551F5F1034B8F3F4
:10C2800010E00E9451558823E1F31F5F1630C8F378
:10C2900010E0212F4FEF5FEF6FEF7FEF8FEF9FEFFA
:10C2A0000E945E60C0908705D09088051092880536
:10C2B0001092870583E2E82E8BE0F82E1FE121E043
:10C2C000A70168E0C6010E94155D1150E8E0F0E0AA
:10C2D000EE0EFF1ECE0EDF1E17FFF1CF28960FB613
:10C2E000F894DEBF0FBECDBFDF91CF911F91FF90BD
:10C2F000EF90DF90CF9008957F928F929F92AF92B0
:10C30000BF92CF92DF92EF92FF920F931F93CF9342
:10C31000DF93CDB7DEB76C970FB6F894DEBF0FBED4
:10C32000CDBF0E946E0E782E80E00E942F0E40E05E
:10C3300050E060E0CA010E942B2A86E08E010F5E69
:10C340001F4FF80111928A95E9F7FF24A80167E0D1
:10C350008F2D0E943B5584E190E00E94C116F3941A
:10C360002FE32F1598F70E94782519821A82A12CA5
:10C3700000E4B02E20E0AE014F5F5F4F68E0C501E2
:10C380000E94155D89819A81EFEF8F3F9E07E1F052
:10C390000E94E8258C01892BB9F08F818F70682F5E
:10C3A000F801808191810E9422278B819C81F80174
:10C3B000828393838D819E81848395838F819885E9
:10C3C000892F992780FD168288E090E0A80EB91E7B
:10C3D00089819A818F5F9F4F69F619861A861B861D
:10C3E0001C86B9E08B2E912C8C0E9D1E20E0A401A2
:10C3F00068E0C5010E94155D89859A85AB85BC857D
:10C4000080509040A040B14008F0AAC08D859E8524
:10C41000009709F4A5C028E28030920708F0A0C078
:10C42000FF242F85388937FF02C0A2E0FA2E8C0145
:10C430002115310589F089011F7740E050E0BA01EC
:10C44000C8010E94B95E2D853E852817390719F469
:10C4500081E0F82A01C08901F40120813181428103
:10C460005381CF2CDD242115310541055105D1F52E
:10C470000E9486297C01C0FE08C04496AC0160E0A1
:10C4800070E0C8010E94B95E8C01C8010E94C025FD
:10C490008C010097E1F0FC01448155816681808127
:10C4A00091810E942B2A60E070E0F80180850E9453
:10C4B0008C2AF801828193810E94C025009739F06F
:10C4C000FC0164817581808191810E94752AC1FE81
:10C4D00004C0F701868581608687F70186858260C2
:10C4E00086873EC0802F8F778F8B000F012F001F14
:10C4F000110B1195802F8F77888FF40180818F77B2
:10C50000898FE7E05695479537952795EA95D1F7B6
:10C51000822F8F778A8F77E05695479537952795A5
:10C520007A95D1F7822F8F778B8F67E05695479555
:10C53000379527956A95D1F7822F877053E0CC0CF9
:10C54000DD1C5A95E1F78C298C8FAE01495E5F4F57
:10C550006CE08FEF0E943B550E9451558823E1F318
:10C5600088E090E0A80EB91E89859A85AB85BC85C8
:10C5700080509040A040B14008F433CF03E21BE06C
:10C580004FE1F42E20E0A80168E0C5010E94155D8E
:10C59000FA94085F1F4F88E090E0A80EB91EF7FEDE
:10C5A000F1CF83E00E942F0E84E690E00E94C11636
:10C5B0008B819C810E94D165872D0E942F0E6C96E5
:10C5C0000FB6F894DEBF0FBECDBFDF91CF911F91A4
:10C5D0000F91FF90EF90DF90CF90BF90AF909F9022
:10C5E0008F907F9008952FEF3FEFE9E8F5E08FE11E
:10C5F000208331833796815087FFFACF0895AC01AD
:10C60000FC0123E0F695E7952A95E1F7ED5DF44FFF
:10C61000808199279A012770307002C0959587957F
:10C620002A95E2F7440F551F382F317080FF02C062
:10C630004F5F5F4F20E0E9E8F5E08081918184174A
:10C64000950759F4868180FF0CC0332319F082E5E9
:10C6500090E0089587E490E008952F5F37962032A8
:10C6600060F3332319F082E790E0089587E690E0C5
:10C67000089508951F93CF93DF93EC01162F892B14
:10C6800009F4A2C0662319F08E8180FD9DC011239C
:10C6900009F481C08091690690916A06A0916B06A9
:10C6A000B0916C068896A11DB11DBC01CD010E9400
:10C6B0008A14882309F488C04881598190E0E9E808
:10C6C000F5E0BA01B3E076956795BA95E1F7208178
:10C6D00031818FEF2F3F380779F02417350761F04C
:10C6E000868180FF09C0A3E036952795AA95E1F7DA
:10C6F0002617370709F468C09F5F3796903238F3E2
:10C7000061E0888199810E941C1D8091CA069091E8
:10C71000CB06A091CC06B091CD068A839B83AC83D7
:10C72000BD838093690690936A06A0936B06B093CD
:10C730006C068E8181608E8383FF06C0888199811B
:10C74000969587950E94D06648815981CA0164E018
:10C75000969587956A95E1F7682F9A013695279502
:10C760002770307081E090E002C0880F991F2A95F1
:10C77000E2F7982F772740FF06C0FB01ED5DF44FED
:10C780008081892B06C0FB01ED5DF44F909580817F
:10C79000892380833EC08E8182608E83992780FFAB
:10C7A00013C082FF11C08091690690916A06A09122
:10C7B0006B06B0916C068896A11DB11DBC01CD0120
:10C7C0000E948A14882319F480E090E024C0612F2D
:10C7D000888199810E941C1D8091CA069091CB0688
:10C7E000A091CC06B091CD068093690690936A061D
:10C7F000A0936B06B0936C068E8183FF06C0888180
:10C800009981969587950E94D0668FEF9FEF8883D8
:10C81000998381E090E0DF91CF911F910895FF927D
:10C820000F931F93CF93DF938C01F62E805F9F4071
:10C8300018F080E090E051C020E0E9E8F5E0808168
:10C8400091818017910731F12F5F37962032B8F32D
:10C85000FF2089F41CC0008311838091CA06909147
:10C86000CB06A091CC06B091CD0682839383A4839E
:10C87000B58316820FC020E0E9E8F5E08081918160
:10C880008F5F9F4F41F32F5F37962032B8F3C0E0A0
:10C89000D0E003C0EF01309721F4CE01FF20E9F48E
:10C8A0001AC0442319F08681886086830E947F52D3
:10C8B000FC01FF2061F098013695279585859685C6
:10C8C0008217930720F4258736870E9406526F2D22
:10C8D000CE010E943A6381E090E0DF91CF911F91F9
:10C8E0000F91FF9008956F927F928F929F92AF92D7
:10C8F000BF92CF92DF92EF92FF920F931F93CF934D
:10C90000DF930E947F528C01FC0183859927AA271F
:10C91000BB27BC01CD0122E330E040E050E00E94A3
:10C920006D6C6B017C01F80184859927AA27BB27D0
:10C93000BC01CD0124E630E040E050E00E946D6C87
:10C940003B014C01AA24BB24C9E8D5E00FE1888152
:10C9500099818F5F9F4F51F18E81992780FF14C07D
:10C9600082FD24C08A819B81AC81BD818C0D9D1D7F
:10C97000AE1DBF1DBC01CD010E948A148823B1F0F9
:10C980008E8184608E8312C0A114B10471F0F50110
:10C9900022813381448155818A819B81AC81BD8113
:10C9A00082179307A407B50708F45E010150279684
:10C9B00007FFCDCF8091690690916A06A0916B0622
:10C9C000B0916C068896A11DB11DBC01CD010E94DD
:10C9D0008A14882399F08091CA069091CB06A09181
:10C9E000CC06B091CD068897A109B109809369065C
:10C9F00090936A06A0936B06B0936C0600E0C9E8BA
:10CA0000D5E0888199818F5F9F4FE1F08E819927D2
:10CA100080FF18C082FF16C081FD0EC08A819B81F5
:10CA2000AC81BD81860D971DA81DB91DBC01CD012E
:10CA30000E948A14882331F060E0CE010E943A639C
:10CA4000882359F40F5F27960032D8F2A114B1045D
:10CA500021F061E0C5010E943A63DF91CF911F91FF
:10CA60000F91FF90EF90DF90CF90BF90AF909F908D
:10CA70008F907F906F900895CF93DF93EC018FE0BC
:10CA8000C03FD80718F08FEF9FEF23C0D695C7950A
:10CA900083E0CD3FD807C0F4D695C795D695C79506
:10CAA000CE0123E0969587952A95E1F78452904F21
:10CAB0000E942D679927C770D07002C09595879501
:10CAC000CA95E2F780FF03C083E090E002C081E0F6
:10CAD00090E0DF91CF9108951F93CF93DF93039759
:10CAE00011F41FEF01C010E0CCEDDFE0A895612F3D
:10CAF000CE010E94466721968FE0CC3FD807B4F361
:10CB0000DF91CF911F910895EF92FF920F931F93A2
:10CB1000CF93DF93EC018B018FE0C03FD807D0F5B6
:10CB20006330710519F061307105A1F5D695C7958F
:10CB300083E0CD3FD80770F5D695C795D695C795B4
:10CB40007E0153E0F694E7945A95E1F7C7018452C9
:10CB5000904F0E942D67682F9E0127703070033020
:10CB6000110549F481E090E002C0880F991F2A95D1
:10CB7000E2F7682B09C081E090E002C0880F991F9E
:10CB80002A95E2F780956823A895C7018452904FB3
:10CB90000E944667DF91CF911F910F91FF90EF9018
:10CBA00008959F92AF92BF92CF92DF92EF92FF9241
:10CBB0000F931F93CF93DF937C0188EFE81687E0F4
:10CBC000F80608F076C00E947F525C01FC01E58601
:10CBD000F6860E940652CC24DD249924092D1127C3
:10CBE000E016F10608F450C0C801F3E09695879569
:10CBF000FA95E1F7482F98012770307081E090E0B6
:10CC000002C0880F991F2A95E2F7982FE801CC0FF0
:10CC1000DD1FE42FFF27ED5DF44F8081892309F0AC
:10CC2000219640E061E0CE010E940F6440E0642F55
:10CC3000CE010E940F6460E081E00E9468180894B1
:10CC4000E11CF11CFF92EF920894E108F1080894AE
:10CC5000C11CD11CDF92CF9288E10E946D519F933D
:10CC60008F9382E08F930E94461A84E690E00E94A0
:10CC7000C1168DB79EB707960FB6F8949EBF0FBE2C
:10CC80008DBF0C5F1F4FACCFF501838599270E94A4
:10CC9000C1169394F3E0F91508F0A0CF84E690E074
:10CCA0000E94C11602C00E94720E0E940C1F8823AF
:10CCB000D1F3DF91CF911F910F91FF90EF90DF9013
:10CCC000CF90BF90AF909F900895EF92FF920F93F7
:10CCD0001F93CF93DF9380916D06682F7727109273
:10CCE0006D06E3E2FCE08191882311F0706805C0D5
:10CCF0008DE0E232F807B9F3B4F340E050E0809100
:10CD0000600A9927481759079CF4DC019A01F90138
:10CD1000E40FF51FE052F84F878180FF02C0706476
:10CD200007C04F5F5F4F275F3F4F4A175B077CF39A
:10CD300040E050E08091610A9927880F991F4817B9
:10CD4000590704F57C01E3EAFAE003E61AE0C3EED2
:10CD5000DAE09991D8018D918D01981759F480816D
:10CD6000282F3327892F99278095909528233923B9
:10CD7000232B11F0706206C04F5F5F4F31964E1546
:10CD80005F053CF3CB01DF91CF911F910F91FF9095
:10CD9000EF90089590916D06982B90936D060895ED
:10CDA0009C0187E0283F3807A0F4F90183E0F6955D
:10CDB000E7958A95E1F7ED5DF34F2770307081E0DC
:10CDC00090E002C0880F991F2A95E2F72081282B56
:10CDD00020830895089528E28030920740F40E944D
:10CDE000C025FC01892B19F0878181608783089514
:10CDF0000895CF93DF9310926D0680E091E0E3E217
:10CE0000FCE011920197E9F7C3E6DAE0A3EEBAE09D
:10CE1000E3EAFAE08091610A9927880F991F009749
:10CE200041F09C018D919191892B89932150304043
:10CE3000C9F7E0EEF7E08091600A9927009751F07A
:10CE40009C0187818E7F8783215030403A9621153F
:10CE50003105B9F7DF91CF910895E199FECF9FBBDE
:10CE60008EBBE09A99278DB308954115510569F05D
:10CE7000DC01E199FECF7FBB6EBBE09A6F5F7F4F15
:10CE80000DB20D9241505040B1F70895E199FECF97
:10CE90009FBB8EBB6DBB0FB6F894E29AE19A0FBEB2
:10CEA00008954115510589F0DC018FB7E199FECF56
:10CEB0007FBB6EBB0D900DBAF894E29AE19A8FBFDA
:10CEC0006F5F7F4F4150504089F70895DC0101C0EA
:10CED0006D9341505040E0F708950F931F93CF9307
:10CEE000DF93CDB7DEB72C970FB6F894DEBF0FBE39
:10CEF000CDBF0B891C89ED89FE893EE03C83098307
:10CF00001A834FEF5FE74D835E83AE01495E5F4F4B
:10CF1000BF01CE0101960E9428692F813885020F3A
:10CF2000131FD8011C922C960FB6F894DEBF0FBECB
:10CF3000CDBFDF91CF911F910F910895FB01DC01CF
:10CF40008D910190801911F40020D1F7990B08956B
:10CF5000FB01DC0101900D920020E1F70895FB0137
:10CF6000DC014150504030F08D910190801919F44E
:10CF70000020B9F7881B990B0895FB01DC01415093
:10CF8000504030F08D910590801919F40020B9F7C8
:10CF9000881B990B08952F923F924F925F926F9248
:10CFA0007F929F92AF92BF92CF92DF92EF92FF92C9
:10CFB0000F931F93CF93DF93CDB7DEB76E970FB666
:10CFC000F894DEBF0FBECDBF898B9A8B6B8B7C8BA9
:10CFD0004D8B5E8B3C011F8A188EF30191903F01AF
:10CFE000892D99270E94E76C892BB9F70DE29016DD
:10CFF00009F4FFC01BE2911609F4F7C02D893E89A0
:10D000002115310509F4DAC02031310509F4D6C003
:10D01000ED89FE89EF2B41F430E3931609F4C9C082
:10D020004AE050E04D8B5E8B8D899E89AA2797FD43
:10D03000A095BA2F898F9A8FAB8FBC8F8F89988DCF
:10D04000892B09F4B1C060E070E080E090E8298DA0
:10D050003A8D4B8D5C8D0E94186D29873A874B87DE
:10D060005C876D877E878F87988B58E0DE011196ED
:10D07000FE01399601900D925A95E1F7CC24DD24FA
:10D080007601AA24BB2429803A804B805C802D81C4
:10D090003E812D8F3E8F092D1127C8010E94DB6C28
:10D0A000892BC9F1C8010E94E06C892B09F46BC07F
:10D0B00070ED970E892D99276D897E8986179707C0
:10D0C00054F5B7FC24C02C143D044E045F04F8F062
:10D0D000C214D304E404F504A9F021E0A22EB12C7B
:10D0E000C701B601298D3A8D4B8D5C8D0E946D6C08
:10D0F0006B017C01C90CD11CE11CF11CD3019D907A
:10D100003D01C9CFAD8CBE8CA816B90634F73FEFF0
:10D11000A32EB32EF3CFB7FE29C0EF89F88DEF2BE6
:10D12000E1F0C12CD12CE12C90E8F92E02E210E0C4
:10D130001093240D0093230D8B899C89892B09F46E
:10D1400060C0AB2839F0C3010197AB89BC898D93CE
:10D150009C9357C089899A89F8CF8FEFC82E8FEF9B
:10D16000D82E8FEFE82E8FE7F82EE0CFAF89B88D5D
:10D17000AB2B11F3F094E094D094C094C11CD11C5B
:10D18000E11CF11CD9CFC8010E94C16C892B19F296
:10D19000C8010E94BF6C892B21F0802F8753982EE5
:10D1A00089CF802F8755FBCF6FEF7FEF8FEF9FE702
:10D1B0004ECF08E010E00D8B1E8B36CF40E3941667
:10D1C00009F026CFF3018081883719F0883509F0FE
:10D1D0001FCFD30111969C9082E090E0680E791EDB
:10D1E00060E170E06D8B7E8B13CFD3019D903D018C
:10D1F00005CF21E030E02F8B388FF30191903F0174
:10D20000FDCEC701B6016E960FB6F894DEBF0FBE15
:10D21000CDBFDF91CF911F910F91FF90EF90DF90E5
:10D22000CF90BF90AF909F907F906F905F904F9006
:10D230003F902F900895DC015C91552341F05F7D74
:10D2400051341CF05B350CF45C931196F5CF0895C6
:10D250002F923F924F925F926F927F928F929F9206
:10D26000AF92BF92CF92DF92EF92FF920F931F93F4
:10D27000CF93DF93CDB7DEB762970FB6F894DEBFDA
:10D280000FBECDBFAA24BB2465014C016D877E87EC
:10D290004F87588B44245524FC0146825782838152
:10D2A00081FD5BC28FEF9FEF6FC240FE44C2862DAF
:10D2B00080538A30E0F4F0E36F1641F42A89222388
:10D2C00029F4772019F480E091E08BC08AE09A89F4
:10D2D000989F902D1124892F860D80538A8B882347
:10D2E00014F4EFE7EA8B43FC38C27A8836C243FE77
:10D2F00005C0FA89FF2311F421E02A8B862D992796
:10D3000087FD90958836910554F5853691050CF08A
:10D310006BC08835910509F4D3C089359105B4F403
:10D320008B32910509F442C08C32910544F480326D
:10D33000910509F43FC0839709F442C0F2C18D32D0
:10D340009105D9F18E9709F440C0EBC18336910560
:10D3500009F454C08436910509F478C0E2C18037DD
:10D36000910509F4A5C08137910584F48C369105A7
:10D37000B1F18D3691052CF48936910509F466C01A
:10D38000D0C18F36910509F490C0CBC18537910586
:10D3900009F498C08637910524F483379105B9F1D3
:10D3A000C0C18837910509F48BC0BBC180E190E012
:10D3B000482A592AE0E2F0E005C080E890E011C078
:10D3C000E0E4F0E04E2A5F2AC8C188E090E0482AF5
:10D3D000592AEFEFFEEF4E225F221A8ABEC184E087
:10D3E00090E0482A592AB9C10F2EFFE3AF2EF02D45
:10D3F0007A940F2EF3E66F2EF02D3AC1EF85F8895F
:10D40000CF0102968F87988BA0807A9431C1EF85E7
:10D41000F889CF0102968F87988BA080B18043FE58
:10D420000BC0EA898E2F992787FD9095BC01C50115
:10D430000E94626C898B07C0F50101900020E9F71A
:10D440003197EA19E98BF9897F1A12C142FE0BC0A4
:10D45000EF85F889CF0104968F87988B20813181E1
:10D46000428153810DC0EF85F889CF0102968F87E5
:10D47000988B808191819C01442737FD4095542FE2
:10D4800059016A01552364F4E2E0F0E04E2A5F2A74
:10D49000D094C094B094A094A11CB11CC11CD11C08
:10D4A0008FEB9FEF482259222BC098E0998B0AC03E
:10D4B000E0E4F0E04E2A5F2A0F2EF8E76F2EF02D01
:10D4C000F0E1F98B42FE0BC0EF85F889CF0104969D
:10D4D0008F87988B20813181428153810BC0EF85EA
:10D4E000F889CF0102968F87988B808191819C016A
:10D4F0004427552759016A01EFECFFEF4E225F22C6
:10D500001E010894211C311CF989EF2EFF240027ED
:10D510001127C601B501A80197010E94F66CDC0134
:10D52000CB01F10180838A301CF0860D815203C04B
:10D53000F1018081805DF10181931F01C601B50178
:10D54000A80197010E94F66C59016A012115310565
:10D5500041055105F1F6CE010196A22CA81AC2018F
:10D5600082739070892B09F07A9446FE0FC0872D44
:10D57000992787FD9095F989F03131F40F2EFEEF50
:10D580007F2EF02D780E02C0782E7A9443FE12C0C2
:10D590008A89282F332727FD30958A2D99278217CE
:10D5A00093072CF0E7EFFFEF4E225F2203C0FA89CA
:10D5B000FA19FA8B43FE03C02A89721A01C07A183D
:10D5C000C20180789170892B69F4872D7A9418169E
:10D5D0004CF4B40180E290E00E942F6C872D7A9485
:10D5E0001816BCF341FE04C0B4018DE290E00BC0FC
:10D5F00044FE04C0B4018BE290E005C045FE05C0C6
:10D60000B40180E290E00E942F6C46FE0FC0B4018E
:10D6100080E390E00E942F6C8989803139F4862D57
:10D62000992787FD9095B4010E942F6C50FE0DC084
:10D63000872D7A9418164CF4B40180E390E00E9490
:10D640002F6C872D7A941816BCF343FE11C08A897B
:10D65000982F91509A8B18165CF4B40180E390E0F7
:10D660000E942F6C8A89E82FE150EA8B1816ACF3E0
:10D67000842D807869F4872D7A9418164CF4B401BF
:10D6800080E290E00E942F6C872D7A941816BCF3EC
:10D69000F3E66F1641F48A2D992787FD9095B40122
:10D6A0000E942F6C2DC023E76216B1F48989815046
:10D6B000898B8F3F29F1F5018081992787FD90950E
:10D6C0000894A11CB11CB4010E942F6C998991503F
:10D6D000998B9F3F81F714C0CE0101962816390619
:10D6E00079F08E010F5F1F4FF10182911F01992781
:10D6F00087FD9095B4010E942F6C20163106A1F78A
:10D70000842D8078A9F0872D7A9418168CF4B401B2
:10D7100080E290E00E942F6C872D7A941816BCF35B
:10D7200007C0862D992787FD9095B4010E942F6C24
:10D730004424552412C0F5E26F1641F444245524C4
:10D7400043941A8A7A882AE0298B07C0862D992764
:10D7500087FD9095B4010E942F6CF401838183FFB3
:10D7600008C0ED85FE85CF0101968D879E87649068
:10D7700005C0ED85FE856190ED87FE87662009F086
:10D7800094CDF4018681978162960FB6F894DEBF3E
:10D790000FBECDBFDF91CF911F910F91FF90EF9002
:10D7A000DF90CF90BF90AF909F908F907F906F90C1
:10D7B0005F904F903F902F9008950F931F93CF93BA
:10D7C000DF93CDB7DEB72C970FB6F894DEBF0FBE50
:10D7D000CDBF8C0136E03C8389839A832FEF3FE7EE
:10D7E0002D833E83CE0101960E942869AF81B885C2
:10D7F000A00FB11F1C922C960FB6F894DEBF0FBE7F
:10D80000CDBFDF91CF911F910F9108950F931F937B
:10D81000CF93DF93CDB7DEB72C970FB6F894DEBF6A
:10D820000FBECDBF8C013EE03C8389839A832FEFEE
:10D830003FE72D833E83CE0101960E942869AF8188
:10D84000B885A00FB11F1C922C960FB6F894DEBFBE
:10D850000FBECDBFDF91CF911F910F9108950F9310
:10D860001F93CF93DF938C01EB018B81992781FF6D
:10D8700022C082FF14C02E813F814C815D8124171C
:10D8800035073CF4A881B9810D93A883B9832E8113
:10D890003F812F5F3F4F2E833F83C8010EC0E88535
:10D8A000F985802F0995892B31F4EE81FF8131961E
:10D8B000EE83FF83F2CF8FEF9FEFDF91CF911F9128
:10D8C0000F910895FC016150704001900110D8F74C
:10D8D000809590958E0F9F1F0895629FD001739F32
:10D8E000F001829FE00DF11D649FE00DF11D929FFC
:10D8F000F00D839FF00D749FF00D659FF00D99273B
:10D90000729FB00DE11DF91F639FB00DE11DF91F5E
:10D91000BD01CF0111240895991B79E004C0991F1E
:10D92000961708F0961B881F7A95C9F78095089579
:10D9300097FB092E07260AD077FD04D00CD006D01D
:10D9400000201AF4709561957F4F0895F6F7909531
:10D9500081959F4F0895AA1BBB1B51E107C0AA1FC9
:10D96000BB1FA617B70710F0A61BB70B881F991F80
:10D970005A95A9F780959095BC01CD01089585FD34
:10D9800017C080629923A1F4813694F08B3784F418
:10D990000895992369F4803269F0893059F08B3009
:10D9A00039F408958F93EDDF8F9109F08062089527
:10D9B0009927882708959923D9F780958078089525
:10D9C0009923B1F78033A4F38A3394F70895992308
:10D9D00079F7803279F38A3069F38C3059F38D30DE
:10D9E00049F3893039F38B3019F70895A1E21A2EE3
:10D9F000AA1BBB1BFD010DC0AA1FBB1FEE1FFF1FF3
:10DA0000A217B307E407F50720F0A21BB30BE40B42
:10DA1000F50B661F771F881F991F1A9469F7609589
:10DA20007095809590959B01AC01BD01CF01089543
:10DA300097FB092E05260ED057FD04D0D7DF0AD05C
:10DA4000001C38F450954095309521953F4F4F4F2D
:10DA50005F4F0895F6F790958095709561957F4F8B
:06DA60008F4F9F4F089557
:10DA66005A7A41003F004800484C00485400484656
:10DA7600002E0053544F50002100474F0048414CA0
:10DA860054004C004C4300460046580054005900D0
:10DA960056004D5400535200535300534500404026
:10DAA600004200534F000001E03C0401B935060175
:10DAB600B9350801A4350B01AB350E01B23511019C
:10DAC600F8351301F83518010D361A010D361D010A
:10DAD6002236220144362401CE372701FF37290199
:10DAE60048392C019E3A2E01CD3530014E3B32018C
:10DAF600743B3501BF3B3801EE3B3B01543C3E01D4
:10DB060086544101813C4301B23C0000000080057F
:10DB1600C3308105C8308403CD308503FC308804CA
:10DB2600263189044D318C0378318D039131900370
:10DB3600AF3194031E32950257329802733299011F
:10DB460096329C029B329D03BE32A001E532A201B1
:10DB56004233A4035933A5017D33A6018633A701B9
:10DB66008C33C4019233C602373EC7032D3EC8012B
:10DB76009533C901D233CA011434CB01AD34000048
:10DB8600000000010000FF00020000FF00000A4B39
:10DB9600FF00030000FF00001D4CFF00000644FFCD
:10DBA6000000E140FF00002741FF0100DD42FF01C8
:10DBB600003941FF01000642FF0100B543FF0200A4
:10DBC6001047FF02007F46FF02009447FF0200F362
:10DBD60047FF02002347FF02003647FF02003E468A
:10DBE600FF03040000FF0300B94B13030500001AEE
:10DBF6000300C84AFF030600001A03000049FF039A
:10DC0600000549FF04005D4DFF0400B74DFF050008
:10DC16000A49FF0500014DFF06002349FF0600746F
:10DC260049FF0600C04AFF0600C44AFF2534642D9A
:0ADC36002534643A20002534640010
:00000001FF
